:1000000000600020D9F70100ADF90100ADF9010051
:10001000ADF90100ADF90100ADF90100ADF9010044
:10002000ADF90100ADF90100ADF9010091F1010058
:10003000ADF90100ADF9010061F20100B1F201007A
:10004000ADF90100ADF90100ADF90100ADF9010014
:10005000ADF9010061DB0100ADF90100D5F201004D
:10006000ADF90100ADF90100ADF90100ADF90100F4
:1000700025E901001DEA0100ADF90100ADF901001B
:10008000ADF90100ADF90100ADF90100ADF90100D4
:10009000ADF90100ADF90100ADF90100ADF90100C4
:1000A000ADF90100ADF90100ADF90100ADF90100B4
:1000B000FDE20100ADF90100ADF90100ADF901006B
:1000C000FFFFFFFFFFFFFFFFFFFFFFFFFFFFFFFF40
:1000D000FFFFFFFFFFFFFFFFFFFFFFFFFFFFFFFF30
:1000E000FFFFFFFFFFFFFFFFFFFFFFFFFFFFFFFF20
:1000F000FFFFFFFFFFFFFFFFFFFFFFFFFFFFFFFF10
:1003E000FFFFFFFF606A0200FFFFFFFFFFFFFFFF4D
:1003F000FFFFFFFFFFFFFFFFFFFFFFFFFFFFFFFF0D
:10040000FFFFFFFFFFFFFFFFFFFFFFFF7E3BFFFF41
:020000021000EC
:1000000010B5064C2378002B07D1054B002B02D0EE
:10001000044800E000BF0123237010BDF4E0FF1F7F
:10002000000000004469020008B5084B002B03D013
:100030000748084900E000BF07480368002B03D0C9
:10004000064B002B00D0984708BDC04600000000BA
:1000500044690200F8E0FF1FF0E0FF1F000000000D
:10006000164B002B00D1144B9D46402292029A1A47
:10007000924600218B460F461348144A121A12F07A
:10008000DAFA0F4B002B00D098470E4B002B00D014
:1000900098470020002104000D000D48002802D0E0
:1000A0000C4800E000BF12F06FFA200029000EF0AB
:1000B000F1F812F053FAC04600000800006000207A
:1000C0000000000000000000F4E0FF1FF0F6FF1F3A
:1000D0000000000000000000002934D001230022AD
:1000E00010B488422CD301242407A14204D28142B7
:1000F00002D209011B01F8E7E400A14204D28142C7
:1001000002D249005B00F8E7884201D3401A1A4343
:100110004C08A04202D3001B5C0822438C08A0427A
:1001200002D3001B9C082243CC08A04202D3001B30
:10013000DC082243002803D01B0901D00909E3E7AA
:10014000101C10BC7047002801D00020C04307B429
:10015000024802A14018029003BDC046D900000029
:100160000029F0D003B5FFF7B9FF0EBC4243891A4E
:100170001847C046002941D010B4041C4C40A44686
:1001800001230022002900D54942002800D5404221
:1001900088422CD301242407A14204D2814202D2F6
:1001A00009011B01F8E7E400A14204D2814202D216
:1001B00049005B00F8E7884201D3401A1A434C0813
:1001C000A04202D3001B5C0822438C08A04202D349
:1001D000001B9C082243CC08A04202D3001BDC0871
:1001E0002243002803D01B0901D00909E3E7101CB2
:1001F0006446002C00D5404210BC7047002806D051
:1002000003DB0020C043400801E08020000607B463
:10021000024802A14018029003BDC0461900000028
:100220000029EBD003B5FFF7A7FF0EBC4243891AA4
:100230001847C0467047C0468446101C62468C462C
:10024000191C634600E0C0461FB501F0E9FE002816
:1002500001D40021C8421FBD10B501F019FE404273
:10026000013010BD10B501F0DBFE002801DB0020DD
:1002700010BD012010BDC04610B501F0D1FE002810
:1002800001DD002010BD012010BDC04610B501F0F9
:1002900049FE002801DC002010BD012010BDC04631
:1002A00010B501F03FFE002801DA002010BD01204A
:1002B00010BDC0468446081C6146FFE71FB500F02C
:1002C000E9FB002801D40021C8421FBD10B500F091
:1002D0006FFB4042013010BD10B500F0DBFB002881
:1002E00001DB002010BD012010BDC04610B500F09C
:1002F000D1FB002801DD002010BD012010BDC0464B
:1003000010B500F07FFB002801DC002010BD0120AB
:1003100010BDC04610B500F075FB002801DA0020C2
:1003200010BD012010BDC046002B11D1002A0FD1F5
:10033000002900D1002802D00021C943081C07B4BD
:10034000024802A14018029003BDC046E9FEFFFF2B
:1003500003B4684601B5029800F07EF8019B9E4602
:1003600002B00CBC7047C0469C460304F0B51B0CA1
:1003700017043F0C150C1E1C041C000C7E436B4321
:1003800047434543FB18300C1818874202D9802395
:100390005B02ED18030CED1863465C434A433604D8
:1003A000360CA118000480194919F0BD9E2110B522
:1003B000C905041CFFF7AEFF002803D1201C00F084
:1003C00055FE10BD9E21C905201C00F0D9FC00F08F
:1003D0004DFE80231B06C018F3E7C0460000000056
:1003E00038B50E4B0C4A041C0D1CFFF759FF0028B2
:1003F00004D1201C291C02F055FC38BD074B064ACD
:10040000201C291C02F01AF902F04CFC80231B0668
:10041000C018F2E7C046C046000000000000E041FE
:10042000F0B583B0161C1F1C0090019102F050FD26
:10043000041C0D1C221C2B1C301C391CFFF794FFC4
:10044000009A019B121A8B410899201C0A604B608C
:10045000291C03B0F0BDC046F0B583B0141C1D1CB0
:100460000090019102F010FF221C2B1C061C0F1C97
:10047000FFF77AFF009A019B121A8B410899301CF2
:100480000A604B60391C03B0F0BDC046F8B54302AA
:100490004400C50F4E024800240E2A1C9B09000E82
:1004A000C90FB6098D425BD0221A002A00DC89E010
:1004B00000281DD1002E00D075E0580704D00F226F
:1004C0001A40042A00D004338021C90419402A1C90
:1004D00000293AD00134FF2C00D17FE09B015B0A58
:1004E0005B02E4B2E405580AD20720431043F8BD8A
:1004F000FF2CE2D08021C9040E431B2A00DD2DE130
:10050000311C2020D140821A9640721E96410E4323
:100510009B1B5801D1D59B019F09381C02F0BAFCE6
:10052000421F974094425BDC141B1F231B1B3A1C89
:100530009F40611C3B1CCA405F1EBB41134300240B
:10054000BBE7131EB9D100230022DB08FF2C04D126
:10055000002B43D08020C00303435B025B0ABFE74C
:10056000211A002940DD002823D0FF2CA5D08020AF
:10057000C00406431B2900DDEEE0301C2027C840E4
:10058000791A8E40711E8E4106439B19590100D481
:1005900093E70134FF2C55D0714901221A400B40DA
:1005A0005B08134389E7013A002AB1D0FF2CA4D19C
:1005B00083E7002E00D180E701390029E5D0FF2C28
:1005C000D8D17AE7002A1BD1621CD2B2012A4BDDB6
:1005D0009F1B7A0123D5F71A0D1C9EE700237FE7A6
:1005E0005F4BA41A3B4068E7002946D1611CC8B2A2
:1005F000012829DDFF2924D0F3185B080C1C5CE7D7
:10060000002C13D0FF2818D08024E4045242234346
:100610001B2A4DDD0123F31A041C0D1C79E7002F62
:1006200000D07AE70023002200248EE7002B3BD085
:10063000D243002AEFD0FF28EAD1331CFF240D1C3F
:100640003BE7FF24002380E7002C5CD1002B00D186
:1006500080E0002E00D130E79B19580100D42CE730
:100660003F4A0124134028E7002C15D1002B40D12C
:10067000002E63D0331C0D1C1FE7002C21D1002B52
:1006800054D0C943002904D0FF284CD01B2958DD81
:1006900001239B19041C79E7002B19D1002E48D0A7
:1006A000331C0D1CFF2408E7331C041C0D1C04E73D
:1006B0001C1C2025D440AA1A93405A1E9341234360
:1006C000A9E7FF282FD08024E40449422343DDE733
:1006D000FF24002E00D1F0E68022DB08D203134273
:1006E00004D0F608164201D1331C0D1CDB00FF2498
:1006F000E3E6002E00D1E0E69A1B500100D420E78B
:10070000F31A0D1CD9E6002B0DD0FF24002E00D1CA
:10071000D3E68022DB08D2031342E7D0F608164264
:10072000E4D1331CE2E7331CFF24C6E6331C041C6F
:10073000C3E6802300229B04FF2406E7231C00223B
:1007400003E71C1C2027CC40791A8B40591E8B4193
:1007500023439EE7331CB0E6012616E70126D7E6C1
:10076000FFFFFFFBF0B55F4656464D464446F0B4EA
:1007700046024500C00F85B00F1C760A2D0E80463C
:1007800041D0FF2D26D08024240400212643F600EA
:100790007F3D89468B46F90F7C027800640A000E83
:1007A00000918A463CD0FF2834D080231B041C4390
:1007B0000023E4007F380193009F4346019A7B4069
:1007C00049469C4611430F2900D971E0764F8900B4
:1007D0007F58BF46002E3ED10822022391469B46F9
:1007E000D9E75A46341CC24601920199022937D0F2
:1007F000032900D1CFE0012900D0ABE053460B40E4
:100800000022002632E0002E19D10421012289465F
:100810009346C0E7221C531E9A4102320192CBE755
:1008200001270197002CC7D0201C02F033FB431F87
:100830009C4076235B420021181A0191BCE7301CD2
:1008400002F028FB7625431F9E406D4200232D1A9F
:1008500099469B469FE70C23032199468B469AE7CE
:10086000D446012367463B40FF2200267602D2058C
:10087000700ADB071043184305B03CBC904699460C
:10088000A246AB46F0BD80260023F603FF22EDE72B
:1008900000220026EAE78020C00306423BD0044243
:1008A00039D1061C26437602760A009BFF22DDE73B
:1008B000281A039076016401A64239D3361B1A2206
:1008C00001230120311C5B007600002901DBB442CA
:1008D00001D8361B0343013A002AF3DC741EA641FB
:1008E000341C1C43039A7F32002A27DD630704D09F
:1008F0000F232340042B00D00434270103D52B4BB6
:10090000039A1C408032FE2A0BDD012361460B4016
:10091000FF220026AAE706437602760A4346FF2214
:10092000A4E7A40101236746660AD2B23B409DE7D3
:10093000039F1B22013F03970023C2E77E23039FEF
:100940005B42DB1B1B2B07DD012361460B400022B2
:1009500000268BE7D446C5E7221CDA40039B9E3372
:100960009C40231C5C1EA34113435A0704D00F2252
:100970001A40042A00D004335F0105D501236146E3
:100980000B400122002671E79E01624601231340BD
:10099000760A00226AE78026F60326437602760A64
:1009A0005346FF2262E7C04698270200FFFFFFF789
:1009B0004A02430270B55C0A550A43004A001B0E06
:1009C000C60F120EC90FFF2B05D0FF2A08D0012039
:1009D00093420BD070BD0120002CFBD1FF2AF6D131
:1009E0000120002DF6D101209342F3D1AC42F1D188
:1009F0008E4205D0002BEDD1201C441EA041E9E71A
:100A00000020E7E74A024302F0B55C0A550A4300BA
:100A10004A001B0EC60F120EC90FFF2B31D0FF2A42
:100A200034D0002B16D1604260418446002A14D095
:100A3000002820D18E4217D1934215DC04DBAC4252
:100A400012D80020AC4212D27042704140420123C1
:100A500018430CE0002AEDD194466F426F41604686
:100A6000002805D1002FE5D0704201231843F0BDC6
:100A70000020002FFBD14842484140420123184347
:100A8000F5E7002CCBD002204042F0E7002DC8D083
:100A9000F9E7C0464A024302F0B55C0A550A430032
:100AA0004A001B0EC60F120EC90FFF2B27D0FF2ABC
:100AB00029D0002B10D0002A15D194466F426F41E7
:100AC0006046002815D00020002F04D1484248413C
:100AD000404201231843F0BD604260418446002A31
:100AE000ECD00028F2D18E4211D07042012318437D
:100AF000F1E7002FF7D0704201231843EBE7022003
:100B0000002CE8D1D3E70220002DE4D1D1E79342B5
:100B1000EBDC04DBAC42E8D80020AC42DBD2704214
:100B20007041404201231843D5E7C046F0B55F4607
:100B300056464D464446F0B44402460083B00F1C6E
:100B4000640A360EC50F002E41D0FF2E22D080231E
:100B50001B0400201C43E4007F3E82468046391C73
:100B60004B007F02C90F7F0A1B0E8B463BD0FF2B29
:100B700034D0802212041743FF007F3B00215A46E5
:100B80006A40019252460A430F2A63D87A4892007B
:100B900082589746002C3FD108220223924698465D
:100BA000DDE70195404602282AD1019A012515402A
:100BB000FF2300246402DB05600AED071843284385
:100BC00003B03CBC90469946A246AB46F0BD002C13
:100BD00027D10420012282469046C0E7391C4A1ED4
:100BE00091410231CBE70121002FC8D0381C02F01F
:100BF00051F9431F9F4076235B421B1A0021BEE739
:100C0000032800D1AEE001284FD1019842461040A0
:100C1000C5B200230024CDE70C2303209A4680466A
:100C20009DE7201C02F036F97626431F9C40764251
:100C30000023361A9A46984691E780240025E4035B
:100C4000FF23B7E75B463C1C01938846AAE73C1CA0
:100C50008846A7E7250C24043A0C240C3F04F61818
:100C60003F0C211C231C794353436F435543FB180E
:100C70000A0C9B18B1469F4202D980225202AD183D
:100C800009041A04090C521894011B0C611E8C41B2
:100C9000920EED181443AD012C43230105D501221A
:100CA00063080120144081441C434B467F33002BD2
:100CB0002DDD600704D00F222240042A00D0043426
:100CC000220103D52D4B1C404B468033FE2B17DDF4
:100CD000019B01251D400024FF236BE78020C003FA
:100CE000044208D0074206D1041C3C436402640A53
:100CF0005D46FF235EE704436402640AFF2359E76D
:100D00000198A4010125640ADBB2054052E77E2365
:100D10005B424A469B1A1B2B05DD019B01251D40AA
:100D20000024002346E7221CDA404B469E339C40B9
:100D3000231C5C1EA3411343580704D00F221A4002
:100D4000042A00D004335A0105D5019B01251D401A
:100D5000002401232EE701989C010125640A054027
:100D6000002327E78027FF03019B3C436402012502
:100D70001D40640AFF231DE7D8270200FFFFFFF78D
:100D8000F8B5C20F430244004D024800240E161C61
:100D90009B09000EC90FAD09FF2800D183E0012790
:100DA00079408A425CD0221A002A00DC8EE00028BA
:100DB0001ED1002D00D07AE0580704D00F221A402F
:100DC000042A00D004338021C90401221940324092
:100DD00000293AD00134FF2C00D183E09B015B0A4B
:100DE0005B02E4B2E405580AD20720431043F8BD81
:100DF000FF2CE1D08021C9040D431B2A00DD31E125
:100E0000291C2020D140821A95406A1E95410D432D
:100E10005B1B5801D0D59B019F09381C02F03AF8A2
:100E2000421F974094425FDC141B1F231B1B3A1C7C
:100E30009F40611C3B1CCA405F1EBB411343002402
:100E4000BAE7131EB8D100230022DB08FF2C04D11F
:100E5000002B47D08020C00303435B025B0ABFE73F
:100E6000211A002944DD002827D0FF2CA4D080209F
:100E7000C00405431B2900DDF2E0281C2027C840E0
:100E8000791A8D40691E8D4105435B19590100D4C3
:100E900092E70134FF2C59D0734901221A400B40CC
:100EA0005B08134388E7002D00D07AE777E7013A23
:100EB000002AADD0FF2CA0D17EE7002D00D17BE72A
:100EC00001390029E1D0FF2CD4D175E7002A1BD1CC
:100ED000621CD2B2012A4BDD5F1B7A0123D5EF1AC7
:100EE0000E1C9AE700237BE75F4BA41A3B4063E7A5
:100EF000002946D1611CC8B2012829DDFF2924D070
:100F0000EB185B080C1C57E7002C13D0FF2818D0F7
:100F10008024E404524223431B2A4DDD0123EB1AB3
:100F2000041C0E1C75E7002F00D076E7002300227A
:100F300000248AE7002B3BD0D243002AEFD0FF28C1
:100F4000EAD12B1CFF240E1C36E7FF2400237CE78C
:100F5000002C5CD1002B00D180E0002D00D12BE7CC
:100F60005B19580100D427E73F4A0124134023E7C7
:100F7000002C15D1002B40D1002D63D02B1C0E1C52
:100F80001AE7002C21D1002B54D0C943002904D0EA
:100F9000FF284CD01B2958DD01235B19041C75E781
:100FA000002B19D1002D48D02B1C0E1CFF2403E769
:100FB0002B1C041C0E1CFFE61C1C2026D440B21A5D
:100FC00093405A1E93412343A9E7FF282FD0802442
:100FD000E40449422343DDE7FF24002D00D1EBE682
:100FE0008022DB08D203134204D0ED08154201D160
:100FF0002B1C0E1CDB00FF24DEE6002D00D1DBE6FF
:101000005A1B500100D41CE7EB1A0E1CD4E6002B2F
:101010000DD0FF24002D00D1CEE68022DB08D203C4
:101020001342E7D0ED081542E4D12B1CE2E72B1C5C
:10103000FF24C1E62B1C041CBEE6802300229B0477
:10104000FF2402E7231C0022FFE61C1C2027CC40C3
:10105000791A8B40591E8B4123439EE72B1CABE62C
:10106000012512E70125D3E6FFFFFFFB4302590AE2
:101070004300C20F1B0E00207E2B0DDD9D2B0CDCD0
:10108000802000040143952B0ADC9620C31AD94026
:101090004842002A00D1081C7047034BD018FBE7D8
:1010A000963B9940F4E7C046FFFFFF7F70B5041EF2
:1010B0003CD0C60F00D04442201C01F0EBFE9E2322
:1010C000251C1B1A962B0CDC083884406402640A29
:1010D000DBB2321C6402DB05600AD20718431043FE
:1010E00070BD992B0ADD0522121A211CD1400A1C61
:1010F000011C1B318D40691E8D411543052801DD02
:10110000421F9540164C2C406A0704D00F22154010
:10111000042D00D0043461010CD59F23181AFF2838
:101120001AD0A401640AC3B2321CD3E70022002300
:101130000024CFE7E408FF2B04D06402640ADBB28A
:10114000321CC7E7002C04D08020C0030443640293
:10115000640A321CFF23BDE7321CFF230024B9E7D9
:10116000FFFFFFFB10B5041E33D001F093FE9E235A
:101170001B1A962B09DC083884406402640ADBB22F
:101180006402DB05600A184310BD992B0ADD0522B5
:10119000121A211CD1400A1C011C1B318C40611EFB
:1011A0008C411443052801DD421F9440144A22401B
:1011B000610704D00F210C40042C00D004325101EF
:1011C0000AD59F23181AFF2816D09401640AC3B2C7
:1011D000D6E700230024D3E7D208FF2B03D0540224
:1011E000640ADBB2CCE7002A06D08024E40314436F
:1011F0006402640AFF23C3E7FF230024C0E7C0465C
:10120000FFFFFFFBF8B55F46564644464D46F0B437
:101210000C034D00CE0F610A440F2143C400180394
:1012200080465800400D8246D80F84464046400A0A
:10123000530F0343D0006D0D371C8346524666455D
:1012400000D1A4E0AF1A002F00DC09E1002A3BD155
:10125000184300D0EAE0630700D187E00F23234062
:10126000042B00D182E0221DA242A44164428023CB
:1012700009191B040B40371C141C002B00D17CE007
:10128000CE4B01359D4200D105E1CD4BE40819401C
:101290004807490204430B0B002000211B031A0BD3
:1012A0000B0D6D051B0513436A08C64DFF071D4056
:1012B00015436D006D08291C3943201C3CBC904629
:1012C0009946A246AB46F8BDBC488542C3D08020B3
:1012D00000040343382F00DDF0E01F2F00DD24E180
:1012E0002020C01B1A1C814682405846F840024309
:1012F000944658464A469040421E9041FB40624602
:1013000002431F1CA21A9442A4416442C91B091B38
:10131000141C0B029FD549024F0A002F00D1C8E0D0
:10132000381C01F0B7FD021C083A1F2A00DDB5E0A9
:101330002821091A201C9740C84007439440954231
:1013400000DDB2E0551B691C1F2900DDDCE01F2217
:10135000551B3B1C221CAB40CA40AC40651EAC4137
:101360001343CF401C43391C002574E780231B0422
:101370000B40371C002B00D082E7904B4807E40855
:101380000443C9089D4248D009030B0B84E7AA1AFD
:101390009446002A00DC98E05046002852D0874846
:1013A000854200D157E78020000403436246382A73
:1013B00000DDFCE01F2A00DD4AE120226046101A11
:1013C0001A1C82408246914658466246D0404A46A0
:1013D00002439046584652469040421E9041424633
:1013E00002436046C3401219A242A4416442591804
:1013F0000919141C080200D42DE7704B01359D42D9
:1014000000D122E16E4B60081940012323401C1CCF
:101410000443CB071C4349081DE7231C0B433AD068
:1014200080231B030B431B031B0B35E7013F002FDE
:1014300065D15846221A9442A4416442C91A091B34
:10144000141C66E75846184300D104E701225242B3
:1014500094446046002800D0C5E058460219C3E70E
:10146000002F73D1681C4005400D012800DCDEE030
:101470005A46A21A9442BF41C81A7F42C71B38027B
:1014800000D489E05A46141BA3459241591A52428E
:101490008F1A664641E700230024FDE6271C283802
:1014A00087400024954200DC4CE74549AD1A39409D
:1014B000D1E6201C01F0EEFC203034E75A461A43F6
:1014C000531E9A41D2B200271CE7002A00D0DCE06C
:1014D000681C4205520D012A00DC8DE0374DA84200
:1014E00000D1F3E05D462A19A242A4416442591892
:1014F0000919CC07520814434908051CABE62F48CC
:10150000854200D0E6E6A6E62B1C1F3B3A1CDA40DB
:10151000131C20296CD03F22551BAF403C43601E5A
:1015200084411C430021002595E6381C20381A1CF4
:10153000C240101C202F5DD04022D71BBB405A4612
:101540001A43531E9A4102430027DBE6002D3BD08D
:101550001A4DAA4500D193E080252D047F422943EE
:10156000382F00DDACE01F2F00DD29E12025ED1B29
:10157000081C261CA840FE40AC400643651EAC413A
:101580003443F9405D462C1BA34592415B1A5242FD
:10159000991A55466646BCE6131C3B43141C002BA7
:1015A00000D0BAE60027002100250024E5E65A46CF
:1015B0001A43531E9A41D2B2002314E7FF070000DA
:1015C000FFFF7FFFFFFF0F800D1C254358D0FF4317
:1015D000002F51D1041BA3459241591A5242891A36
:1015E0005546664695E69648854200D0DEE632E6E8
:1015F000002793E70023A2E7081C2043002D00D01A
:10160000C4E0002800D1F7E05846184300D122E694
:1016100058460219A242A441644259180919141CDF
:101620000A0200D417E6874B0125194013E6081C6F
:101630002043002D39D1002871D15946194303D0D8
:10164000191C5C46664606E600270021002494E645
:10165000604620381A1CC24060469146202800D1BE
:10166000ACE04022121A93405A461A43531E9A4144
:101670004B461A430023B6E6714DAA4500D06FE7EA
:10168000191C5C4655466646E5E5002D22D10D1C29
:10169000254377D0D543002D71D15C445C45924100
:1016A0005918524289185546A4E600284DD159468A
:1016B000194300D194E0191C5C466646604DCAE5AA
:1016C0000C43611E8C41E4B200215BE7051C002144
:1016D000002452E65A4DAA4554D0554280221004A7
:1016E0000143382D00DD81E01F2D00DD92E0202236
:1016F000501B0A1C84468240201CE840024390464E
:1017000062469440601E844142461443E9405C4472
:101710005C459241CB185242991855466AE65846A4
:10172000184300D197E55846271ABC429241C81A7F
:101730005242801A020266D55846041BA3459241C4
:10174000591A5242891A664685E55846184333D0DD
:101750004807E40804438020C9080003014208D078
:10176000DD08054205D15946CA085C071443291C07
:101770006646630FC9001943E400314D6BE5304AFA
:101780009245AED1191C5C46554664E5002836D01A
:101790005846184310D080254807E408C9082D038F
:1017A00004432942E5D0D8082842E2D15D46EA0840
:1017B0005C071443011CDCE7214D4CE5002353E793
:1017C0003D1C203D0A1CEA40151C202F34D0402629
:1017D000F71BB9400C43611E8C412C430021D1E61C
:1017E00080210027C903164D0024C6E50C43611E65
:1017F0008C41E4B200218AE7191C5C462BE5191CD8
:101800005C460F4D27E5031C3B4300D11CE7011C40
:101810003C1C20E52020404240190A1CC240904652
:10182000202D0BD04020451BA9400C43611E8C414C
:1018300045462C4300216AE70021CBE70021F4E76D
:10184000FF070000FFFF7FFFF0B5564644465F46A6
:101850004D46F0B41F1C0B031B0B98464B0087B082
:10186000041C81465B0DC80F161C9A460090002B85
:1018700051D06A4B9A4531D08022414652030A43E7
:10188000630FD2001A43664B90460025E200914652
:101890009A44002402953B031B0B9B46FD0F7B00E3
:1018A000311C5B0D019560D05C4A934254D080217D
:1018B000584649030143720FC9001143584A8B46E9
:1018C0009B18F1000020009A04436A4003920F2CF9
:1018D00000D9ADE0534EA4003459A7464046044316
:1018E0006ED1002102250824884689460295D2E758
:1018F000009C0298C34649460194022864D00328FC
:1019000000D1ABE2012800D038E2019A0024024065
:101910000025A14660E0434623434AD040460028C4
:1019200000D1C0E101F0B6FA031E272B00DDB3E1C0
:1019300028210D1A211C083B4246E9409A400D1C03
:101940001543221C9A40A8469146374B00251B1A86
:101950009A46002402959EE75A4616430320002E1D
:10196000B1D1B34600210220ADE75A4632431BD025
:101970005B46002B00D18AE1584601F08BFA2728FC
:1019800000DD7DE12822171A011C321C08395B4654
:10199000FA408B40171C1F43331C8B40BB46191C5D
:1019A000214B1B1A00208EE70027BB460021012097
:1019B00089E70020012504248046814602956AE7D4
:1019C00003250C24029566E7019C0394039D0122E4
:1019D0002A400024114DA146002000212403260B9B
:1019E0000C0D2405114B34432D0523402B435B0084
:1019F0005B08D207191C4846114307B03CBC90460F
:101A00009946A246AB46F0BD0022802424039146AD
:101A1000024DE1E700240025A146DDE7FF070000B5
:101A200001FCFFFF182802000DFCFFFFFFFF0F80E5
:101A30005546ED1A0495D84500D953E100D14EE141
:101A4000049C0025013C4E4604944746A94658464E
:101A500003020C0E1C430902250C23041B0C0091ED
:101A6000381C291C0193FEF737FB0199834641433B
:101A7000381C8A46291CFEF773FB330C09041943F2
:101A80008A450CD95B460919013B8C4200D947E1D4
:101A90008A4500D844E10222524293440919534630
:101AA000CB1A181C291C9846FEF716FB071C019838
:101AB000291C784382464046FEF752FB36040B044D
:101AC000360C33439A4509D91B197A1E9C4200D91A
:101AD00024E19A4500D821E1023F1B195E463204F9
:101AE0001743380CBB46009E009F51463F0C320402
:101AF0005B1A5946BA46120C0F043F0C90465146E9
:101B00007A434F434146414356467043CF19160C22
:101B1000BE19B14202D980277F02C019310C1204CC
:101B20003604120C4018B618834200D2C4E000D12B
:101B3000BEE0191A4846861BB145BF417F42CF1B04
:101B4000A74200D113E1291C381CFEF7C5FA019900
:101B500002904143381C8946291CFEF701FB330CD7
:101B60000904194389450CD9029B0919013B8C4290
:101B700000D9FFE0894500D8FCE0029F0919023F27
:101B800002974F46CF1B381C291C0597FEF7A4FA75
:101B9000071C0198291C784381460598FEF7E0FA56
:101BA00036040904360C0E43B14509D936197B1E9B
:101BB000B44200D9E0E0B14500D8DDE0023F36197B
:101BC000029D4946761A290439430B0457460A0CEC
:101BD0001B0C40464546584355437B437A43EB181C
:101BE000070CDB199D4202D980256D0252191D0C8C
:101BF00000041B04000C52191B18964235D300D167
:101C0000FCE001231943049E994FF519002D00DCD7
:101C1000A1E0480709D00F230B40042B05D00B1D72
:101C20008B42894149428B44191C5A46D20107D53F
:101C3000904B5C46049E80271C40FF00A346F5198C
:101C40008D4B9D427ADD039C0122224000248B4D66
:101C5000A146C1E680242403474627424CD13C4399
:101C60002403240B009A854DB6E63619481EB4426B
:101C70005ED9011C9642C4D1009E9E42C1D1C2E7EA
:101C8000031C283B311C99408B46002188E6301C00
:101C900001F000F9203072E6283B211C9940002217
:101CA0008846914651E6201C01F0F4F820303BE6CE
:101CB0000021B14500D33DE7009F5A46B944B945DC
:101CC000BF417F423F19FB18013A9C421ED2984205
:101CD00000D97EE000D1B5E0191A93462AE789457C
:101CE00000D8ADE64846464642467708D307460840
:101CF000C0071E438146AAE65846204212D104433B
:101D000024032A1C240B89465C4D65E6A342E3D1DB
:101D1000009F4F45DBD9211A93460BE7171CDDE6E0
:101D20009B46BCE63C432403240B009A534D53E6E8
:101D3000B24259D800D18AE0011C62E75F46C90867
:101D40007B07039E0B437C026D0501229946240B01
:101D50006D0D324040E64A4B049FDB1B382B10DDF3
:101D6000039C0122224000240025A14634E60121E3
:101D7000494248E7029304E71F1C21E7019C0394B2
:101D800041E71F2B40DC3F48049F0C1C3A18584683
:101D90009140DC40904020430A1C511E8A41011CA6
:101DA00011435A46DA40131C480709D00F220A4053
:101DB000042A05D00A1D8A42894149425B18111C38
:101DC0001A0234D5039C0122224000240125A14699
:101DD00002E6009F02214942B9448B44B94589413A
:101DE00049420919CB18A4E6009D881E6900A94242
:101DF000AD416D422C19361900913AE7002B00D005
:101E000033E70024009437E71F4A049C5D46121B09
:101E1000D5402A1C202B1FD01C4E5F46A3199F4083
:101E20003B1C19434B1E994111430023BCE75A0741
:101E3000C9080A43039F91465B0201221C0B3A40EA
:101E40000025C9E54E45C4D89346002172E6009F9F
:101E50009F42C9D3011C0FE70023E2E7802424033B
:101E60005F463C432403240B019A8946034DB3E5A6
:101E7000FF030000FFFFFFFEFE070000FF0700005A
:101E800002FCFFFF1E040000E2FBFFFF3E04000017
:101E9000F0B55F4656464D464446F0B40D1C041C52
:101EA0008046E80F814618030F03000B3F0B83B0F9
:101EB00084461B48009749005E00DF0F490D92469B
:101EC000760DBB4681420CD01548864210D00120C9
:101ED000B14215D003B03CBC90469946A246AB46F1
:101EE000F0BD009F01202743F4D10D488642EED17A
:101EF000604602430120002AECD10120B142E9D121
:101F0000009B6345E6D1D045E4D1D94506D00029F0
:101F1000E0D11C43201C441EA041DBE70020D9E790
:101F2000FF070000F0B55F4656464D464446F0B404
:101F3000CD0FDE0FAC461D032D0BB146374E0F0300
:101F40004C00AB465D0080463F0B640D92466D0D24
:101F5000B44232D0314EB54235D0002C0ED1384388
:101F600041424141081C002D0BD0002919D1CC451C
:101F70002DD0654668420123184318E0002DF6D1A4
:101F8000281C59460A4353425341002806D1002BCE
:101F9000EDD0634658420123184308E00020002B8F
:101FA00005D14A46504250414042012318433CBCAF
:101FB00090469946A246AB46F0BD3E1C0643C9D0AA
:101FC00002204042F3E75E461643C6D0F8E7AC4233
:101FD00007DC0BDA6146484248414042012318437E
:101FE000E5E76646704201231843E0E75F450AD8FB
:101FF0000ED000205F45DAD2654668426841404213
:1020000001231843D3E76246504201231843CEE729
:10201000D045F8D80020D045EED3C8E7FF07000030
:10202000F0B556464D4644465F46F0B40D1C83B0AD
:10203000041C0190E80F814618030F03000B3F0BAF
:1020400084463548009749005E00DF0F490D9246EF
:10205000760DB846814234D02F48864236D00029CA
:1020600018D0002E1FD1341C67463A4353425341C7
:10207000002C1FD00020002B05D142465042504179
:1020800040420123184303B03CBC90469946A24607
:10209000AB46F0BD0098044360426041041C002E32
:1020A000E2D00028E9D1C14515D04F46784201233E
:1020B0001843E8E7002BF6D04B465842012318435B
:1020C000E1E7009F02202743DDD1C5E767460220F4
:1020D0001743D8D1C3E7B14204DD4A465042012339
:1020E0001843D0E7B14207DB00986045E4D80AD036
:1020F000009F00206745C6D24F4678427841404253
:1021000001231843BFE7019A5245D5D8019A002010
:102110005245F1D3B7E7C046FF070000F0B5564679
:1021200044465F464D46F0B41F1C0B031B0B9A46FA
:102130004B0087B0041C80465B0DC80F161C029331
:102140008146002B68D0694B0299994232D0802297
:10215000534652031A43D200630F1A439246644A0D
:10216000E000891880460291002400253B031B0BE8
:102170009B467800FB0F321C400D039300D175E0A5
:102180005A4B984269D08022594652030A43730F32
:10219000D2001A43564B9346C018F200002303990D
:1021A0004E4671401C430F2C00D9A9E0514EA400AB
:1021B0003459A74653461C4300D087E00025AA4661
:1021C000A84608240225D1E74946022D6CD0032DEC
:1021D00000D117E2012D00D058E10D40EDB20024EE
:1021E000A9460023A0460020002125030A0D1C0556
:1021F0002D0B1205404B2A43134023435B004C46F2
:102200005B08E207191C4046114307B03CBC9046EE
:102210009946A246AB46F0BD5346234350D05346A1
:10222000002B00D184E1504600F034FE031E272B22
:1022300000DD76E128210D1A211C083B5246E940B9
:102240009A400D1C1543221C9A40AA4690462B4BDF
:1022500000241B1A0293002588E75B461E430323D4
:10226000002E9CD1B3460022022398E75B463343FD
:1022700021D05846002800D14EE100F00BFE27285F
:1022800000DD42E128210F1A021C311C083A5B468E
:10229000F94093400F1C1F43331C9340BB461A1C4C
:1022A000164B181A00237AE701230B4000249946A5
:1022B000A0460E4B97E70027BB46002201236EE79E
:1022C000002104248A46884601254FE70C24032573
:1022D0004CE700258024A9462403A846034B82E747
:1022E000DA46904603991D1C6FE7C046FF070000C1
:1022F00001FCFFFF58280200FFFF0F800DFCFFFFCD
:10230000029F160C381804904046070C0004000C7D
:102310001204120C031C5343041C3D1C744355430C
:1023200098463B1C73436419A44644460293230C0D
:1023300063449D4204D9029D802464022D190295B4
:102340001D0C039545462C041B04240C1C190594F4
:102350005C46230C051C58432404240C8446381C7A
:10236000604365435F438146CC44280C6044BB46D0
:10237000814502D980277F02BB442D04070C2D0C18
:10238000000440195546BC462F04E3448446280CFB
:102390003D0C2F1C5743B8462F1C77434243B94688
:1023A00047463F0C9144BA46D14446434A4502D978
:1023B00080225202B6184F463A0CB6183A044746E5
:1023C0003F043F0CB8462F1C67435D4344435843CA
:1023D00065190190380C2D184244B846AC4204D916
:1023E000019880235B02C0180190039C029F201C6F
:1023F0006044C0196045A44147466442A4462B048A
:102400003C049946240C4C44A046D8448018C2464B
:10241000E24490429241574652429146F219E245B7
:10242000BF417F424B46BC46D845BF41D4187F428E
:1024300063461F432D0C7F19B24292414C45AD417A
:1024400052426D421543019E7D19AB19E20D5B02AC
:10245000059F134342023A439A46531E9A41C30DC5
:10246000101C18436402204380465046C0010DD51D
:10247000454601225646049C6B082A401A43F3073E
:1024800001341A43760804949046B246049E634F82
:10249000F319002B61DD404640070BD00F22444664
:1024A0002240042A06D0424604324245804140423E
:1024B000824490465546ED0107D5594B5646049F38
:1024C00080201E40C000B2463B18564A934200DDB1
:1024D000EAE644465546E2086807104301226C02CA
:1024E0005B050A408046240B5B0D91467BE6DA468D
:1024F00090461D1C69E680242403574627421CD1C0
:102500003C432403240B484B6DE6031C283B311C41
:1025100099408B460022C3E6301C00F0BBFC203003
:10252000ADE6283B211C994000228A4690468EE663
:10253000201C00F0AFFC203078E65846204207D13E
:10254000044303992403240B89469046364B4AE6FC
:102550003C432403240B344B45E6344B049E9B1B25
:10256000382B06DD01230B4000249946A0460023AA
:1025700039E61F2B25DC049C2D4D4646601952463A
:1025800044468640DC4082405746301C2243DF40B0
:10259000441EA04102433B1C540709D00F201040A9
:1025A000042805D0101D9042924152429B18021CF3
:1025B0001D021AD501230B4000249946A046012391
:1025C00011E61C48049C5546001BC540281C202BC6
:1025D00016D0194E5746A21997403A1C43461A4343
:1025E000531E9A4102430023D6E758075B02D208E4
:1025F0001C0B01230B401043994680460023F2E553
:102600000022EBE7802424035046012304431940B1
:102610002403240B8946044BE5E5C046FF03000074
:10262000FFFFFFFEFE070000FF07000002FCFFFFA8
:102630001E040000E2FBFFFF3E040000F8B55F4609
:10264000564644464D46F0B40C034D00CF0F610A88
:10265000440F2143C4001803DE0F8046B4464646AB
:102660005800760A530F3343D600D14A6D0DBA464F
:10267000400DB346904200D1F5E06246012672401B
:102680009446674500D1ABE02F1A002F00DC11E122
:1026900000283ED15846184300D0F1E0600700D131
:1026A00097E00F232340042B00D122E1221DA242F8
:1026B000A4416442802309191B04012750460B40A2
:1026C0000740141C002B00D179E0B94B01359D4225
:1026D00000D10BE1B74BE408194048074902044315
:1026E0000B0B002000211B031A0B0B0D6D051B05A6
:1026F00013436A08B04DFF071D4015436D006D0878
:10270000291C3943201C3CBC90469946A246AB4646
:10271000F8BDA7488542C1D0802000040343382F6C
:1027200000DDFDE01F2F00DD31E12020C01B1A1C61
:102730005E468240FE40324394465A468240101C18
:10274000421E9041FB40624602431F1CA21A944263
:10275000A4416442C91B091B141C0A029ED54902EC
:102760004F0A002F00D1D6E0381C00F093FB021C6A
:10277000083A1F2A00DDC3E02821231C091A9740CC
:10278000CB401F439440954200DDC0E0551B691CBF
:102790001F2900DDEAE01F22551B3B1C221CAB4019
:1027A000CA40AC40651EAC411343CF401C43391CAA
:1027B000002573E780217E4D0027C90300247C4B50
:1027C0004807E4080443C9089D4250D009030B0B95
:1027D00087E780231B04012752460B40174071E70F
:1027E0002A1A9446002A00DCA1E0002854D0704840
:1027F000854200D152E78020000403436046382818
:1028000000DD0EE11F2800DD57E162462020801A1E
:102810001E1C8640B1465E46D6404A4632435E465E
:1028200086409046301C421E90414246024360461C
:10283000C3401219A242A441644259180919141C38
:10284000080200D42AE75A4B01359D4200D131E1FC
:10285000584B60081940012323401C1C0443CB073C
:102860001C4349081AE71E4300D00AE705E7231C6A
:102870000B433BD080231B030B431B031B0B30E795
:10288000013F002F6DD15E46A21B9442A4416442D9
:10289000C91A091B141C60E75846184300D1FDE60D
:1028A00001267642B4446046002800D0D0E05E465F
:1028B0003219BFE7002F00D080E0681C4005400DB2
:1028C000012800DCE8E05A46A21A9442BF41C81A27
:1028D0007F42C71B3E0200D498E05846041BA34524
:1028E0009241591A52428F1AE2463AE700230024D5
:1028F000F7E680231B04012756460B403740E1E6EC
:10290000271C283887400024954200DC3EE72949EF
:10291000AD1A3940C2E6201C00F0BCFA203026E790
:102920005A461A43531E9A41D2B200270EE7002A94
:1029300000D0DEE0681C4605760D012E00DC90E03C
:102940001B4DA84200D1F5E05E463219A242A441D7
:10295000644259180919CC07520814434908051C48
:102960009CE61348854200D0D9E697E62B1C1F3B16
:102970003E1CDE40331C20296FD03F22551BAF4048
:102980003C43601E84411C430021002586E6381C20
:1029900020381E1CC640301C202F60D04022D71B80
:1029A000BB405A461A43531E9A4102430027CDE6C4
:1029B000FF070000FFFF7FFFFFFF0F80002D37D0D4
:1029C000B64DA84200D18FE080252D047F422943D7
:1029D000382F00DDA8E01F2F00DD24E12025ED1BAE
:1029E0000E1CAE40B046261CFE404246AC4016438C
:1029F000651EAC413443F9405A46141BA34592412D
:102A00005B1A5242991A051CE246A6E6131C3B4388
:102A1000141C002B00D0A4E6002700210025002470
:102A2000CDE65A461A43531E9A41D2B2002300E71C
:102A30000D1C254358D0FF43002F51D15A46141B7B
:102A4000A3459241591A5242891A051CE24684E66E
:102A50009248854200D0D1E620E6002790E7002387
:102A60009FE7081C2043002D00D0C2E0002800D1C1
:102A7000EFE05846184300D110E658460219A2422A
:102A8000A441644259180919141C0A0200D405E62D
:102A9000834B0125194001E6081C2043002D38D145
:102AA00000286FD15946194303D0191C5C46E246F1
:102AB000F4E500270021002481E6604620381A1C36
:102AC000C2406646101C202E00D1AAE04022921B74
:102AD00093405A461A43531E9A4102430023A8E6E4
:102AE0006E4DA84200D073E7191C5C46051CE246F7
:102AF000D4E5002D22D10D1C254376D0D543002DE1
:102B000070D15C445C459241591852428918051CA9
:102B100096E600284CD15946194300D14AE6191CC3
:102B20005C46E2465D4DB9E50C43611E8C41E4B262
:102B3000002161E7051C0021002440E6574DA84212
:102B400053D05542802216043143382D7BDC1F2D93
:102B500000DD8CE02022561B0A1CB446B240261C25
:102B6000EE403243904662469440661EB44142466F
:102B70001443E9405C445C459241CB185242991899
:102B8000051C5DE65846184300D187E55E46A71B45
:102B9000BC429241C81A5242801A060260D5584679
:102BA000041BA3459241591A5242891AE24675E51F
:102BB0005846184333D04807E40804438020C90826
:102BC0000003014208D0DD08054205D15946CA0874
:102BD0005C071443291CE246630FC9001943E40053
:102BE0002E4D5BE52D4A9042AFD1191C5C46051C69
:102BF00054E5002830D05846184310D080254807A7
:102C0000E408C9082D0304432942E5D0D808284226
:102C1000E2D15D46EA085C071443011CDCE71F4D66
:102C20003CE5002355E73D1C203D0E1CEE40351CC5
:102C3000202F2ED04026F71BB9400C43611E8C413B
:102C40002C430021D8E60C43611E8C41E4B20021E4
:102C500090E7191C5C4621E5191C5C460F4D1DE5EB
:102C6000031C3B4300D124E7011C3C1C16E5202635
:102C7000764276190A1CF2409046202D0BD0402651
:102C8000751BA9400C43611E8C4145462C43002115
:102C900070E70021D1E70021F4E7C046FF070000FC
:102CA000FFFF7FFF70B50B1C124C09030E0B590080
:102CB000021C490DDD0F0020A14211DD0E488142AA
:102CC0000FDC8020400306430C48401A1F280BDD10
:102CD0000B4A521AD640321C5042002D00D1101C13
:102CE00070BD084BE818FBE7074BC240C9188E407F
:102CF0003243F1E7FE0300001D040000330400002E
:102D000013040000FFFFFF7FEDFBFFFFF8B5041E7B
:102D100031D0C70F00D04442201C00F0BBF8184D42
:102D20002D1A0A2819DD0B38844024036D05240B65
:102D30006D0D3A1C0026002000210B0D2403240BEE
:102D40001B0523430F4C2D051C402C4364006408D5
:102D5000D307211C301C1943F8BD061C1536231C53
:102D6000B3401E1C0B23181AC44024036D05240B0A
:102D70006D0D3A1CDFE70022002500240026DAE76B
:102D80001E040000FFFF0F8010B5041E28D000F0C5
:102D900081F8154A121A0A2815DD0B3884402403DD
:102DA0005205240B520D0023002000212403181C7F
:102DB0000B0D240B1B0523430C4C12051C40144324
:102DC0006400610810BD031C1533211C99400B1CC5
:102DD0000B21081AC44024035205240B520DE3E7CB
:102DE000002200240023DFE71E040000FFFF0F8005
:102DF00043001B0E5A1C4102D2B270B54C0AC50FDB
:102E0000012A17DDE02292006407090B98180022BE
:102E100000231E0D221C34050C431B4940054008AD
:102E20002140014349004908ED070B1C2B43101CAE
:102E3000191C70BD002B15D1002C1CD0201C00F0DB
:102E400029F80A281ADC0B21091A231CCB40191C6B
:102E5000031C15339C400D4B0903181A4005090B40
:102E6000400DD4E7002C03D06407090B0848CEE7D7
:102E700007480021CBE700200021C8E7011C0B39DF
:102E80008C40211C0024E6E7FFFF0F80890300002F
:102E9000FF0700001C2101231B04984201D3000CF2
:102EA00010391B0A984201D3000A08391B099842BD
:102EB00001D30009043902A2105C40187047C046D3
:102EC00004030202010101010000000000000000F3
:102ED000F0B544465F4656464D46F0B41C1C85B0DE
:102EE000002900DADBE00F1C0021061C8A46101CBA
:102EF000191C002C00DAC9E0019600908946804632
:102F0000002951D1B84200D871E0FFF7C3FF002873
:102F100009D020234546311C1B1A85408740D940E3
:102F2000A8460F4386404246150C13041B0C291C6F
:102F3000381C9B46FDF7D0F85B464343041C291C14
:102F4000381C9946FDF70CF9330C080418438145E9
:102F500009D94044631E804500D978E1814500D8F5
:102F600075E1023C40444946411A8946081C291C27
:102F7000FDF7B2F85A464243071C291C48469346BF
:102F8000FDF7EEF836040904360C0E43B34507D9B5
:102F900046447B1EB04502D8023FB34500D81F1CF3
:102FA00024042743002403E0B94211D90024002758
:102FB0005246381C211C002A03D03B1C00215842D9
:102FC000A14105B03CBC90469946A246AB46F0BD37
:102FD000081CFFF75FFF041E00D0BFE0B94500D218
:102FE00042E1019D0099071C8D424741E0E700281E
:102FF00004D101200021FDF76FF880464046FFF71D
:1030000049FF002852D1414644460B043C1B1B0C8F
:10301000A3460D0C00930124291C5846FDF75CF8CB
:10302000009F81464743291C5846FDF799F8330C09
:10303000090419438F4208D94B464144013B884556
:1030400002D88F4200D91AE19946C91B8B46081C49
:10305000291CFDF741F8009B291C4343071C5846D7
:103060000093FDF77DF83604009D0904360C0E43ED
:10307000B54207D946447B1EB04502D8023FB5424F
:1030800000D81F1C49460E04374391E75246D243ED
:10309000031C0C1C924600215842A1412CE700273A
:1030A00046428F41012149428A4620E720231B1ACC
:1030B0004246351C82403C1CDD40DC4087402B1CD6
:1030C000150C3B43291C8640201C00931704904696
:1030D000FDF702F83F0C011C794381468B46201C0A
:1030E000291CFDF73DF8009C0904230C19438B456E
:1030F0000CD94B464144013B884500D9BDE08B4586
:1031000000D8BAE002225242914441445C460C1B72
:10311000201C291C0194FCF7DFFF391C4143041CCF
:103120008B460198291CFDF71BF8009A090413042B
:103130001B0C19438B4509D94144631E884500D9AE
:1031400097E08B4500D894E0023C41445B46CB1AA3
:1031500049469B460B041C4300975DE7009D2023D6
:103160001B1A4A468240DD401543391C009AD9405B
:1031700082408846311C0092D9403A1C82400B1C88
:10318000134301932F0C2B041B0C391C4046029354
:10319000FCF7A2FF029A81464243391C40469346FF
:1031A000FCF7DEFF019A0904130C19438B450AD979
:1031B0004B464919013B8D425DD88B455BD90223B3
:1031C0005B42994449195A468A1A101C391C0392C9
:1031D000FCF782FF029B80464343391C03989B46C1
:1031E000FCF7BEFF019A090413041B0C19438B451D
:1031F0000AD943464919013B8D4238D88B4536D907
:1032000002235B42984449195D464D1BAB46494633
:10321000009D0F04424617432A04120C3B042D0C58
:103220001B0C380C111C594342436B436843D318A1
:103230000D0C5B198C469A4202D9802252028018EA
:103240001D0C401983450CD303D00024B0E61C1C90
:1032500089E665462A041B04120C9B18A6409E4270
:10326000F3D2013F0024A3E600240127A0E69846FC
:10327000CAE71C1C6AE79946A5E7994646E7022279
:10328000524291444144E0E6F0B55F4656464D4611
:103290004446F0B40D1C85B0061C92469846029038
:1032A000019103921F1C141C8346A946002B59D17F
:1032B000AA4269D9101CFFF7EDFD00280AD020238F
:1032C0001B1A311CD94085400B1C2B43864084407F
:1032D0009946B346250C23041B0C291C48469846E6
:1032E000FCF7FAFE4646071C4643291C4846FCF7F5
:1032F00037FF5A460904130C19438E4209D909199C
:103300007B1E8C4200D957E18E4200D854E1023F27
:103310000919891B8946081C291CFCF7DDFE434658
:103320004343061C291C48469846FCF719FF5A4699
:10333000130409041B0C1943884508D90919731E85
:103340008C4200D936E1023E884500D832E138048B
:1033500030430027391C05B03CBC90469946A24634
:10336000AB46F0BD019A934262D8181CFFF792FD5C
:10337000041E60D1019B9F4200D22CE1029F039961
:103380008F4260410027E5E7002A04D10120002197
:10339000FCF7A2FE041C201CFFF77CFD002800D0D7
:1033A000B9E023042D1B1B0CA946260C98460127C7
:1033B000311C4846FCF790FE41464143051C8A46B5
:1033C0004846311CFCF7CCFE5A460804130C18433F
:1033D000824507D900196B1E844202D8824500D964
:1033E00010E11D1C5346C31A181C311C9A46FCF7E9
:1033F00073FE41464143814688465046311CFCF7E6
:10340000AFFE5A46130409041B0C194388450BD917
:103410004B460919013B8C4200D9CFE0884500D8C2
:10342000CCE002235B42994428044946084391E7D3
:10343000002700208EE720231B1A42465746824071
:10344000DF401743524682400192321CDA40291C69
:10345000D9408540131C2B4302933D0C3B041B0CAD
:103460008846081C291C9A46FCF736FE53464343FF
:103470008146291C40469B46FCF772FE029A0904CD
:10348000130C19438B4506D94B46C919013B8F4292
:1034900000D8ABE099465A468A1A101C291C93465C
:1034A000FCF71AFE53464343291C804658469A4669
:1034B000FCF756FE029A090415042D0C29438A458F
:1034C00006D94346C919013B8F4200D886E0984689
:1034D0005746CF1BBA464946019F0804424610434F
:1034E0003D042D0C03043F0C1B0C020C291C5943FA
:1034F00055437B437A43EB180F0CDB198C469D42F6
:1035000002D980277F02D2191D0C521992455FD330
:1035100056D000271EE720231B1A311C2F1CD94030
:10352000DF4085400B1C84402B4386400193B3460B
:103530002304260C1B0C381C311C9846FCF7CCFDD0
:1035400042464243051C311C381C9146FCF708FEDC
:10355000019F09043B0C1943894507D909196B1EC2
:103560008C424DD889454BD9023D09194A468A1AE1
:10357000101C311C9246FCF7AFFD43464343071C29
:10358000311C50469946FCF7EBFD019A09041304DF
:103590001B0C1943894507D909197B1E8C422DD86C
:1035A00089452BD9023F09194B46CB1A2D04994660
:1035B0002F43FDE61E1CCAE61F1CAAE6994633E708
:1035C00061460A041B04120C9B18A6409E42A0D21E
:1035D00001380027BEE600270120BBE68A4500D857
:1035E00075E702235B429844C91971E78B4500D8FF
:1035F00050E702235B429944C9194CE71F1CD3E7EB
:103600001D1CB3E7023D0019ECE6C04602780B78BA
:1036100001300131002A01D09A42F7D0D01A704708
:1036200030B5033985B0041C4E2900D99FE06C4B9E
:1036300089005B589F460C2000F048FE201C06F0D5
:1036400079FE002005B030BD8020000206F094F91C
:103650000223011C80201943000206F0ADFB162056
:10366000F0E700F0B1FD011C201C06F019FE5D48DA
:103670000AF038F881B2201C06F012FE5A480AF00F
:1036800031F881B2201C06F00BFE201C06F052FE21
:103690000020D7E706F0AEFD03286AD80021534882
:1036A00006F08AFB52480521524A05F0CBFA201C4D
:1036B00006F040FE032000F009FE0020C2E70420CF
:1036C00000F004FE201C06F035FE0020BAE70020C2
:1036D00000F0FCFD201C06F02DFE0020B2E70120CA
:1036E00000F0F4FD201C06F025FE0020AAE70220D1
:1036F00000F0ECFD201C06F01DFE0020A2E70520D6
:1037000000F0E4FD201C06F015FE00209AE73A4D7B
:103710004C23E95C06F0B6FD4D23E95C201C06F065
:10372000B1FD201C06F006FE00208BE7684602A9CA
:1037300000F090FD002815D06B461978201C06F08B
:10374000A1FD201C029906F0C3FD0BE006F0F2FD7E
:103750000A2000F0BBFD002074E706F053FD051EB3
:10376000012D18D9201C06F0E5FD00206AE716207F
:1037700068E7201C06F056FD011C1C4806F01CFBE7
:1037800000211A4806F0C6F80521031C1B4A1848F8
:1037900005F058FA8BE7002816D1174A7023D15C40
:1037A000201C06F06FFD201C06F024FD0028D9D057
:1037B000201C06F027FD00280AD1281C451EA84120
:1037C000083000F083FDCDE70B4A7123D15CE7E7B9
:1037D000281C451EA841063000F078FDC2E7C0460F
:1037E00098280200245E02002C5E020083B00000D4
:1037F00050580200F029020014F4FF1FD4290200DF
:10380000F8B5144D00262B6800240127002B16D094
:103810002B1D00220433191F096801320029F9D138
:1038200094420CD2A300E8580AF008FD002802D008
:103830003B1CA3401E432B680134002BE8D1064AF1
:10384000AC23D35C0020002B01D00120A0403043EA
:10385000F8BDC04610E0FF1F14F4FF1FF8B5104D6F
:1038600000262B6800240127002B16D02B1D0022D8
:103870000433191F096801320029F9D194420CD28E
:10388000A300E8580AF0CEFC002802D03B1CA3405D
:103890001E432B680134002BE8D1301CF8BDC04614
:1038A00048E0FF1F38B5144D2B68002B1AD02B1D94
:1038B000002204331C1F24680132002CF9D19042ED
:1038C00010D280002C5801290DD000290FD00229D8
:1038D00008D1201C0AF0A6FC01235840C1B2201CCC
:1038E0000AF090FC38BD201C0AF074FCFAE7201C9A
:1038F0000AF07CFCF6E7C04648E0FF1F08B5044B21
:103900001868002802D006F011FD08BD0020FCE771
:1039100010E1FF1F10B50549041C07F011F9201C28
:1039200007F020F9024B1C6010BDC0462136010093
:1039300010E1FF1F08B50E480AF080FC0D4B1A7A03
:1039400082420ED0DA68022A07D95A7A002A0CD0AD
:103950005A6801325A6000225A720122DA601872E3
:1039600008BDDA680132DA60F9E701225A72F4E739
:10397000805F020014F4FF1FF0B5474680B4524C3C
:103980000C22236882B01A421DD0504AA25C002A41
:103990004ED15A0760D54E4B0521181C4D4A98460A
:1039A00005F050F90EF01AFD23681A0706D54046B7
:1039B0000521494A05F046F90EF040FD47484849BF
:1039C00009F0FAFB30E0414BE35C002B30D1404A78
:1039D00005219046101C434A05F034F90EF042FDD3
:1039E0000EF076FD404D3E49281C09F0E5FB4046AF
:1039F00005213E4A05F026F97026712702E0642071
:103A00000BF0E2F8A35D002B02D1E35D002B04D0A4
:103A1000281C09F0E7FB0028F1D0281C09F0E2FB84
:103A200000280DD10023E36602B004BC9046F0BD2F
:103A3000274B0521181C2E4A984605F003F9CDE7BF
:103A4000743D7122AA5C7023EB5C40460092042115
:103A5000284A05F0F7F8E5E71D4A251C101C05214A
:103A600090467435244A05F0EDF80EF0FBFC281C56
:103A70001B4909F0A1FB404605211C4A05F0E2F86C
:103A80007023E35C271C7026002B06D10AE064201B
:103A90000BF09AF8BB5D002B04D0281C09F0A2FBA8
:103AA0000028F4D0281C09F09DFB002800D17BE7FA
:103AB000743D7122AA5C7023EB5C404600920421A5
:103AC0000C4A05F0BFF86FE714F4FF1FDB0200009B
:103AD00050580200402A0200CC2A02007CF4FF1F4A
:103AE000307500000C2B020088F4FF1F782A0200BA
:103AF000E82A0200902A02005C2A020030B583B056
:103B000009F086FF1C4805F023FF04281FD9002177
:103B1000194805F0FFFE8023184CDB00184D1843B0
:103B200020600521281C174A05F08CF820688206C1
:103B300018D41548002109F03FFB2368A46B281C0A
:103B400000940521114A05F07DF803B030BD0A4804
:103B500005F012FF8023DB00084C18432060084D5D
:103B60008206E6D50A4805F007FF0A4941430648A0
:103B700009F022FBE1E7C04666B0000014F4FF1F25
:103B8000505802002C2B020048F4FF1F542B020057
:103B900080B0000060EA0000F0B54F464646C0B471
:103BA0006F4D83B0281C09F00FFB6E4C6E482168E6
:103BB000CE0809F097FDC300181AC3175B0F181839
:103BC000C01086192660694E69483268D70809F026
:103BD00089FDC3001B1AD817400FC018C010C019A8
:103BE00030602A7A23686A7298423CD2614D2A7802
:103BF000002A00D172E0604F0123381C2B7009F0BD
:103C0000F1FA00284BD03B7C002B00D19EE05B4DAD
:103C1000AC220123AB545A4A90461278002A00D1B4
:103C20008DE02368574A934247D857490A78894616
:103C3000002A00D17BE001234946381C0B7009F0B3
:103C4000D1FA031C0020002B67D1AC23EB5C002BC6
:103C50001CD00021AE22A95441460B7003B00CBC0D
:103C600090469946F0BD002A48D1444D414A002370
:103C7000281C13709C30AC22AB5409F0A5FA404AC2
:103C80009046AC23EB5C0020002B11D122683D4B09
:103C90009A4202D800230121DCE70023D9E7384B00
:103CA0003D1C9C3D9846AC23EB5C0020002BEDD0E6
:103CB0002368344A304F9342B7D9334A9146127839
:103CC000002A22D100234A46381C137009F07CFADE
:103CD000AC23EB5C0020002BBBD1D7E70090052183
:103CE0002A482B4A04F0AEFF234F0123381C2B70C7
:103CF00009F078FA002800D085E7D0E70090052188
:103D00002248244A04F09EFFAFE736681F48009619
:103D10000521214A04F096FFD4E736681B48009637
:103D200005211E4A236804F08DFF01208DE73268CB
:103D30001648009205211A4A04F084FF7BE7124AD4
:103D4000281C9C30137009F03FFA9AE731680F483D
:103D50000091144A0521236804F074FF57E7C04618
:103D6000B8F4FF1F20E1FF1F2C5E02001CE1FF1FC3
:103D7000245E020001E0FF1FB0F4FF1F14F4FF1FD8
:103D800014E1FF1F410E000000E0FF1F5058020029
:103D9000882B0200E42B02007C2C0200482C02003D
:103DA0000C2C0200BC2B020038B5254CE06F0AF049
:103DB00045FA8423E35C85224340DBB2051CA3540F
:103DC000002B07D0002837D18723E0540AF000FFEA
:103DD0008023E0508423E5548823E0580AF02EFA2B
:103DE0009023E35C91224340DBB2051CA354002BDB
:103DF00007D000281CD19323E0540AF0E9FE8C235D
:103E0000E0509023E5540F480AF018FA9423E05448
:103E10000D480AF013FA9623E0540C480AF00EFA03
:103E20009923E0540A480AF009FA9B23E05438BD6C
:103E300000229223E254E0E700228623E254C5E701
:103E400014F4FF1F7C5E020024610200386102004E
:103E5000585F0200F0B54E4657464546E0B482B082
:103E6000041C0EF0EFF9BA4E01238622B3549222BD
:103E7000B354B8480AF0E2F9B74BF054002800D028
:103E800042E1B64A92464C23B54AF4545046231CAC
:103E9000052104F0D7FE0BF007F84B23F25C3F2A14
:103EA00009D9013AF2544A23F25C0132D2B23F2AD4
:103EB00000D927E1F2544925735D1733DB00F71869
:103EC0003C720BF06FFB7860735D0133DBB23F2B0C
:103ED00000D9002373554B23F25C00240132F254C5
:103EE0000AF0E6FF504605219E4A04F0ABFE30235F
:103EF000FA21F454490001233122301CB35410300C
:103F00000A1C01930094002306F0ACFE5C23964843
:103F1000F45474660AF05EF9944A5046052104F0A0
:103F200091FEFA2040000AF04FFE914A1068904638
:103F3000002816D0042400258E4F06E04246105972
:103F4000231D00280DD0251C1C1C0AF043F97859AC
:103F50000028F3D00AF038FE42461059231D0028ED
:103F6000F1D1854900240B1C04CB002A1ED0043358
:103F70001A1F12680134002AF9D1804AA300D2180E
:103F80009146CF18002508E07B19043B1868013CD6
:103F90000AF02CF9043D002C08D04A465319043B82
:103FA00018680028F0D00AF00FFEEDE7744C201CD2
:103FB0000AF010F964200AF007FE201C0AF016F936
:103FC000704C02E000200AF0FFFD201C0AF036F9D8
:103FD0000028F7D06C4D2868002816D06B4B0424BD
:103FE0000027994605E02859231D00280DD0271CDD
:103FF0001C1C0AF0EFF84A46D0590028F3D00AF00A
:10400000E3FD2859231D0028F1D10A200AF0DCFD28
:104010002B1C04CB0024002A20D004331A1F126862
:104020000134002AF9D1594AA300ED18D218A94643
:104030009046002509E04A465319043B1868013CA4
:104040000AF0D4F8043D002C08D042465319043B32
:1040500018680028EFD00AF0B7FDECE705214C4ABC
:10406000F36A504604F0EEFDB42189007258531CE7
:104070007350002A50D1474B1B789A073CD4022238
:104080003123F254B2239B00F018434909F094F80D
:10409000301C3C30414909F08FF8301CFA219C302B
:1040A000C90009F089F8301CA430642109F084F8B3
:1040B000301C6421B03009F07FF80EF08FF9FFF763
:1040C00073FE9423F25C9523F2549623F25C9723BB
:1040D000F2549923F25C9823F2549B23F25C9A23C6
:1040E000F25409F095FCFFF709FCF06202B01CBC29
:1040F00090469946A246F0BD50460521284A04F054
:10410000A1FDBCE70022D5E6144B0521181C254A69
:104110009A4604F097FDB6E6B124A4003259052171
:1041200050460092204A04F08DFD0AF0BDFE0023A7
:104130001E4833510AF082F8AF239B00F0540AF076
:1041400047FDB0239B00F0500AF0B2FE97E7C0464F
:1041500014F4FF1F685E0200DA02000050580200EB
:10416000C42C0200D82C02006C5F0200E42C020078
:10417000ACF0FF1FCC6702007CE0FF1F006702006D
:10418000706002005C60020010F4FF1FD467020040
:10419000F02C020000F00740DC050000A0BB0D0081
:1041A000242D0200B02C0200002D0200BC5F020092
:1041B000014B58687047C04614F4FF1F014B59600B
:1041C0007047C04614F4FF1F38B50C4D0C4AAC23A1
:1041D000281CD45C09F086FA0A4B984202DC802342
:1041E0001B021C43281C09F07DFAF423FF3398427C
:1041F00002DC80235B011C43201C38BD2C5E0200C6
:1042000014F4FF1F410E000070B5041C21600E1C49
:104210000AF0DEFC002560606572301C0AF00EF8C2
:10422000A572E572207270BD08B5024808F0CCFF97
:1042300008BDC04650F4FF1F024B012148225864BC
:104240009954704714F4FF1F014B186C7047C04617
:1042500014F4FF1F70B5061C0D1C0AF025FE124B4E
:104260004B229A5C0024002A17D04A22995C17310D
:10427000C9005918097A3170995C1731C900591869
:1042800049682960995C0131C9B23F2909D899541C
:104290004B22995C0124013999540AF009FE201C33
:1042A00070BD9C54F4E7C04614F4FF1F08B50AF033
:1042B000FBFD054B002249215A544A215A544B21F7
:1042C0005A540AF0F5FD08BD14F4FF1F00B583B081
:1042D0006A4600235370044B10706946186D002223
:1042E0000AF088FC03B000BD14F4FF1FF8B54F4678
:1042F0004646C0B4304809F0A1FF041E37D02F4C09
:104300002368002B3CD0042B41DC013323602C4C70
:10431000B625AD00635B002B08D0013B9BB2635315
:10432000052B38D00CBC90469946F8BD254AAF27DE
:10433000101C904609F082FFBF00E35D061C83421B
:10434000F0D00AF045FCE6558146002E0AD1B02394
:104350009B00E258B1239B00821AE2501A4BE35CA7
:10436000002B20D1B0239B004A46E250DAE71748E1
:1043700009F030FF164809F039FF104B1C60C6E702
:10438000134809F027FF236801332360BFE70F4874
:1043900009F02CFFBBE70B4C201C09F027FF201C69
:1043A00009F0E6FEBEE7404609F014FF404609F07A
:1043B000E5FE32236353D5E74C61020024E1FF1F81
:1043C00014F4FF1FBC5F0200DA02000084600200E8
:1043D000E8600200F0B54F464646C0B4A54C83B035
:1043E0002368D80704D59622A25C002A00D035E1C4
:1043F000A14F0521381CA14A04F024FC21680920A2
:10440000490500D5E3E000210AF0C0FF226805203D
:10441000D20700D4E3E002210AF0B8FF23680620A7
:104420009B0700D4E3E003210AF0B0FF20680006F8
:1044300000D4E3E0072003210AF0A8FF21680A2046
:10444000490700D4E3E002210AF0A0FF2268082017
:10445000D20600D4E3E001210AF098FF23680E2081
:10446000DB0500D4E3E002210AF090FF206880051C
:1044700000D4E3E002210F200AF088FF21688906BA
:1044800000D4E3E07E4805F077FA7E4D7E4A2B1C8F
:1044900043430521381C04F0D5FB002001210AF01C
:1044A0008BFF774805F068FA684309F0E5FF0BF0E9
:1044B00079F8051C64200AF087FB0AF095FF962026
:1044C00040000AF081FB0BF06DF880460AF088FF8F
:1044D0002268061C920600D5BDE032794046451B95
:1044E0003368052100920195684A381C04F0AAFB44
:1044F0003268111C930500D4CEE0930600D428E264
:10450000634A0223381C052104F09CFB0AF0CCFC12
:104510004B23E25C3F2A09D9013AE2544A23E25C88
:104520000132D2B23F2A00D9A2E0E2544925635DAC
:104530001733DB001B1998464046022303720BF029
:1045400031F841464860635D0133DBB23F2B00D94F
:10455000002363554B23E25C0132E2540AF0A8FCCD
:104560003268111C530600D42CE212239946484AA3
:10457000381C052104F066FB0AF096FC4B23E25C34
:104580003F2A09D9013AE2544A23E25C0132D2B20D
:104590003F2A00D90022E2544925635D4A46173379
:1045A000DB001B191A7298460AF0FCFF434658605C
:1045B000635D0133DBB23F2B00D9002363554B23EE
:1045C000E25C0132E2540AF073FC31686BE00221D4
:1045D0000AF0DCFE22680520D20700D51BE7002187
:1045E0000AF0D4FE236806209B0700D51BE70021B4
:1045F0000AF0CCFE2068000600D51BE7072000214A
:104600000AF0C4FE21680A20490700D51BE70021F3
:104610000AF0BCFE22680820D20600D51BE7002164
:104620000AF0B4FE23680E20DB0500D51BE700214D
:104630000AF0ACFE2068800500D51BE700210F20A2
:104640000AF0A4FE2168890600D51BE7002000219E
:104650000AF0B2FE2BE709F04FFF3EE706480521BE
:104660000C4A04F0EFFA03B00CBC90469946F0BD3A
:1046700000225AE714F4FF1F50580200642D020074
:1046800080B0000060EA0000982D0200B82D020002
:10469000C42C0200302D0200900600D561E74023B3
:1046A000134000D158E1080600D446E111231D1C37
:1046B000CB4A381C052104F0C5FA0AF0F5FB4B2360
:1046C000E25C3F2A09D9013AE2544A23E25C013212
:1046D000D2B23F2A00D90022E2544921635C8846C5
:1046E0001733DB001B191D7299460AF05BFF4B461E
:1046F00058604046235C0133DBB23F2B00D81AE1FF
:10470000002323544B23E25C0132E2540AF0D0FB35
:1047100031684A0500D465E11F231D1CB04A381CCE
:10472000052104F08FFA0AF0BFFB4B23E25C3F2A1D
:1047300009D9013AE2544A23E25C0132D2B23F2A5B
:1047400000D90022E2544921635C88461733DB001C
:104750001B191D7299460AF025FF4B4658604046CA
:10476000235C0133DBB23F2B00D8E2E0002323546B
:104770004B23E25C0132E2540AF09AFB3168CB052C
:1047800000D427E110231D1C954A381C052104F094
:1047900059FA0AF089FB4B23E25C3F2A09D9013A16
:1047A000E2544A23E25C0132D2B23F2A00D900220D
:1047B000E2544921635C88461733DB001B191D72E4
:1047C00099460AF0EFFE4B4658604046235C0133A1
:1047D000DBB23F2B00D8AAE0002323544B23E25C3A
:1047E0000132E2540AF064FB3168480400D40DE160
:1047F00013231D1C7A4A381C052104F023FA0AF001
:1048000053FB4B23E25C3F2A09D9013AE2544A2385
:10481000E25C0132D2B23F2A00D90022E25449239D
:104820009846E35C1733DB001B191D7299460AF0AA
:10483000B9FE494648604246A35C0133DBB23F2BD8
:1048400073D90023A3544B23E25C0132E2540AF0F3
:104850002FFB31680A0475D51D231D1C604A381CC6
:10486000052104F0EFF90AF01FFB4B23E25C3F2A1D
:1048700009D9013AE2544A23E25C0132D2B23F2A1A
:1048800000D90022E25449239846E35C1733DB0049
:104890001B191D7299460AF085FE4946486042463A
:1048A000A35C0133DBB23F2B3DD90023A3544B2340
:1048B000E25C0132E2540AF0FBFA33791E25D80794
:1048C0002DD51E231D1C464A381C052104F0BAF9BB
:1048D0000AF0EAFA4B23E25C3F2A09D9013AE25492
:1048E0004A23E25C0132D2B23F2A00D90022E254CC
:1048F0004926A75D1737FF00E7193D720AF052FEFF
:104900007860A35D0133DBB23F2B00D90023A355B0
:104910004B23E25C0132E2540AF0CAFA1425281C47
:10492000FFF798FA9FE6A354C1E7A3548BE72354FB
:1049300054E723541CE72354E4E6480524D5112307
:104940001D1CEBE633791D25D907E8D51D231D1C59
:10495000B9E753063BD402231D1C100603D5002DD6
:1049600000D1D6E6A4E6500508D5002D00D106E713
:10497000D4E612231D1C500500D5CFE6D00508D57E
:10498000002D00D131E7FFE611231D1CCA0500D51B
:10499000FAE64A0407D5002D00D15BE72AE74B046D
:1049A00031D41F231D1C0A0402D5002D85D055E7E4
:1049B0003279D10702D5002DB0D084E7002DAED1D9
:1049C0000425ACE71306D4D512231D1C70E6022380
:1049D0009946CCE54B040AD510231D1C0AE7C046B6
:1049E000C42C0200CA05DAD51F231D1CCCE60A041C
:1049F00002D510231D1C31E733791025D8078ED539
:104A000010231D1C5FE71F231D1CF3E6080402D5BD
:104A100013231D1C22E733791325D80700D47EE722
:104A200013231D1C4FE7C046F0B5444656464D467D
:104A30005F46F0B4BA4C01238622A3549222A354B9
:104A400083B0C8228046201C10300092019332228D
:104A500000238A46322106F005F9B248002104F00D
:104A600059FFBA2582B26253002A00D136E1AE4A1C
:104A70000004030C9146AD4A4846052104F0E2F8D3
:104A80005C235246E25430230122E2545346002B69
:104A900000D09BE0201C5430002108F08DFBFFF774
:104AA0002DF84246882A00D127E18B2A00D027E141
:104AB0009F4BA048009301230193642164220023AB
:104AC00006F0D0F88020000204F056FF071E00D147
:104AD000BAE05346009348460521974A434604F0FE
:104AE000B1F84D234246E2544846944A43460521D4
:104AF00004F0A8F80AF0D8F94B23E25C3F2A09D960
:104B0000013AE2544A23E25C0132D2B23F2A00D990
:104B1000E2E0E2544925665D43461736F600A619E1
:104B200033720AF03FFD7060635D0133DBB23F2BEF
:104B300000D9002363554B23E25C0132E2540AF0B2
:104B4000B7F964200AF040F842468B2A0DD07C4821
:104B500009F04CFB484605217A4A04F073F84346B5
:104B6000882B02D18023DB002360FA2040000AF06A
:104B70002BF801223023E254B3239B000025E5509B
:104B8000FFF712F99423E25C9523E2549623E25C4A
:104B90009723E2549923E25C9823E2549B23E25C3E
:104BA0009A23E254684BE25C002A00D0A1E023681B
:104BB000002B04D042468B2A01D0FFF70BFC03B038
:104BC0003CBC90469946A246AB46F0BD251C7435C8
:104BD0000DF048FC0DF07CFC281C5C4908F0ECFA58
:104BE000484605215A4A04F02DF87026712702E044
:104BF000642009F0E9FFA35D002B02D1E35D002BE7
:104C000004D0281C08F0EEFA0028F1D0281C08F087
:104C1000E9FA002877D14F4D4F49281C08F0CCFA0B
:104C20000026281C012344380193C821C8220023F0
:104C3000009606F017F88020543D00022E6004F024
:104C40009BFE071E00D044E7524600920521434ACE
:104C50004346484603F0F6FF414900250A1C08CAAE
:104C6000002B20D00432131F1B680135002BF9D113
:104C70003C4AAB00D218C91893468A46002609E080
:104C800052469319043B1868013D09F0AFFA043EFF
:104C9000002D08D05A469319043B18680028EFD01D
:104CA00009F092FFECE7304E3068002800D118E799
:104CB0002E4B04259A4606E070592B1D002800D182
:104CC0000FE72F1C1D1C09F085FA5246D059002809
:104CD000F2D009F079FFEFE700221AE7124B052125
:104CE000181C234A994603F0ADFFFA235B01635376
:104CF000C1E6E5540DF0B8FA59E78023DB002360E4
:104D0000FEF73AFED4E6743D7122AA5C7023EB5C98
:104D1000484600920421174A03F094FF7BE7C046FF
:104D200014F4FF1FD3F3000050580200102E0200AD
:104D30001027000024F4FF1F642E0200C42C020080
:104D40006C5F0200A82E0200DB020000307500003C
:104D5000782A020068F4FF1F88130000302E02003A
:104D6000ACF0FF1FCC6702007CE0FF1F0067020071
:104D7000E82D0200902A0200F0B544464D465F46F9
:104D80005646F0B4914C01238622A3549222A35498
:104D900083B0C8228046201C10300092019332223A
:104DA0003221002305F05EFF8948002104F0B2FDA6
:104DB000BA2582B26253002A00D1FBE0854A000482
:104DC000030C914648460521834A03F03BFF00222D
:104DD0005C23201CE2545430012230230021E25491
:104DE00008F0EAF9FEF78AFE4246882A40D08B2A6C
:104DF00041D17A4B7A4800930123019364216422C4
:104E0000002305F02FFF8020000204F0B5FD071EEF
:104E100000D0C0E000900521724A4346484603F0A6
:104E200011FF714900250A1C08CA002B26D0043244
:104E3000131F1B680135002BF9D16C4AAB00D21847
:104E4000C91893468A46002609E052469319043B46
:104E50001868013D09F0CAF9043E002D0ED05A46EB
:104E60009319043B18680028EFD009F0ADFEECE779
:104E70008023DB002360FEF77FFDBAE75C4E3068DD
:104E8000002815D05B4B04259A4605E070592B1D70
:104E900000280DD02F1C1D1C09F09CF95246D0593A
:104EA0000028F3D009F090FE70592B1D0028F1D195
:104EB0004D234246E25448464F4A4346052103F0FB
:104EC000C1FE09F0F1FF4B23E25C3F2A08D9013A09
:104ED000E2544A23E25C0132D2B23F2A64D8E2545F
:104EE0004925665D43461736F600A61933720AF067
:104EF00059FB7060635D0133DBB23F2B00D90023A7
:104F000063554B23E25C0132E25409F0D1FF642087
:104F100009F05AFE42468B2A0DD0384809F066F94E
:104F200048460521364A03F08DFE4346882B02D1C0
:104F30008023DB002360FA20400009F045FE0122B7
:104F40003023E254B3239B000025E550FEF72CFFED
:104F50009423E25C9523E2549623E25C9723E25487
:104F60009923E25C9823E2549B23E25C9A23E25467
:104F7000244BE25C002A19D12368002B04D042465E
:104F80008B2A01D0FFF726FA03B03CBC9046994625
:104F9000A246AB46F0BD00230093484605211A4ABD
:104FA000434603F04FFE83E7002298E7E5540DF0F7
:104FB0005BF9E1E7074B0521181C144A994603F0F9
:104FC00041FEFA235B016353FCE6C04614F4FF1F65
:104FD000D3F3000050580200102E020010270000EA
:104FE00024F4FF1F302E0200ACF0FF1FCC6702003C
:104FF0007CE0FF1F00670200C42C02006C5F02000F
:10500000A82E0200DB020000642E0200E82D020040
:10501000F0B54D4644465F465646F0B4CE4C87B098
:1050200031230022E25408F0F3FC201C1030CB495D
:1050300009F020F900226420C94909F0C5F9201CB3
:105040007C30C849FFF7E0F801258623201CE55491
:105050008830C549FFF7D8F89223E5548020C34B28
:1050600000021D7804F088FCAD06ED0F0223023526
:10507000034206D0011C80209943000204F09CFEEC
:105080001B25281CFEF7E6FEB94ABA4B04AD904634
:105090009946022608F0BCFC206D291C0A2209F062
:1050A000B5FD002862D12B784046052B00D1DAE00F
:1050B00005214A4603F0C6FD2B780C2B00D9DAE017
:1050C000AD4A9B00D3589F468020000204F054FC58
:1050D000011C80203143000204F06EFEDAE7A74B8A
:1050E000201C01226030A649E25408F065F8002235
:1050F0005C23E254CEE70DF0EBF9CBE70DF0B2F90B
:10510000C8E70DF09BF9C5E70DF068F9C2E79D48C7
:1051100008F05AF8BEE79A499B4808F04DF89A4AB9
:105120001721603A5C23D154B4E79549964808F0BA
:1051300043F8954A0021603A5C23D154AAE78120C4
:105140001521FFF771FCA5E70120FEF783FEA1E71B
:105150008020FFF711FE9DE789498B4808F02CF865
:10516000894A0521603A5C23D15493E73023E35CFC
:10517000002B00D101E2012B00D082E0834A1268AB
:10518000002A00D17AE2824808F02CF8002816D0D4
:105190007F4808F019F87D4B7E481B68DE0808F050
:1051A000A1FAC200121AD3175B0F9B18DB10774AC3
:1051B0009B191360764A508983429B415842B82319
:1051C000E054201CA43008F00DF8002800D03EE286
:1051D000AC23E35C002B00D106E2FEF7E5FD6E4850
:1051E00008F00CF8002800D016E26B4E0C22543E5A
:1051F00033681A4200D0F6E29A0704D58422A25CF2
:10520000002A00D034E31A0604D59022A25C002ABA
:1052100000D04EE3DA0704D59622A25C002A00D023
:1052200040E39A0600D5D4E2DA0608D59922A25CBA
:10523000002A04D09822A25C002A00D16DE3DA058E
:1052400000D5AEE29B23E35C9422A15C9522A1549D
:105250009622A15C9722A1549922A15C9822A15484
:105260009A22A35415E706214A4603F0EBFC2B785B
:105270000C2B00D824E740460421484A03F0E2FC06
:1052800008E70CF0DFFF01238622A3549222A354E7
:10529000354808F0D3FF424BE054002800D0E7E146
:1052A00004224C23E25440463E4A0423052103F0E5
:1052B000C9FC09F0F9FD4B23E25C3F2A09D9013A08
:1052C000E2544A23E25C0132D2B23F2A00D90022E2
:1052D000E2544926A75D04231737FF00E7193B7204
:1052E0000AF060F97860A35D0133DBB23F2B00D98F
:1052F0000023A3554B23E25C00260132E25409F05F
:10530000D7FD40460521284A03F09CFC3023FA21B2
:10531000E654490001233122201CA35410300A1CFA
:1053200000960193002305F09DFC5C231F48E65482
:10533000666608F04FFF404605211D4A03F082FCD7
:10534000FA20400009F040FC1A4B04261868002798
:10535000002838D144E0C04614F4FF1FFC6002006E
:105360003539010020600200685E020000F007404D
:1053700050580200B42E02000C2A0200DB0200008A
:1053800060EA000050F4FF1F74F4FF1F18E1FF1FD4
:10539000C4F4FF1F245E020068F4FF1FCC2E02003D
:1053A000DA020000C42C0200D82C02006C5F02005C
:1053B000E42C0200ACF0FF1FD64A331D90590028A0
:1053C0000ED0371C1E1C08F005FFD34AD059002808
:1053D000F2D009F0F9FBCF4A331D90590028F0D1E3
:1053E000CE4B002604CB002A21D004331A1F1268AA
:1053F0000136002AF9D1CA4AB300D2189346C74AE7
:105400000027D218924609E05246D319043B186887
:10541000013E08F0EBFE043F002E08D05A46D31997
:10542000043B18680028EFD009F0CEFBECE7BD483C
:1054300008F0D0FE642009F0C7FBBA4808F0D6FE99
:1054400002E0002009F0C0FBB74808F0F7FE002892
:10545000F7D0B64B042618680027002807D113E0C0
:10546000B24A331D905900280ED0371C1E1C08F07C
:10547000B1FEAF4AD0590028F2D009F0A5FBAB4AE3
:10548000331D90590028F0D10A2009F09DFBA74B4D
:10549000002604CB002A21D004331A1F12680136DB
:1054A000002AF9D1A24AB300D21893469F4A002796
:1054B000D218924609E05246D319043B1868013EBF
:1054C00008F094FE043F002E08D05A46D319043B3E
:1054D00018680028EFD009F077FBECE70521954A22
:1054E000E36A404603F0AEFBB42189006258531CC6
:1054F0006350002A00D039E18F4B1B789A0704D5FE
:10550000404605218D4A03F09DFB02223123E254DF
:10551000B2239B00E0188A4907F04EFE201C3C3065
:10552000884907F049FE201CFA219C30C90007F089
:1055300043FE201CA430642107F03EFE201CB03046
:10554000642107F039FE0CF049FFFEF72DFC94238F
:10555000E25C9523E2549623E25C9723E25499237C
:10556000E25C9823E2549B23E25C9A23E25408F025
:105570004FFAFEF7C3F9E0628BE5271C3C37FEF7D4
:1055800013FC381C07F03AFE061E5DD14822A35CCE
:105590009246002B7ED1626E002A00D18DE0201C45
:1055A000603007F01FFE002800D19CE15C23E75C1F
:1055B000052F00D1B8E17B427B418426F61A301CCE
:1055C000391CFFF731FA9423E25C9523E2549623C9
:1055D000E25C9723E2549923E25C9823E2549B23F4
:1055E000E25C9A23E25454E5AD23E35C002B00D146
:1055F000F3E523685B0500D4EFE540460521524AF8
:1056000003F020FBFEF7D0FB201C543007F0F6FD22
:10561000031C0220002B04D05C23E05C002800D196
:10562000D0E09423E25C9523E2549623E25C972336
:10563000E2549923E25C9823E2549B23E25C9A2390
:10564000E254FEF707FC24E516278226B7E7FEF7AB
:10565000A3FA002800D1BBE5404604213B4A03F0F1
:10566000F1FA3B4B01228820E254FFF785FB10E55D
:1056700040460521374A03F0E5FA11E6364808F0BE
:1056800031F8364A031C106006214046344A03F0C4
:10569000D9FA78E5616C381C07F08EFD5346E65464
:1056A000236C40460521002B00D0B3E02D4A03F0C7
:1056B000C9FA626E002A00D071E71B4808F0BEFDEF
:1056C000002800D1CCE0B326B600A259002A0DD0A4
:1056D000B1239B00E758002F00D0B5E0B2239B0018
:1056E000E01807F07FFD002800D0A7518423E35C79
:1056F000002B00D092E01C4807F074FD002800D178
:1057000061E7FEF749FA002800D15CE70027882608
:1057100055E7C046ACF0FF1FCC6702007CE0FF1FDE
:1057200000670200706002005C60020010F4FF1F5E
:10573000D4670200F02C020000F00740242D020084
:10574000DC050000A0BB0D00842F02004C2F0200DE
:10575000DB020000B02C0200245E020018E1FF1FF3
:10576000342F0200F82E0200B8F4FF1FB126B60055
:10577000A259052140460092784A03F063FA09F0E5
:1057800093FB00237648A35108F058FDAF239B00FC
:10579000E05409F01DFAB0239B00E05009F088FBAB
:1057A000B3E69B23E35C002B00D14DE59A23E35C39
:1057B000002B00D048E5404605216A4A03F042FA32
:1057C0001D202EE740460521674A03F03BFA0420DE
:1057D00027E7664807F012FD002800D096E0634BEB
:1057E000343B1B6820E56248143007F007FD0028B1
:1057F00007D09423F35C002B03D09523F35C002B9C
:1058000001D02368F8E4404605215A4A03F01AFA09
:10581000102006E7584A03F015FABCE68623E35C3D
:10582000002B00D067E78723E35C002B00D062E702
:1058300009F0CEF98023E3581827C01A4F4B892668
:10584000984200D9BBE656E7E3584D4A4046052149
:1058500003F0F8F9B52200239200A351A35045E7C5
:1058600040460521474A03F0EDF987260127A6E6C1
:105870008622A25C002A00D0C5E48722A25C002A0E
:1058800000D0C0E409F0A4F98023E358C01AF4233F
:10589000FF3398425DD9404605213B4A03F0D2F9D7
:1058A0001120BEE640460521384A03F0CBF912200C
:1058B000B7E69222A25C002A00D0ABE49322A25C5D
:1058C000002A00D0A6E409F083F98C23E358C01A1B
:1058D000F423FF3398423ED9404605212C4A03F079
:1058E000B1F91F209DE62B4808F0A8FC00281DD028
:1058F000294808F0A3FC002800D1E4E65C23E75C1B
:105900008B26002F00D15AE6862658E64046052110
:10591000224A03F097F9142083E640460521204AE5
:1059200003F090F913207CE68C2648E65C23E75CC4
:10593000052F0CD07B427B418626F61A164808F0CC
:105940007DFC0028DAD1002E00D13CE637E68C261B
:10595000F4E7236857E423685CE4C046002D0200A6
:10596000BC5F0200F82F0200A82F020048F4FF1FBE
:1059700068F4FF1FB82F0200E42E02000F2700007A
:105980001C2F0200082F020014300200C82F020052
:10599000283002005C600200945F0200D82F0200F1
:1059A000E82F020008B558680CF0CCFDC0B2FEF735
:1059B0008DFC002008BDC04608B50220FEF786FC1D
:1059C000002008BD144970B51E1C0B6C041C151C6E
:1059D000002B16D0081C3C3007F020FC0F49021C9D
:1059E000201C05F00FFE012D09DD706820220378D0
:1059F0009343482B09D00CF0A5FDFEF71DFC0020B9
:105A000070BD074905F0FEFDEDE70649201C05F0D5
:105A1000F9FDFEF709FCF2E714F4FF1FB4300200B1
:105A2000D0300200E4300200F0B544465F464D46F7
:105A30005646F0B41D4F85B003924B23FB5C814664
:105A4000984642464A23FC5C002A1DD0184A3F2350
:105A5000002593469A460026221C1732D200BA1817
:105A6000137A52684846009259462A1C013405F0C0
:105A7000C9FDE4B2331C5246A24273415B42013578
:105A80001C40EBB29845E7D8039B012B05DDFEF7E0
:105A90000DFC4846074905F0B5FD002005B03CBCAB
:105AA00090469946A246AB46F0BDC04614F4FF1F8F
:105AB000F03002000031020000B583B0012A0DDD94
:105AC0005A680A496B4605F0B7FD002806D16A46B8
:105AD0001378002B05D10020FEF7F8FB002003B05F
:105AE00000BD0120FEF7F2FBF8E7C04618310200C6
:105AF00008B5024806F074FC08BDC0463C30020000
:105B0000F0B55F4656464D464446F0B4A1B09346C4
:105B1000824605935922002308A88946129383548C
:105B20005F463978002931D0081C2038C3B20137CC
:105B30005A2B66D8764B4AB29A18203A12780F251B
:105B40001540ED00592208AEB4565B191B5D1B09C8
:105B5000B354072B4ED86F4A9B00D3589F46423907
:105B6000C9B2362900D9B9E26B4B89005B589F4610
:105B700049B26C2961D07A29D3D1139A03239A436D
:105B800002231343139339780029CDD1129821B001
:105B90003CBC90469946A246AB46F0BD139E0423FA
:105BA000334349B213932A2955D0109B30399A00B8
:105BB000D3185B0059181091B3E749B22A2943D092
:105BC000119B30399A00D3185B0059181191A8E73E
:105BD000C0B21028A5D8514B80001B589F46002307
:105BE0001093119314930F9313932022582308A812
:105BF000C25496E749B24846D047129B01331293EC
:105C00008FE70025424B9DE73022582308A8C25455
:105C100087E7139E08233343139382E7139C4023A3
:105C2000234313937DE7139A20231343139378E7B9
:105C3000139910230B43139373E7139A03239A4387
:105C40000123134313936CE70599059C09680434F9
:105C50001191059465E70598059C0068043410903F
:105C600005945EE7139E802333431393059C0598A8
:105C7000216804300A91002900D1A9E20023CB5603
:105C8000002B00D1AEE20B1C013300229A56002AF1
:105C9000FAD15B1A0F93139B05909E0500D42CE15B
:105CA0001098002801D101221092190500D540E278
:105CB00003221A40012A00D179E2002A00D16DE2C4
:105CC000022A00D035E2059C802122684900043474
:105CD0000892194005949E0602D5002A00D114921C
:105CE000141C00290AD0002A00DA50E213998220FD
:105CF000C0000840141C102800D13FE26D467635E4
:105D0000D90400D50A9D064B57229346984628E0B1
:105D1000183502008C330200AC33020088340200D4
:105D2000D434020008AE5846335C082B00D1E1E1C0
:105D3000102B00D1DAE1022B00D1D3E1201C0A2183
:105D4000FAF70EFA201CCEB20A21FAF7C5F9041CA4
:105D50006B1E41460A938B5D2B700F9B0A9D01338E
:105D60000F93109B5A1E1092002BDBDC002CD9D114
:105D70006B1C0A938822139BD200134200D0DDE1F2
:105D8000119A0F99149C0919521A1192129E002C03
:105D900000DCC4E00025190674D408AA5319342184
:105DA000595648460135D047A542F6D1139BAD1947
:105DB00012951C071FD41199582208A80C1C865C48
:105DC0008846013C002900DCFCE176B24B46321CDF
:105DD000A94656461D1CBA46171C281C391CB0473C
:105DE000013CFAD22B1C4D469946139B574642461E
:105DF000B246AD1812950F9E80220A9C1A40002EC2
:105E000000DCADE1002A00D078E1A31998463A1CE5
:105E10002B1C4F464546B1469846564692460021B1
:105E20006156381C0134B047AC42F8D15346B246F3
:105E30004E46B9461F1C139B454675191295190706
:105E400000D46EE6582308AAD65C119B1C1C984609
:105E5000013C002B00DCB3E176B24B46321CA94674
:105E600056461D1CBA46171C281C391CB047013C5D
:105E7000FAD22B1C57464D46B246994643465D1909
:105E800012954EE608A94B1934331978CBB21A1C77
:105E9000613A192A01D8203BD9B249B248460135A6
:105EA000D047A542EED181E7059C059823680430D0
:105EB000002B00D088E1D6490A910023CB56002B55
:105EC00000D18FE10B1C013300229A56002AFAD12F
:105ED000DFE6139E80233343139305986A465632B8
:105EE0000068059C0A9208A93622885404340122CD
:105EF0000F9205949E0500D5D2E6119A0F99002ABB
:105F000000D114E18A4200DB11E1149C111C091933
:105F10000F92521A1192129E002C00DD3AE70025D2
:105F200045E7139E8023334303229343B94A08A8CD
:105F3000134310215722815408222D21109234221C
:105F4000815435223E218154022213931492A4E6F7
:105F500013988022024380239B0013431020572173
:105F600008AC13936054960600D496E63021342290
:105F7000A15435227821A154022214928DE6139A5D
:105F800080239B0013430221572008AC1393215414
:105F9000960600D481E630203422A05462203522B7
:105FA000A054149179E6139B97E78022139852002E
:105FB000024380239B0013430A21572208AC13930A
:105FC000A1546AE6139AF4E7139AC4E7139E301CAF
:105FD000B04640076CD40623109305248E4BE40092
:105FE0001C192568666881497F482A1C331CFBF709
:105FF0002BFC06900791059B07220895099607330D
:1060000093431C1C186859680834794A794B0594E5
:1060100002900391FAF726F9002800D044E1069A8D
:10602000079B02980399FBF7EDF802900391FCF7A8
:1060300039FE83460E90FCF7A7FE021C0B1C02984B
:106040000399FCF7FBFA84460C1C231C6246281CAF
:10605000311CFCF763F80C900D91FAF7C1F908AE0A
:1060600057230A226D46F254109B7635041C0A957C
:10607000002B00D0D8E0694B4446234300225E4603
:1060800013931092089608E6139A80239B001343FB
:106090000820572108AC13936054960600D4FCE501
:1060A00034223021A15401221492F6E5139B3BE7E0
:1060B000109C002C00DC8EE0062C00DC86E04E4DAF
:1060C0004E4E063C281C311C4D4A4E4B013CFCF701
:1060D00025F8002CF8D1051C0E1C84E700230F9333
:1060E000139BDAE501262640640831E60F26264098
:1060F00024092DE607262640E40829E6A0192B1CD2
:106100003A1C051C4F469846B146564692462178A1
:10611000CBB21A1C613A192A02D8191C2039C9B20B
:1061200049B2381C0134B047AC42F0D17EE6149C31
:1061300029E6802149001940089ACCE52D225C050A
:1061400000D42B22582108AE715630290AD00A9566
:106150002A700F99119A01310F91149C139B12E62A
:1061600000266AE601211491342172540F9A119885
:106170000132821A1192129E01240BE6342320224E
:1061800008A8C25401231493089C0B1CB6E5802177
:10619000C90052420B4308921393A7E5059C802146
:1061A00022684900043419400892059493E5059E3D
:1061B00080213268490004361940089205968AE524
:1061C00000235CE6002214E6154975E6013C05E76C
:1061D00014490A9152E5054A03490B4D0B4E0691AD
:1061E000079208E7002355E5000000000000E03FAB
:1061F00000000000000000000000000080842E412C
:106200000000000000002440000000000000F03FFB
:10621000CC34020002020000E8340200011B00003E
:106220007C350200743502002F495720834688468A
:106230001CE008AA5E46935D082B31D0102B2BD0B2
:10624000022B25D0201C0A21F9F78AFF201CCEB290
:106250000A21F9F741FF041C6B1E40460A93835D37
:106260002B700F9B0A9D01330F93109B5A1E1092A7
:10627000002BDEDC002CDCD16B1E0A932E232B704E
:106280000F9B13990E9A01330F9388469346F2E6BB
:10629000012626406408DFE70F2626402409DBE7B5
:1062A00007262640E408D7E78023DB004146194350
:1062B0001391069A079B884602980399FCF7BEF94A
:1062C00002900391FCF7EEFC83460E90FCF71EFD56
:1062D000021C0B1C02980399FCF7B0F980221206ED
:1062E00084468C18B1E6C046D4340200C046C0468D
:1062F0000CB400B583B004AB04CB0193FFF700FCF2
:1063000003B008BC02B0184710B508600730C008D9
:1063100048600C1C08F044FCA060002803D06268B0
:1063200000210CF088F910BD4368073110B5C90889
:10633000041C994207D88068002803D062680021B5
:106340000CF079F910BD4160806808F02DFC6068A0
:1063500008F026FCA060EFE7031C1A6800208A42C0
:1063600009D99B68002B06D0CA0807209B5C014016
:106370000B4101201840704703688B420CD9836899
:10638000002B09D0CA089B180722114001228A401D
:10639000111C1A78114319707047C04630B5002996
:1063A00010D00123084D41185B42FF2402780130D0
:1063B0005A4022409200AA581B0A53408842F5D105
:1063C000D84330BD0020FCE7843502004140FF2364
:1063D0001940034B8900CB58000A58407047C0460B
:1063E00084350200012040427047C046C0437047D8
:1063F00030B5002A0CD0074D8A18FF240B780131E4
:10640000434023409B00EB58000A58409142F5D18D
:1064100030BDC0468435020038B5041C0D1E12D0B4
:10642000081C0CF018F900280DD0291C2818074D5D
:10643000FF220B780131634013409B00EB58240A84
:106440005C408142F5D1201C38BDC0468435020035
:1064500010B5054C031C4118FF201A780133504039
:10646000205C8B42F9D110BD84390200F0B55F4643
:1064700056464D464446F0B489B0059303680391EF
:106480000492DA89061C0027FF2002978346002A1F
:1064900000D168E0181C029906AA01F047FE002806
:1064A00027D1F1880191002923D0708933894700D1
:1064B000069A98460124BC46611E89B245464D4362
:1064C000ADB25319009119785F46090639438A46DF
:1064D000195C574609040F4361465B5C1B023B4352
:1064E000224FBB421ED00199A14202D90134A4B26D
:1064F000E2E700253068002101F0B8FD029B01337E
:106500009BB202933368029FDA89BA4227D90028E6
:1065100001D1002DBED009B03CBC90469946A246A0
:10652000AB46F0BD029F019B00987B43039FC118BF
:106530003960B3890498ED185219059FB847F1885E
:10654000051C0191A142D5D90028D3D17089338986
:10655000470001349846069ABC46A4B2ACE7002D29
:10656000D9D10028D7D11620D5E7C046FFFF0000BB
:10657000F0B5564644465F464D46F0B48BB00590A4
:106580000E1C0792181C142200211C1C0CF053F83E
:106590000598A680036820609B681B8A63811A1C8B
:1065A000042B00D2042259005B189A1890B2A081E3
:1065B00008F0F6FA658920617019291C0138F9F78D
:1065C000D9FD011C6943059AA389C918136889B2CA
:1065D0009B682181D868F9F77FFD059B22689B683D
:1065E000E0800393A38800040093D389000C434305
:1065F000052101935148039B514A02F023FB206877
:10660000C389002B00D197E000220692934608AA86
:106610000598594601F08AFD00220492002850D1C5
:10662000E3889946002B4CD0FF20002582461CE0D1
:106630007A1C16D0FF2F14D05A46009201963F487C
:106640000421404A3B1C02F0FDFA638900215A00F4
:10665000D218089B98190BF0EEFFE08801228146C2
:1066600004920135ADB24D452BD22689089A6E436E
:106670006389B6B290469219590017785118D25CC6
:1066800050463F060743120417430A7809A812022E
:10669000C918174304220BF0ACFF2B4B9F42C7D104
:1066A000A089A18830184044FFF778FE099B9842E2
:1066B0001CD0009621480421244A5B4602F0C2FA0D
:1066C000C3E70598049901F0D1FC5B4601332268C9
:1066D0009BB29B46D3895B4517D9002897D00BB056
:1066E0003CBC90469946A246AB46F0BDE0885A466F
:1066F0005043A189089B761828189919079A904742
:10670000E388012099460690ABE70028E7D1069878
:10671000002811D1002B0FD00025059E01E0002894
:10672000DDD1291C301C01F01BFC22680135D38906
:10673000ADB2AB42F3D8D2E70020D0E7843A0200F2
:10674000903A0200CC3A0200FFFF0000AC3A02008F
:10675000F0B54D4644465F465646F0B4C688041C24
:1067600085B00D1C081C311C9046F9F7B5FC311C96
:1067700087B2281CF9F7F4FC23892069594389B2B0
:1067800089460090A3892068391C4A4601F0FAFA2C
:10679000002806D005B03CBC90469946A246AB46C0
:1067A000F0BD216966898A4653461A785046FF2310
:1067B00012061A43835D710051441B041A430B787F
:1067C00003A81B021A439346891904220BF011FFF8
:1067D0005946013109D05846009004212A482B4AD5
:1067E0002B1C02F02FFA1620D4E7002E09D000252A
:1067F00000235246535566890135B542F9DB2369BA
:106800009A4650460090391C20684A46331C01F0D5
:10681000FDFA0028BED1A28941464A44009192B2B5
:10682000A3882068391C01F0F1FA0028B2D16589EB
:106830002069002D25D00022401900218154638950
:1068400001329A42FADB206949464A194019009000
:1068500092B22068391C01F0D9FA00289AD1A18897
:106860004046FFF79BFD638903905A009A184A44FB
:1068700003AB0093206892B2391C042301F0C6FADE
:1068800088E70023E0E7C046843A0200F43A0200B9
:10689000F0B5474680B4C488051C0E1C82B0081CA5
:1068A000211CF9F719FC80B28046211C301CF9F735
:1068B00057FC2B890A1C5A436B8992B25F00B9B20C
:1068C0002E69002B08D0F719002400263E556B894D
:1068D00001349C42FADB2E6976185218286892B26D
:1068E0000096414601F092FA02B004BC9046F0BD19
:1068F000F0B55F4656464D464446F0B489B0079120
:106900000168061CCB89894600218B4606910591BA
:106910005B4560D9F488002C57D0002200233769EA
:10692000924603935D4665435544211C281CF9F7A4
:10693000D3FB80B28046211C281CF9F711FC338957
:106940000A1C5A43009792B2B3894846414601F067
:1069500019FA002806D009B03CBC90469946A246D8
:10696000AB46F0BD376973893978FF2209061143B8
:10697000FA5C5B0012041143DA5D0B1C1202134334
:10698000013309D053460133F4889BB29A46A3429F
:1069900008D232689146C5E7039B049501339BB248
:1069A0000393EFE7039B002B1CD00599002902D02D
:1069B000069A934216D9049A079B31681A60CB89CC
:1069C000894603990122069105925A46013292B2F4
:1069D00093465B459ED805991C204B424B415B4238
:1069E0001840B8E75A463368013292B29946934646
:1069F000DB89EEE7F0B556465F464D464446F0B4B7
:106A0000374A061C87B03748052102F01BF9306869
:106A1000C289002A61D00023FF279946B84649461B
:106A200004AA01F083FB002834D1F38800279C4698
:106A3000002B50D02C4BBB4600249A46039761464E
:106A400003E00134A4B28C4222D23289049F101C8C
:106A5000604380B23818057873892D0647462F4366
:106A6000C55C5B001B5C2D043D431B022B43FF2BCD
:106A700001D05345E5D1FF210BF0DDFD039B01342F
:106A8000F18801330127A4B20393BB468C42DCD3C7
:106A9000039F01E00027BB465946306801F0E6FA43
:106AA0004B460093041C3B1C0E4805210F4A02F084
:106AB000C9F84B46013330689BB29946C3894B45B0
:106AC00001D9002CABD0201C07B03CBC90469946A5
:106AD000A246AB46F0BDBB46DEE70024F3E7C04666
:106AE000483B0200843A0200FFFFFF00543B0200D3
:106AF000F0B55F4656464D464446F0B4374B89B034
:106B00001968071C8A46002964D03549354A412353
:106B100098468B4691465946381C04F073FD5346FF
:106B20009A680025D6681089311C4143890A136888
:106B3000128A039189020139009201900491029610
:106B40002949381C424604F05DFD51464C68002C32
:106B500021D041463B1C07919846E189A089321C0F
:106B6000331C4A434343A7680493D3180291013B63
:106B7000910A01900391059300972B1C40464946CA
:106B8000079A04F03FFD64680135002CE5D10799B0
:106B900043461F1C884653469A8B002A12D113493C
:106BA000381C04F02FFD53461A6801219246884490
:106BB000002AB0D1002009B03CBC90469946A246BC
:106BC000AB46F0BD331C5343381C9B0A084904F004
:106BD00019FDE4E7074904F015FDEBE728E1FF1F85
:106BE000003C0200743C0200443C0200304A0200B7
:106BF000A03C0200E43B0200F0B55F464D4656461D
:106C00004446F0B40023136083B08246081C0F1C76
:106C100090460BF020FD3C4B051C18680121814675
:106C20008B46002868D0484683681C68201C0BF0FF
:106C300012FD85423ED94A465668002E08D0B468F7
:106C4000201C0BF008FD854213D97668002EF6D182
:106C50004B461A689146002AE5D1012041460B684F
:106C6000002B49D003B03CBC90469946A246AB46A7
:106C7000F0BD381C211C2A1C06F0BEF90028E4D106
:106C800040460268002A0AD049468B6850461B6875
:106C90001E4900923A1C04F0B5FC0020DEE7B36800
:106CA0004046494603604160B3890381F38902731A
:106CB0004381CAE7381C211C2A1C06F09DF90028D4
:106CC000B9D141460A68002A09D04846836810496C
:106CD0001B68504600923A1C04F094FCDDE74946DC
:106CE0008B68414618680A810860484648601B89DD
:106CF0004B815B460B739EE7504606493A1C04F0F5
:106D000081FC0020AEE7C04628E1FF1F283D0200BD
:106D1000F43C0200C83C0200F0B5444656464D46DD
:106D20005F46F0B487B002AE151C9968321C8046ED
:106D30001C1CFFF761FF002807D1002007B03CBCF6
:106D400090469946A246AB46F0BDE0680BF0FAFBD0
:106D50008346042D43DC01229246002406E02349A9
:106D60002A1C04F04FFC0134A245E6DD33895A4663
:106D70009D1872892D199B1840469D42EFDC3268A0
:106D80002B1C1B4904F03EFC7768ABB2BA689946ED
:106D900013894B4510D82B04164A1B0C16480421A6
:106DA00001F050FF02229146009540461349326897
:106DB0004B4604F027FCD6E7B86908F08BF87B69EE
:106DC000B86801337B6143684946DB689847814670
:106DD000B86908F085F84B46002BC4D0E4E7206979
:106DE0000BF0B0FB82460028B7DCA6E75C3D020052
:106DF000783D0200903D02008C420200A83D020056
:106E000070B528220C1C84B0061C081C00210BF055
:106E100012FC204B201C1A68A660226018301C60EF
:106E200008F04AF8051E1BD033891B4EA383A368C4
:106E3000301CD9681A891B6800924A43920A019152
:106E400002920521154A01F0FDFEA368301C1B6863
:106E500004210095124A01F0F5FE281C04B070BD13
:106E6000A06843681B68984733890B4EA383A368C7
:106E7000051CD9681A891B6800924A43920A01913D
:106E80000292301C0521054A01F0DCFE002DE4D001
:106E9000DBE7C04628E1FF1F8C420200C83D02002C
:106EA000D83D0200F0B5474680B4041C82B080692A
:106EB0000D1C171C08F00EF8266AA584002E33D08E
:106EC000A368D9688846002902D08AB242450DD904
:106ED0001A4804211A4A01F0B5FE0226A06907F0FB
:106EE000FFFF301C02B004BC9046F0BD1B89AB42D2
:106EF000EED9A06907F0EEFFA068E36842680133AD
:106F0000414600965668E36000228BB2291CB047C8
:106F1000061CA06907F0E4FF002EDFD1226A2623B9
:106F20003A600122E254DCE7A3680C26D86807F037
:106F300037FE20620028D1D0061CC1E78C42020037
:106F4000203E0200F0B52623C25C83B0041C00255D
:106F5000002A08D0026AC554002A01D0002905D1B0
:106F6000A06907F0BDFF281C03B0F0BD8268858CC6
:106F70001389AB4207D82B1C1E4804211E4A01F07E
:106F800061FE0225ECE7806907F0A4FF6369A06851
:106F9000013363614368291CDB689847051CA069BD
:106FA00007F09EFF002DDBD1A368A68CDD68276A61
:106FB000002D02D0AAB2AA4206D90E4804210F4AD7
:106FC00001F040FE0225CBE71B89B342F5D9A06949
:106FD00007F080FFA06823694268013300972361AE
:106FE0009768ABB2311C0022B847051CA06907F0B6
:106FF00077FFB5E78C420200903D0200383E020068
:10700000F0B55F4656464D464446F0B4814683B0DF
:10701000884692469B46002A4AD049468D6840469B
:10702000EC68211CF9F79CF80B040E1C1B0C9C420D
:1070300006D9E71A574500D95746DB199C420DD2AD
:107040001C4804211C4A01F0FDFD0224201C03B051
:107050003CBC90469946A246AB46F0BD211C40463A
:10706000F9F73AF82B8984B2A342E9D94A469069E4
:1070700007F030FF4946CB6888680133CB6043682E
:1070800059460091BDB2B2B2211C5E682B1CB047BC
:107090004A46041C906907F023FF53465D1BADB2BE
:1070A000AA46B844BB44002DD0D0002CB5D0CDE7C3
:1070B0000024CBE78C420200203E0200F0B5564689
:1070C0004D4644465F46F0B489B0161C99686A463E
:1070D000051C1C1CFFF790FD00282CD000218946C0
:1070E000032E69DC281C3949009A4B4604F08AFAC1
:1070F000281C04F09BFC00281DD001986946836879
:107100004A89DB685A43914515D2314A3149324F99
:10711000924688466A4611894A464B43991810227E
:1071200004ABFFF76DFF021C281C002A0BD02B4973
:107130004B4604F067FA002009B03CBC90469946E3
:10714000A246AB46F0BD51464A4604F05BFA012622
:10715000002401E00134013604AB41461A5D281CCD
:1071600004F050FA281C391C072C2AD0202204F0E5
:1071700049FA102EEED108A904AC8B4623782E22B2
:10718000191C20395F2900D81A1C281C391C01340D
:1071900004F038FA5C45F1D11022281C914404F027
:1071A00045FC0028C7D00198694683684A89DB6896
:1071B0005A434A45AED8BEE7E06806F025F9814655
:1071C00090E72E2204F01EFAC4E7C046503E0200AB
:1071D000903E0200DC2E0200983E02006C3E02004F
:1071E000F0B544464D465F465646F0B48DB008AC07
:1071F00000226281228162609968221C8146FFF729
:10720000FBFC002807D100200DB03CBC90469946FD
:10721000A246AB46F0BD4049089A484604F0F2F950
:1072200004AA21896068FFF73DFE06A805F0CCFF9F
:107230003A4A0025A846934667680499BB682289A4
:10724000DE688A46002E02D0B1B2B14217D9344866
:107250000421344A01F0F6FC022622894846AA1885
:107260003149331C04F0CEF963682622995C002969
:10727000C9D000219954986907F032FEC3E7AA18D3
:1072800092B203921B899342E1D9B86907F022FEBA
:10729000FB68B868013342685146FB600091B3B2A5
:1072A000039956680022B047061CB86907F018FE1B
:1072B000002ED2D1636806A89B680135DB68ADB2A9
:1072C000984405F087FF6389011C9D429B411D4046
:1072D0005845B1D94246D000F8F7FEFEFA27BF0064
:1072E0003D1C4543114EB54210D9311C281CF8F7FE
:1072F000F3FE80467043391C281AF8F7EDFE0C495E
:10730000031C4246484604F07DF9ADE7484609496A
:107310002A1C04F077F9A7E79C3E0200E70300006F
:107320008C420200203E0200B03E020040420F00AC
:10733000D03E0200E43E0200F0B556464D465F46A0
:107340004446F0B44B8983B0061C0D1C002B00D1C1
:1073500091E0574A574B012491469A46631E9BB2CF
:107360002A8998464244301C494604F04BF96F681C
:107370002B89BA6843449BB298461389434517D872
:107380004D4A43464D48042101F05CFC02229046E0
:10739000301C4B49424604F035F96B89A34223D98E
:1073A000404603B03CBC90469946A246AB46F0BD71
:1073B000B86907F08FFD7B69B86801337B6143686A
:1073C0004146DB6898478046B86907F089FD434627
:1073D000002BDDD1301C514604F014F96B89A34217
:1073E00062D90134A4B2B9E7002B57D04346002B31
:1073F000D6D1344B002299462E4B904626229246F7
:107400009B462A8949464244301C04F0FBF82989EE
:107410006F68414489B2381C01AAFFF743FD002878
:1074200033D1BB68D968002936D0019800230022E7
:1074300001E0002C09D1845C0133FF3C621E9441C1
:107440009BB2E4B21A1E8A42F3D35246BB5C002BB5
:1074500004D00023BB54B86907F042FD002C14D1BE
:10746000301C594604F0CEF8434601339BB298468F
:107470006B899845C5D32A89301CD318013B124922
:1074800004F0C0F8002290468AE7301C0F4904F04F
:10749000B9F80122904683E70024D6E74346002B43
:1074A00000D07DE70023E6E7002BA2D10023E2E72E
:1074B000F03E0200083F0200903D02008C420200B4
:1074C0000C3F02001C3F0200403F0200343F02001C
:1074D000F0B556464D4644465F46F0B485B00C1CA8
:1074E0000390151CFFF728FF63898246002B00D10B
:1074F00012E100282DD101218B4623895F46013FEF
:10750000FF18BFB22A1C3B1CA249039804F07AF86A
:10751000BA466768B86907F0DDFC3E6A5246BA842D
:10752000002E67D0BB68D9688946002902D08AB28C
:107530004A4516D998480421984A01F083FB022352
:107540009A46B86907F0CCFC03989549524604F076
:1075500059F8504605B03CBC90469946A246AB4609
:10756000F0BD1B895345E5D9B86907F0B3FCFB684A
:10757000B86801334268FB60494600968BB2566892
:1075800051460022B0478146B86907F0A9FC4A4637
:10759000002A00D0F6E0012326223E6ABB5463682D
:1075A000291C9B68301CDA680BF045F861680A1CDE
:1075B00088462621535C002B27D142469368FF2141
:1075C000DA68301C0BF037F86768BB68D968884602
:1075D000002902D08AB2424534D96F4804216F4A4B
:1075E00001F030FB02239A4603986E49524604F09C
:1075F00009F8AEE7BB68D86807F0D2FA386200280D
:1076000000D0C1E00C218A469BE74B465354116AD7
:10761000002900D18BE0978C92681389BB424DD82A
:1076200004215D48604A3B1C01F00CFB02218A46A4
:107630004346986907F054FC03985C49524603F0AE
:10764000E1FF86E71B895345C7D9B86907F042FCBB
:10765000FB68B86801334268FB60414600968BB214
:10766000516800228C465146E0478146B86907F0D0
:1076700037FC4A46002A00D082E063689B68D968DC
:107680000023002907D0F35CAB4210D1013292B243
:10769000131E8B42F7D30398454903F0B3FF638968
:1076A0005B453CD95B4601339BB29B4625E741498C
:1076B000039803F0A7FF01218A464AE743469869E9
:1076C00007F008FC41464B69886801334B61436809
:1076D000391CDB68984742468146906907F000FCF8
:1076E0004B46002B4AD141464246928C8B689146CC
:1076F000DF680A6A0292002F02D0BAB2BA421CD9DD
:10770000254804212C4A01F09DFA4246906907F071
:10771000E7FB02239A468FE7002800D019E7039879
:1077200026492A1C03F06EFF00239A4611E7906950
:1077300007F0D6FB626890463FE71B894B45DFD9CF
:10774000886907F0C7FB41460B69886801330B6104
:10775000029942680091BBB2494697680022B84737
:1077600042468146906907F0BBFB4346986907F0A3
:10777000B7FB4946002909D0CA465DE7CA4657E724
:10778000CA4631E7CA46DCE6061CCBE66168884695
:1077900013E7C046643F02008C420200203E020014
:1077A000883F0200D03F0200903D0200F03F0200FF
:1077B000083F0200A03F0200383E020008400200DD
:1077C000F0B54D465F4656464446F0B48BB006AD24
:1077D00000226A812A816A6099682A1C071CFFF7C7
:1077E0000BFA002807D100200BB03CBC904699460C
:1077F000A246AB46F0BD6A892B89D1490092381C5C
:10780000069A03F0FFFE381C291CFFF795FD00289F
:10781000E9D16B89002B00D115E10121894604AC27
:10782000BA462F89C749013F4F44BFB2FEB23A1C46
:10783000504603F0E7FE731C6370B31CA370F31C87
:10784000E370331D2371731D6371B31D6A68A371E7
:10785000F31D2670E37193689346111CDA68072ABA
:1078600000D99EE0B84AB948042101F0EBF90222A0
:1078700057469046381CB649424603F0C3FE6B8912
:107880009945B0D3002B00D1D9E041460029AAD1B7
:10789000B04B002291469A46BB462E89AE494E44D3
:1078A000B6B2321C584603F0ADFE311C03AAF6B244
:1078B0006868FFF7F7FA731C6370B31CA370F31CBE
:1078C000E370331D2371039F731D6371B31DA37197
:1078D000381CF31D211C08222670E3710AF07AFE81
:1078E00000284FD1331C08332370013363700133F8
:1078F000A3700133E37001332371013363710133EA
:10790000A3710F366B68E6719B680821DE684942F7
:1079100089198846201C791808220AF05BFE002885
:1079200037D1103E08220823082E07D9FB5CFF2B15
:1079300014D1013292B2131C9642F7D887495846A7
:1079400003F060FE6B682622995C002600290FD0A8
:1079500000219954986907F0C3FA09E05846514646
:1079600003F050FE6B6801262622995C0029EFD1B6
:107970004B4601339BB299466B8999455DD2002EE7
:107980008BD030E75846764903F03CFE01266B6801
:10799000EAE758467349424603F034FE01266B6815
:1079A000E2E71B89BB4200D85CE7886907F092FADE
:1079B00059460B69886801330B61436800949A68E3
:1079C000391C944608230022E0475B4680469869AC
:1079D00007F086FA4146002900D035E1331C083310
:1079E0002370013363700133A3700133E3700133FB
:1079F00023710F3601336371E67101336E68A37131
:107A0000B268D368191C083989B288468B4202D9FA
:107A100008318B4241D24D4804214B4A01F012F902
:107A20000223574698466B68381C9B684E49DA68B3
:107A30004346083A03F0E6FD21E7B0465F4642467A
:107A4000002A00D0CFE62A894849D318013B381CC8
:107A500003F0D8FD381C291CA522FFF739FD0028AA
:107A600000D0C0E66B461A8C4149381C03F0CAFDB1
:107A7000079C6946A2680E8C1389B34238D804214A
:107A800032483C4A331C01F0DDF802218846381C9C
:107A90003949424603F0B6FDA5E61389BB42BAD97F
:107AA000B06907F017FA3369B0680133336143688E
:107AB0000094996842468C460823391CE04780466A
:107AC000B06907F00DFA4246002A00D0BAE05046ED
:107AD000224903F097FD6B89994504D24B46013347
:107AE0009BB299469DE65746002B00D0D0E6AAE708
:107AF000A06907F0EFF96369A06801336361436827
:107B0000311CDB6898478046A06907F0E9F94346D5
:107B1000002BBCD1079A6B4604AC9146101C198C03
:107B2000221CFFF7BFF9002872D149468B68D9683B
:107B3000002900D182E004980023002220E0C04602
:107B40003040020058400200383E02008C420200E1
:107B500090400200C8400200A8400200083F020016
:107B6000F8400200E84002007840020008410200AC
:107B70002C410200903D020068410200002E09D114
:107B8000825C0133FF3A561EB2419BB2D6B21A1E36
:107B90008A42F3D326234946CA5C002A04D0002235
:107BA000CA54886907F09CF9002E31D16B46198CB4
:107BB000079A01319046101C89B2221CFFF772F916
:107BC00000282AD141468B68D968002938D004980A
:107BD0000023002201E0002C09D1845C0133FF3C2A
:107BE000621E94419BB2E4B21A1E8A42F3D326234A
:107BF0004146CA5C002A04D00022CA54886907F0B2
:107C00006FF9002C09D1381C104903F0FBFCEAE5A0
:107C1000381C0F4903F0F6FCE5E50E49381C03F06B
:107C2000F1FC381C291C5A22FFF752FC002800D016
:107C3000D9E5381C291CFFF77FFBD4E50026A9E70E
:107C40000024D4E75746EEE6574613E64C410200BF
:107C500040410200083F0200F0B54F464646C0B41E
:107C600085B00C9E80468946151C00211C22301CC4
:107C70001F1C0AF0E0FC41464A4688683160B26049
:107C8000F781B58103899D4259D2E919994234DCC3
:107C9000424653686A009446002B0BD09A8995425D
:107CA00003D3DC891419A54254DB914235DC5B68AF
:107CB000002BF3D141468A8B4C684346D21B0433D8
:107CC0008A83002C04D106E0231D6468002C02D0B6
:107CD000A289AA42F8D9746042461E6001970095B5
:107CE00093682248DB6805215F43BF0A0297204A58
:107CF0004B4600F0A7FF00200AE0009501970068BE
:107D0000042102901B4A19484B4600F09BFF1C209F
:107D100005B00CBC90469946F0BDDC89A21894458C
:107D2000C5DC009501979B68042102930068124A04
:107D300003904B460D4800F085FF1620E8E70095BC
:107D40000068042101900D4A08484B4600F07AFF74
:107D50000C20DDE700959B68042101930068084A28
:107D600002904B46014800F06DFFE6E780410200BB
:107D70001C420200AC410200F44102008C410200AE
:107D8000D4410200F0B5474680B4041CC08982B0DB
:107D9000161C1F1C0225884204D8281C02B004BCF3
:107DA0009046F0BD226823699046926801332361B2
:107DB000D368A0899E4202D2F419A34206D2114888
:107DC0000421114A00F03EFF0225E6E70918138955
:107DD0008CB2A342F3D94246906907F07BF8424641
:107DE000D36890680133D360089A436800925D6855
:107DF000211C3B1C321CA8474346051C986907F010
:107E00006FF8CAE78C420200203E0200F0B54746F8
:107E100080B4041CC08982B0161C1F1C0225884235
:107E200004D8281C02B004BC9046F0BD22686369E7
:107E30009046926801336361D368A0899E4202D262
:107E4000F419A34206D211480421114A00F0FAFEA7
:107E50000225E6E7091813898CB2A342F3D94246FA
:107E6000906907F037F8424613699068013313614F
:107E7000089A436800929D68211C3B1C321CA8474D
:107E80004346051C986907F02BF8CAE78C420200AC
:107E9000383E020070B5C38902248B4201D8201CF1
:107EA00070BD8369056801338689AA688361891971
:107EB00013898EB2B34206D80B4804210B4A331CF7
:107EC00000F0C0FEEBE7A86907F004F86B69A8684A
:107ED00001336B614368311CDB689847041CA86957
:107EE00006F0FEFFDBE7C0468C420200903D020038
:107EF000F8B5C389051C002B2BD00027AB692E6871
:107F00000133AC89B268AB613C191389A4B2A342B6
:107F100008D8231C10480421104A00F093FE0224C4
:107F2000201CF8BDB06906F0D5FF7369B068013355
:107F300073614368211CDB689847041CB06906F034
:107F4000CFFF0137EB89BFB2BB42E9D9002CD5D0B6
:107F5000E6E70024E4E7C0468C420200903D0200C0
:107F6000F0B50568838983B0A869CE1806F0B2FF22
:107F70002C6AB6B2AE84002C47D0AB68DF68002F05
:107F800002D0BAB2BA420BD935480421354A00F0C2
:107F900059FE0227A86906F0A3FF381C03B0F0BD04
:107FA0001B89B342F0D9A86906F094FFEB68A86872
:107FB00001334268EB600094BBB25468311C00226C
:107FC000A047071CA86906F08BFF002FE2D1012211
:107FD0002623286AEA54AA68D1689446002910D05A
:107FE0000022002401E0002B19D1045D0132FF3C86
:107FF000631E9C4192B2E3B2141E8C42F3D3002B59
:108000000DD100222623EA54C4E7AB680C27D868B8
:1080100006F0C6FD28620028BCD0041CADE762460D
:108020001389B3420BD80E4804210F4A331C00F0C9
:1080300009FE02272623EB5C002BAED0E1E7A869FE
:1080400006F048FF6B69A86801336B614368311C17
:10805000DB689847071CA86906F042FFEAE7C046BC
:108060008C420200203E0200903D0200F0B5046800
:108070002623E25C83B00025002A02D1281C03B02D
:10808000F0BD226AE554002A01D0002903D1A0697D
:1080900006F026FFF2E7A268A58C1389AB4207D849
:1080A0002B1C1F4804211F4A00F0CCFD0225EEE7DF
:1080B000A06906F00FFF6369A0680133636143683C
:1080C000291CDB689847051CA06906F009FF002DF4
:1080D000DDD1A368A68CDD68276A002D02D0AAB284
:1080E000AA4206D90E4804210F4A00F0ABFD022532
:1080F000CDE71B89B342F5D9A06906F0EBFE2369F1
:10810000A0680133426823610097ABB29768311CC5
:108110000022B847051CA06906F0E2FEB7E7C0469A
:108120008C420200903D0200383E0200F0B5474606
:1081300080B40468858982B0A0694D19171C06F0C7
:10814000C9FE266AADB2A584002E33D0A368D968D3
:108150008846002902D08AB242450DD91A48042126
:108160001A4A00F06FFD0226A06906F0B9FE301C25
:1081700002B004BC9046F0BD1B89AB42EED9A069A9
:1081800006F0A8FEE368A06801334268E360414658
:10819000009656688BB20022291CB047061CA069C5
:1081A00006F09EFE002EDFD1226A26233A600122CD
:1081B000E254DCE7A3680C26D86806F0F1FC2062E4
:1081C0000028D1D0061CC1E78C420200203E0200EC
:1081D000F0B556465F464D464446F0B487B003932B
:1081E00010AB1B8882460591161C002B00D1A4E021
:1081F000013B9BB20493002506E0049B9D4233D0D3
:108200005846013500282FD10398B3893468C31824
:10821000AFB2FB189BB2A069984606F05BFE226ADB
:108220004146A1849146002A65D0A368DA68934646
:10823000002A02D092B25A451ED941480421414A2F
:1082400000F000FD02239B46A06906F049FE33685A
:108250002622995C0029D0D000219954986906F013
:108260003FFE049B9D42CBD1584607B03CBC904694
:108270009946A246AB46F0BD1B894345DDD9A069AE
:1082800006F028FEE368A068594601334268E360BF
:108290008BB249460091516800228C464146E04726
:1082A0008346A06906F01CFE5A46002ACCD1012262
:1082B0002623206AE254534605991C68804650469E
:1082C000CF19A368C189BAB20220DF688346914200
:1082D000BDD950464169013141618189002F02D0E9
:1082E000B8B2B84212D9184A1548042100F0AAFCC5
:1082F00002229346ABE7A368D86806F051FC0C2134
:1083000020628B4600289FD081468EE78A181B8901
:1083100092B291469342E6D9A06906F0DBFD23694B
:10832000A06801334268414623610091BBB24946CF
:1083300097680022B847834686E700218B4693E77B
:108340008C420200203E0200383E020008B502487E
:1083500004F046F808BDC0466C3B02000060406077
:10836000C16080607047C046436888604B60436866
:1083700008601960416070474268036880605A6015
:1083800042681360006040607047C046081A43426C
:108390005841C0B27047C04600787047F0B5174DDD
:1083A00047462C6880B4A36882B0DF68061C391C7D
:1083B000F7F792FE2623013FE35C80B23E40804601
:1083C000B6B2002B13D0A28C231C824209D000210C
:1083D000201CFEF7B7FD2868414601AAFEF762FDA2
:1083E0002B681B6A985D02B004BC9046F0BD201C4F
:1083F000414601AAFEF756FD2B68F2E72CE1FF1F6C
:10840000F0B5564644465F464D46F0B48046ABB0A4
:10841000101C0D1C171C8847791C0191061C081C98
:10842000A847BA1C041C0292101CA8472402FB1C7B
:1084300000040443181C9A46A8473443000604432A
:1084400001341AD0391D0391081CA8477A1D0492E3
:10845000061C101CA847BB1D041C0593181CA8472C
:108460002402F91D000404430691081CA847344364
:1084700000062043A44CA0420CD901224046A34947
:1084800003F0C0F800202BB03CBC90469946A246B1
:10849000AB46F0BDF9229200BA180092101CA84712
:1084A0009B4B061CFB180793181CA847994981464B
:1084B00079180891081CA8474A4613020004034390
:1084C0001E43954BFB180993181CA847000606434A
:1084D000A642D2D81AA92AAA894693460C1C761A13
:1084E0003019A847207001345C45F9D148463C2139
:1084F000FDF754FF4B46DB6B984201D00222BDE7EB
:108500003C214846FDF74AFF4946C96B8842F5D1F0
:10851000FDF768FF8021C900C919061C381C834675
:108520002F1C0D1C00E0201C441CB847011C301CF3
:10853000FDF74CFF061CAC42F5D1FDF757FF4B464B
:108540005B6A3D1C03225F46834297D149468E6990
:10855000CC69FDF747FF8346002C14D03B1C301C30
:108560002F1C5D469B4600E0301C461CB847011C92
:10857000281CFDF72BFF013C051C002CF4D15B46A9
:108580003D1C83461F1C5846FDF730FF4A46126AC1
:10859000824201D0042271E7381CA847061C0198CA
:1085A000A847041C0298A84724020004044350462C
:1085B000A847264300060643013612D00398A84771
:1085C000041C0498A847061C0598A8473602000416
:1085D00006430698A8473443060626434A4CA6425B
:1085E0006FD90098A847041C0798A847061C08984C
:1085F000A8473602000406430998A84734430206F8
:1086000022434046454902F0FDFF4B465A6840462A
:10861000434902F0F7FF4B469A684046414902F051
:10862000F1FF4B461A6940463F4902F0EBFF4846CE
:108630000AA904F08DFC0AAA40463C4902F0E2FF78
:1086400048460AA904F06AFC0AAA4046384902F0E2
:10865000D9FF49468A69C96940465318013B3549E3
:1086600002F0D0FF381CA847041C0198A847061C3C
:108670000298A8473602000406435046A8473443F0
:10868000020622432C49404602F0BCFF0398A8474B
:10869000061C0498A847041C0598A8472402000457
:1086A00004430698A8473443020622434046234920
:1086B00002F0A8FF4B461A6A4046214902F0A2FF89
:1086C000E0E60098A847061C0798A8478346089844
:1086D000A84759460B020004034309981E43A847C4
:1086E00000060643A64200D97BE72AAA4C469346D9
:1086F000361B3019A847207001345C45F9D1484633
:108700003C21FDF74BFE6CE7FFFF0F007C440200AD
:10871000E5030000E6030000E703000070430200E9
:108720008C430200A4430200C0430200D84302006D
:10873000F0430200084402002844020044440200BE
:108740006044020010B50549041C02F05BFF201CC8
:1087500003490022FFF754FE10BDC04698440200B2
:108760009983010010B50549041C02F04BFFFC225F
:10877000201C03491202FFF743FE10BDB044020063
:108780009983010038B50E4C051C2368002B12D0CC
:108790000C4902F037FF281C00220B49FFF730FE7E
:1087A000051C20682622825C002A02D00021FEF7E8
:1087B000C9FB281C38BD054902F024FF0025F8E755
:1087C0002CE1FF1FEC4402009D830100CC44020019
:1087D000F0B544465F4656464D46F0B40C1C83B097
:1087E000002800D07BE04B4B4B494C4D9C46F92375
:1087F0009B0007228A460121A94698460192062637
:1088000005270425032002238B46002259460978B8
:108810001B78127809021B040B43134302780020D3
:108820001206134301330DD03A78337812021B0439
:108830001A432B78019D1A432B781B061A43384B99
:108840009A4206D903B03CBC90469946A246AB4634
:10885000F0BD52464D4611782A7809024546120469
:108860000A43297865460A43297809060A439A4249
:10887000E8D8131D011C9C4241410B1C211D8A425A
:10888000404118433FD093073DD11568256051689A
:1088900061609368A360D568E560116921615369DF
:1088A00063619569A561D169E161136A2362556AC3
:1088B0006562916AA162D36AE362156B2563516BAD
:1088C0006163936BA363D26BE263201C3C21FDF7D1
:1088D00065FDE36BC01A43425841C0B2B2E7114A8A
:1088E00011499146114A124B124D8C46124993463A
:1088F000FC229A46A8460191104E114F114D124884
:10890000124B120282E70023995CE1540133402BA1
:10891000FAD1DAE7E7030000E5030000E603000010
:10892000FFFF0F00E6FF0000E7FF000001FC000072
:10893000E5FF0000E4FF000007FC000006FC00006B
:1089400005FC000004FC000003FC000002FC000029
:10895000F0B556465F464D464446F0B40E1C93B003
:1089600000283BD0514B52495248534A9C46534BE6
:108970008846534F5349009091469B46524CFC23E6
:10898000524D5348534A01978A461B02594657464F
:1089900009783F7809023F041B78127839430B436A
:1089A0001206134301330DD02A78237812021B04D8
:1089B0001A43037801981A4303781B061A43464B5F
:1089C0009A4220D9301C4549042209F012FE13B006
:1089D0003CBC90469946A246AB46F0BD404FF923B9
:1089E00040489B004049072200979C4601270223EC
:1089F000804601929A4689460624052504200322D2
:108A0000BB460023C2E74A46474611783A78090236
:108A1000120460460A43009F01780A433978090628
:108A20000A439A42CED80023111D181C02AD8D4274
:108A30005841011C03A882425B410B432DD0910792
:108A40002BD1136857689068D16802930397136914
:108A500057690490906905910693D169136A079745
:108A60000890576A906A09910A93D16A136B0B9721
:108A70000C90576B906BD26B0D910E930F971090DB
:108A800011923C21281CFDF789FCE96B884299D1A1
:108A9000281C311C04F05CFA99E712A92B1C5C1B02
:108AA000A45C1C7001338B42F9D1EAE7E4FF0000BB
:108AB000E6FF0000E7FF0000E5FF000001FC00000A
:108AC00007FC000002FC000006FC000005FC0000A2
:108AD00004FC000003FC0000FFFF0F00084502003B
:108AE000E7030000E6030000E503000008B5044BBF
:108AF0001860044B0448196003F072FC08BDC046BE
:108B000030E1FF1F2CE1FF1F20430200F0B5474674
:108B100080B40F4F8846FC680837381C211CFFF7CB
:108B200035FC061E10D1E5686B69002B05D028695D
:108B300041469847002800D06E616468381C211CAB
:108B4000FFF724FC061EEED004BC9046F0BDC046E4
:108B500034E1FF1F10B5074C052300222370201DB0
:108B60003023E25406F0A8F9201C08300021FFF75A
:108B7000F5FB10BD34E1FF1F014B18707047C04674
:108B800034E1FF1F014B00201856704734E1FF1FEE
:108B9000F8B5144C071C60680E1C06F09BF93023D6
:108BA000E25C002A18D10122251CE2541835291C48
:108BB000281C6F612E61FFF7D1FB606806F08AF90F
:108BC000201C0830291CFFF7CFFB606806F088F9ED
:108BD000606806F085F9F8BD182005F0E1FF051E74
:108BE000F6D0E4E734E1FF1F38B5041E0ED0211C97
:108BF000FFF7B4FB064D686806F06CF9281C0830D6
:108C0000211CFFF7B1FB686806F06AF938BDC04661
:108C100034E1FF1F38B50A4C051C606806F05AF9AC
:108C2000002D04D0231CAA6808339A4203D0606840
:108C300006F056F938BD281CFFF79EFBF7E7C04643
:108C400034E1FF1F0CB4F0B5474680B4364F002224
:108C5000BA5682B0051C0C1C8A4206DA02B004BC6B
:108C60009046F0BC08BC02B01847786806F032F9AC
:108C70002E4A09AB1360904605F0AAFF2C4E303403
:108C8000031C0094301C00212A4AFDF731FB00230D
:108C9000EB56002B40D142461368301C0021089A45
:108CA000FCF72EFF0823FC68DB1998464046211C80
:108CB000FFF76CFB061E10D1E5686B69002B05D031
:108CC00028690D219847002800D06E6164684046ED
:108CD000211CFFF75BFB061EEED00822FC68D219B0
:108CE00090464046211CFFF751FB061E10D1E56857
:108CF0006B69002B05D028690A219847002800D00D
:108D00006E6164684046211CFFF740FB061EEED0F2
:108D1000786806F0E5F8A1E7301C0021064A2B1C14
:108D2000FDF7E6FAB7E7C04634E1FF1F68E1FF1F31
:108D30000D8B0100F8450200044602007047C04652
:108D400038B50C1C4443002C0AD0201C05F028FF29
:108D5000051E03D00021221C09F06DFC281C38BD23
:108D60000025FBE710B50488118800238C4201D050
:108D7000181C10BD911C0230FF2209F03AFC01239F
:108D8000F6E7C046F0B54F464646C0B41B4B1C4EF6
:108D90001A6885B001321A600B880722DC08DD0AE8
:108DA000E4B21A400121AF00A1469140BC59CAB2B9
:108DB0009046002C09D04C4423784246134323703C
:108DC00005B00CBC90469946F0BD802149000120B9
:108DD000FFF7B6FF0B4A0C491378B8510133DBB2E9
:108DE0001370EA0200925218041C01920293074881
:108DF0000521074A2B1CFFF725FFDCE710E4FF1FC6
:108E00006CE1FF1FECE1FF1FFF0700000C460200B2
:108E10001446020038B50A4B0A4C19600023812120
:108E200023604900084A094BFDF7A2FB2368051C93
:108E300005210748074AFFF705FF281C38BDC04633
:108E400004E2FF1F10E4FF1F858D0100F0E1FF1F0A
:108E50000C46020038460200F0B5041C85B00E1E18
:108E600001D000230B70E308D8B20723234001226E
:108E70009A40D1B2174BE20A9200D358002B1ED071
:108E80001B5C16250B4202D1281C05B0F0BD124F09
:108E9000124803A93A1C124B3C80FDF7E7FA051E65
:108EA0000FD1002E03D0B91C301C09F0CCFB00966A
:108EB0000C4806210C4A231CFFF7C4FEE4E71625E4
:108EC000E2E7009004210748084A231CFFF7BAFE96
:108ED000DAE7C0466CE1FF1F0CE3FF1FF0E1FF1F64
:108EE000658D01000C4602006846020050460200F3
:108EF000F0B55F464D4644465646F0B4C308DBB273
:108F000099460723034001229A408BB00D1C9346DB
:108F1000D1B2704FC20A06929200BB58041C059150
:108F20009046002B04D00A1C49465B5C13421DD1BD
:108F3000694B9A46002D08D0281C09F08CFB83B29F
:108F4000FD2B3AD8002B00D07CE00026504600953F
:108F500001960621614A231CFFF774FE301C0BB0FA
:108F60003CBC90469946A246AB46F0BD5C4A09A976
:108F700010805C4B5C48FDF779FA061E58D1564AC2
:108F8000099B101C00930621231C9246574AFFF7A9
:108F900059FE09995448FDF77BFC41467958061C57
:108FA000079100297AD0079A5946131C4B441A7826
:108FB0008A431A70002EC9D1BCE70004000C00904F
:108FC0004B4A50460421231CFFF73CFEFE22079229
:108FD00093464346FE58002E45D04A46B3181A78A9
:108FE00005993F4F0A431A70291C5A46B81C09F0CC
:108FF00000FB079A09A9BB1800229A703A4B3C80E3
:10900000181C9846FDF774FC061E1C2E1FD0002E5F
:109010009CD1099950460091364A0621231CFFF73E
:1090200011FE404609993A1CFDF792FB061C8DE79C
:10903000294900908A46081C2F4A0421231CFFF767
:1090400001FE83E70004000C83460790C1E7404619
:10905000FDF7D0FC061E00D078E7404609A9FDF7D1
:1090600047FC061CD3E7802149000120FFF768FE7A
:10907000224A41461378785001330699DBB21370C7
:10908000CA021F4900925218061C019202935046D0
:1090900005211C4A069BFFF7D5FD9EE7802149006C
:1090A0000120FFF74DFE4246B850144A0699137846
:1090B00007900133DBB21370CA02114900925218B3
:1090C00001920293504605210E4A069BFFF7BAFD16
:1090D00069E7C0466CE1FF1F0C460200A44602008F
:1090E00008E2FF1F658D0100F0E1FF1FBC46020092
:1090F000784602009046020050460200ECE1FF1F55
:10910000FF0700001446020000B5064B83B01A6842
:10911000054B00211868D38900930023FFF758F806
:1091200003B000BDF0E1FF1F04E2FF1F00B5064BD6
:1091300083B01A68054B00211868D3890093002377
:10914000FFF746F803B000BD04E2FF1FF0E1FF1F88
:1091500008B5024B1868FEF7CBFE08BDF0E1FF1F13
:10916000F0B52D4A2D4B5F4656464D464446F0B469
:1091700013602B4B92469B465A4600231360294BA3
:1091800085B01868284B1968FFF744FE0390002843
:1091900007D0039805B03CBC90469946A246AB4622
:1091A000F0BD224B22481A68052190464346214AC9
:1091B000FFF748FD4346002BEBD01F4A002791469E
:1091C0004B4652461E681268964201D253461E60B4
:1091D0005A461268964201D95B461E60164D00241D
:1091E00003E001340C35444510D0A742F9D02A6879
:1091F0009642F6D1019400970D4804210F4A331C82
:109200000134FFF71FFD0C354445EED10C23013727
:1092100099444745D4D1BCE72CE5FF1FFFFF000070
:109220001CE4FF1F18E4FF1F28E5FF1FC8310200E0
:10923000E0460200EC460200CC3102000447020086
:1092400038B50949041C02F0DDF9084D286805F01D
:1092500041FEFFF759FF286805F042FE201C044933
:1092600002F0D0F9002038BD2847020014E4FF1FA7
:109270004447020038B50A49041C02F0C3F9094DFD
:10928000286805F027FEFFF751FFFFF769FF286800
:1092900005F026FE201C044902F0B4F9002038BD78
:1092A0006047020014E4FF1F7C47020038B50A49FA
:1092B000041C02F0A7F9094D286805F00BFEFFF722
:1092C00047FFFFF74DFF286805F00AFE201C044900
:1092D00002F098F9002038BD9847020014E4FF1FFF
:1092E000B4470200F0B5474680B4684F041C3868A4
:1092F0000E1C05F0EFFD664B1D68002D00D1B3E09C
:10930000644900220B1C1868844208D001320C33D7
:10931000AA42F8D1604B00221A60002450E05300AA
:109320009B189B005C4DCB18002232702B601B7980
:1093300003221340022B66D0584B9C4200D180E0A0
:1093400025D8574B9C4200D18BE04DD9554B9C42C0
:1093500047D0554B9C4264D0544B9C425ED0A0B247
:10936000311CFFF779FD8046301C09F074F9434643
:10937000041C002B01D1002C22D12B68301C9968D1
:1093800009F061F9301C09F066F9041C18E0484B3B
:109390009C4240D01BD9474B9C425FD0464AA31801
:1093A0000F2BDCD8201C5038C0B208F00BFF021C79
:1093B000301C424904F012F8301C09F04CF9041C2E
:1093C000386805F08DFD201C04BC9046F0BD3C487B
:1093D00023180F2BC3D8201C7038C0B2FAF7E8FE50
:1093E000E5E7384B1A68E3E7374AA318FF2BB6D8EE
:1093F000201C311C09F080F8422839D0301C09F0BB
:109400002AF9041CDCE7231C30480421304AFFF70A
:1094100019FC0024D4E7FAF7F3F9C8E706F0C2F81C
:10942000C5E72C4C0120211CFFF7D2F900280FD0F2
:10943000201C311C03F08CFD301C09F00CF9041CBD
:10944000BEE7244C0020211CFFF7C2F90028EFD111
:10945000301C2149042209F0CCF8CFE7FAF7FEF9D5
:10946000A5E7FAF7F1FEA2E70B4B00241D60A7E782
:10947000A0B2311CFFF7F0FC8046301C09F0EBF87D
:10948000041C4046002800D175E776E714E4FF1F6E
:10949000C8310200CC31020024E5FF1F02F10000B8
:1094A00081B00000FDF0000001F10000B2B000004A
:1094B00001F9000002F90000B004FFFF902D020046
:1094C0009008FFFF20E4FF1F0080FFFFE04602003E
:1094D0000848020030E5FF1F08450200F0B54D4680
:1094E0005F4656464446F0B4814683B098680021F2
:1094F00003F08AFF3F4B051C1B680193002B0AD029
:109500003D4C0022231C19688D420BD00199013279
:109510000C338A42F7D1484638492A1C02F072F8C7
:10952000002724E053009A189200A41823790322FC
:109530001340022B57D0324A1068924605F0CAFCFD
:10954000304E281C311CFFF7CDFE331C83462E49BC
:1095500048462A1C02F056F86379071C032B02D0F8
:109560005A46002A0BD15146086805F0B9FC381C50
:1095700003B03CBC90469946A246AB46F0BD484677
:10958000224902F03FF800256379012B08D0002B17
:1095900026D0022B16D048461D4902F033F8E2E7E8
:1095A000042290467019414603F02EFF0090002DD2
:1095B00011D148461749009A454402F023F8AB45BB
:1095C000E2D8E8E7082398467019414603F01CFFEB
:1095D0000090002DEDD048460F4902F013F8E8E75F
:1095E00002218846DEE748460C492A1C02F00AF8A8
:1095F0000027BCE7C8310200CC3102002848020035
:1096000014E4FF1F24E4FF1F7448020068480200AE
:10961000304A0200443B0200704802004848020001
:10962000F0B55F4656464D464446F0B4814689B093
:10963000784901F0E7FF484602F0F2F9764B7749A6
:109640001B68774F002407938B464E4607995B466D
:109650000022002907D019688C420BD007990132EB
:109660000C338A42F7D1802301345B029C42EDD156
:10967000002649E05500AD18AD005D44386805F09E
:1096800029FC03222B79111C194090468A46022995
:1096900044D1644B77229946494600230B702D2311
:1096A000202106929A46059120230699059A009159
:1096B00001920293301C53465B49221C01F0A2FF29
:1096C0006B798046032B27D8584A9B009A58E97932
:1096D000AB79301C0091564901F094FF55494A4638
:1096E000301C01F08FFF386805F0FAFB301C02F0E7
:1096F0009DF9013480235B029C4204D04346002B39
:1097000001D10028A2D14646301C09B03CBC90468D
:109710009946A246AB46F0BD474AD8E7414A201CCD
:10972000111C9146FFF7DEFD2B7941461940524648
:109730008846012A4FD12D237221202206938A4682
:1097400005924246022AAFD05B46002219688C423D
:1097500006D0079901320C338A42F7D16523A4E77A
:1097600053009A1892009046D84441464B79012BF9
:1097700017D0002B18D0022B2AD0032B17D101228F
:109780000492284808F067FF41468B79049A5343B6
:109790009842E3D34146CB7953438342DED37623C9
:1097A00083E704230493ECE702220492E9E704210F
:1097B000224A2348FFF746FA1A4808F04CFF0023D4
:1097C000049341461A1CCB7953438342C6D3E6E740
:1097D00008210491D5E75246002A13D11148A968FF
:1097E000F9F714FF002806D0772372216D22069323
:1097F0008A460592A5E7772272232D2106929A4682
:1098000005919EE777227223202106929A460591C0
:1098100097E7C04688480200C8310200CC310200F8
:1098200014E4FF1F24E4FF1FC4480200D0460200D6
:10983000D84802006451020080480200B448020087
:10984000E0460200F0B556464D4644465F46F0B449
:109850002A4BC3B01C68804602F0E2F8284E294922
:10986000221C3368404601F0CDFE274B00221968C8
:10987000264B274D8B4691469A4659462B1C002273
:1098800000290FD019688C4204D001320C335A459C
:10989000F8D107E053009A189200AF183B790B22D9
:1098A0001A420BD032680134A242E6D2002043B003
:1098B0003CBC90469946A246AB46F0BD201C02A98E
:1098C000FFF710FD0028EDD0B96802A8F9F79EFE59
:1098D0000028E7D0012202AB9144514600934A464A
:1098E000231C404601F08EFE404602F09FF831688E
:1098F00001348C42DAD80028BFD1D7E72CE5FF1F0E
:109900001CE4FF1FE8480200C8310200FC480200C6
:10991000CC310200F8B50C4C051C20680E1C05F07B
:10992000D9FA0A4F281C391CFFF7DCFC0025B0428D
:1099300004D3B819082103F067FD051C206805F061
:10994000CFFA281CF8BDC04614E4FF1F24E4FF1F13
:1099500038B5074C051C206805F0BCFA0549281CE1
:10996000FFF7C0FC051C206805F0BAFA281C38BDBA
:1099700014E4FF1F24E4FF1F70B50B4C051C206886
:1099800005F0A8FA094E281C311CFFF7ABFC002596
:10999000002804D0301C002103F036FD051C20688F
:1099A00005F09EFA281C70BD14E4FF1F24E4FF1F7D
:1099B000F0B54E4657464546E0B4674B82B01B684B
:1099C000041C0E1C0193002B0AD0644900250B1CBB
:1099D0001868844206D0019801350C338542F7D1CE
:1099E000022556E06B005D19AD004D192B7903255A
:1099F0002B40012B54D05A4B9C4200D18AE039D9DC
:109A0000584B9C4200D19FE054D8574B9C4200D108
:109A100095E0564B9C4200D06FE0554A00241068F8
:109A2000914605F057FAFCF7DDFC524F824638604C
:109A3000514DA0460FE042462A703019042103F030
:109A4000E3FC291CFFF74EFC3868291CFCF7E4FCFA
:109A5000043438608246301C08F0FDFD8442EAD3AD
:109A60005046FCF7C3FC4B463860186805F038FADE
:109A700000250EE0414B9C422CD033D8404AA3181D
:109A8000FF2B3AD8201C311C08F04AFD051E422D40
:109A900033D0281C02B01CBC90469946A246F0BDAB
:109AA000002AA8D137480421374A231CFFF7CAF8F7
:109AB0000225EEE7354823180F2B1ED80021301C55
:109AC00003F0A2FC011C201C7038C0B2FAF776FB30
:109AD0000025DEE70021301C03F096FCFAF7ACFB12
:109AE0000025D6E72A4B9C4207D10021301C03F009
:109AF0008BFC05F07DFD0025CBE71D4F386805F098
:109B0000E9F9A0B2311CFFF7F3F9051C386805F03C
:109B1000E7F9BEE70221301C03F076FC0221051CA8
:109B2000B01C03F071FC0021041C301D03F06CFC20
:109B3000211C021C281CF9F7B5FE0025A9E7301CE2
:109B400003F0E0FC0025A4E70221301C03F05CFCDC
:109B500005F0D2F900259CE7C8310200CC310200A3
:109B600031F00000FFF00000F8F00000FDF0000010
:109B700014E4FF1F20E4FF1F24E4FF1F81B0000056
:109B80000080FFFFE04602000C4902009008FFFF42
:109B9000B2B0000070B5002182B0061C986803F0D6
:109BA00033FC1A4B041C1B680193002B0AD0184D80
:109BB00000222B1C19688C420AD0019901320C3307
:109BC0008A42F7D1301C1349221C01F01BFD13E01F
:109BD00053009A189200AD182B7903221340012BE1
:109BE0000DD0A9680022201CFFF7E2FEAB68301CF4
:109BF0000949221C01F006FD002002B070BD301C96
:109C00000649221C01F0FEFCF6E7C046C8310200FE
:109C1000CC310200284802004449020028490200D1
:109C2000F0B546464F46C0B4804683B098680021E0
:109C30001D1C03F0E9FB514B041C1B680193002B16
:109C40000BD04F4E0021301C321C13689C4210D0A8
:109C5000019B01310C329942F7D140464949221CFF
:109C600001F0D0FC0025281C03B00CBC904699469E
:109C7000F0BD4F007F18BF00F7193B7903221A404F
:109C8000012A74D0EB68051C994600232A68944287
:109C900005D0019A01330C359342F7D146E05A00C2
:109CA000D3189B00F6187379012B37D0002B5CD0AA
:109CB000022B58D0032B48D1484608F0CCFCB3798E
:109CC00001256B43984231D3F3795D4385422DD30F
:109CD0003B7903221340022B11D02B4D286805F04D
:109CE000F9F82A4E201C311CFFF7FCFA404628499F
:109CF000221C331C01F086FC286805F0F1F8201CBA
:109D000049460022FFF754FE051C4046002D15D1A0
:109D10002049221C4B4601F075FCA4E70425484667
:109D200008F099FCB3796B439842CDD240461A496A
:109D30004A46231C01F066FC051C94E72A1C1749BF
:109D4000231C01F05FFC051C8DE715480421154A12
:109D5000FEF778FF484608F07EFCF37900255D4366
:109D60008542E3D3B4E70825D9E70225D7E7404683
:109D70000D49221C01F046FC002574E7C8310200A1
:109D8000CC3102002848020014E4FF1F24E4FF1F26
:109D900098490200DC49020068490200BC490200FF
:109DA000E0460200B44802002849020008B500223B
:109DB000FFF7FEFD08BDC04610B584B0041C0A1CA8
:109DC00001A8054903F00AFB201C01A90022FFF7A6
:109DD000EFFD04B010BDC046902D020008B5084B41
:109DE00000221860074B08481960084B1A6002F0FF
:109DF000F7FA074805F060F8FFF7B2F908BDC0466A
:109E000018E4FF1F28E5FF1FFC4B020020E4FF1FA2
:109E100014E4FF1FF8B5C327041CBF00E3590E1C50
:109E2000984702280AD0182503E0013DADB2002D65
:109E300035D0201CE35998470228F6D1C327BF002C
:109E4000201CE3599847002829DB3070E359201C77
:109E50009847002823DB7070E359201C984700289E
:109E60001DDBB0700025201CE3599847002819DB42
:109E70007319D870B17801358D42F4D90331301C93
:109E8000FCF7E6FAB378F318DB7883420FD1337826
:109E900022789A4201D0FF2B0CD10020F8BD01207E
:109EA0004042FBE7B178301C0331FCF7D1FA0320C4
:109EB0004042F3E704204042F0E7C046F0B54F4689
:109EC0004646C0B48F78051C033783B0081C0E1CAF
:109ED000391CFCF7BDFAC4239B0081469846281C18
:109EE000EB580221984700244346315DEB58281C6B
:109EF00001349847BC42F7D1C4239B00EB58281C7F
:109F00004946984703B00CBC90469946F0BDC04600
:109F100008B5C6239B00C05801F092F808BDC046A2
:109F200008B5C6239B00C05849B201F06DF808BDC2
:109F300000B5C62385B09B00C05803AB009302A9AF
:109F40000122642305F0FEFB002806D1039B012BB0
:109F500003D16B46187A05B000BD01204042FAE7F4
:109F6000F0B54F464646C0B4C5B000236A46041C4F
:109F70001374602939D0612905D0012045B00CBC8B
:109F800090469946F0BD624A815C0079814200D3D7
:109F90008CE065186D794B1CDBB2A3542D029842FE
:109FA00000D8AFE0E3185B790231C9B22B43A1546A
:109FB0009846884200D8A7E06B466E4611331036AB
:109FC000FF361D1C944601E01D1C111C4A1C611823
:109FD0004F79D2B261466254591E0F70904202D935
:109FE0000133B342F0D1404662E0494A0179835CD3
:109FF00000208B420CD2E01840795D1CEDB2A554D4
:10A000000002A94204D9651969790233A3540843AF
:10A0100004A9FFF767F9002870D004A808F01BFB1B
:10A02000C0B200286AD00826FF36A25D002304A92A
:10A03000CD5CFF2A07D0511CA2180432C9B2FF32EE
:10A040005571A1550A1C0133D9B28842EFD8CD23EE
:10A050009B00E158A61DD71C0131FF36E150301C92
:10A06000391CFCF7F5F9C4239B008146E258201CFB
:10A0700002219846904700254246715DA258201C57
:10A0800001359047BD42F7D1C4239B00E358201C03
:10A090004946984782239B00E0180823FF33E25C7F
:10A0A000311C033208F0A5FA002067E7002004AD58
:10A0B00000232B7004A9FFF779FECD239B00E25803
:10A0C000A61D0132E2500823FF33E75CFF36033759
:10A0D000391C301CFCF7BCF9C4239B008146E258B4
:10A0E000201C02219846904700254246715DA258E7
:10A0F000201C01359047BD42F7D1C5E70823FF3347
:10A10000E25CA4E7281CD2E7181C04ADD0E7C046E7
:10A110000B030000F8B5161CCE220F1C9200002184
:10A12000041C1D1C08F087FAC3239B00E750C423BE
:10A130009B00E65040236370CC2300229B002570D7
:10A14000E254C9239B00E018002103F035F8F8BD64
:10A1500010B5811C041CFFF75DFE00281FD1E378B9
:10A16000990736D42279002A36D05AB2002A17DB52
:10A170006079A1780622FF32A1540222134362784B
:10A1800040210A40134383225200A354144A01235E
:10A19000A35484225200A0540822FF32A35410BDBD
:10A1A000104AA25C5A40D107E2D40F4A6079A25CFF
:10A1B0008242DED182229200A118201CFFF77EFE8F
:10A1C0000A48637904210A4AFEF73CFD0C2040420C
:10A1D000E5E70A204042E2E70B204042DFE7C046C5
:10A1E0000B030000090200000B020000F84C020003
:10A1F000184D0200024B0279C35CD01AC0B27047FE
:10A200000B03000010B506490479425C031C0020D2
:10A21000944203D99818013240795A5410BDC0466F
:10A220000B03000070B516490479425C031C002042
:10A23000A2421FD298184079551CEDB25D5400021D
:10A24000AC4218D95D196D79961CF6B228435E545C
:10A250000004B4420ED99E197679D51CEDB25D5436
:10A260003602AC4209D95D196C7904325A54231C68
:10A270003343184370BD0004FCE73043FAE7C0469F
:10A280000B0300000822FF32835C10B5FF2B05D0C2
:10A29000C4180434FF3401336171835410BDC046C7
:10A2A0000822FF32835C70B5FF2B10D0C5185C1CF0
:10A2B00004350E0AE4B2FF356E71C9B28454FF2C26
:10A2C00005D004190434FF3402336171835470BD26
:10A2D0000822FF32835CF0B5FF2B26D0C6180D0C88
:10A2E0005C1C0436FF36E4B22F0A77718454EEB258
:10A2F000FF2C1AD0041904349D1CFF346671EDB292
:10A300008EB28554360AFF2D0FD04519DC1C04355A
:10A31000E4B2FF356E71C9B28454FF2C05D0041924
:10A320000434FF34043361718354F0BDCD239B00AA
:10A33000C0587047F0B5CD234F4646469B00C0B489
:10A34000C258861D0132C2500823FF33C75CFF3656
:10A350000337051C83B0391C301CFCF779F8C42383
:10A360009B008146EA58281C022198469047002409
:10A370004246315DAA58281C01349047BC42F7D1AF
:10A38000C4239B00EB58281C4946984782239B0016
:10A39000E8180823FF33EA5C311C033208F029F97E
:10A3A00003B00CBC90469946F0BDC046F0B54E4691
:10A3B00045465746E0B4CB230E1C9B00C921C55827
:10A3C0008900A8B0041C401802F0FEFE002D0ED03B
:10A3D000201C311C6A689047002805D128B01CBC9D
:10A3E00090469946A246F0BD2D68002DF0D1112E61
:10A3F00000D9AEE2CE4AB300D3589F4618AB984678
:10A40000181C0A2105F0A2FA404608F024F9082396
:10A41000FF33C0B2E55C002200280FD041468F5CBC
:10A42000FF2D07D06E1C65190435F6B2FF356F712C
:10A43000E654351C0132D6B2B042EFD8CD239B0092
:10A44000E258A61D0132EF1CFF36E250391C301CC9
:10A45000FBF7FEFFC4239B008146E258201C02212B
:10A460009846904700254246715DA258201C013550
:10A470009047BD42F7D1C4239B00E358201C4946B6
:10A48000984782239B00E0180823FF33E25C311CCD
:10A49000033208F0AEF80020A0E7CD239B00E2587D
:10A4A000A61D0132E2500823FF33E75CFF36033775
:10A4B000391C301CFBF7CCFFC4239B008146984617
:10A4C000201CE3580221984700254246715DA2589E
:10A4D000201C01359047BD42F7D1C4239B00201CAE
:10A4E0004946E3589847822189006018CCE7637891
:10A4F0004022934308226370FF32A35CFF2B00D1FC
:10A500006EE2E1180431FF31581C00254D71C0B2D4
:10A51000C721A0548900665CFF2800D160E22018A2
:10A52000991C0430C9B2FF304671FF27A154FF299E
:10A5300006D06118DF1C0431FFB2FF314D71A75402
:10A54000CD239B00E258A61D0132FF360337E250AF
:10A55000391C301CFBF77CFFC4239B0081469846C6
:10A56000201CE3580221984700254246715DA258FD
:10A57000201C01359047BD42F7D1AEE7CD239B00AB
:10A58000E258A61D0132E2500823FF33E75CFF3694
:10A590000337391C301CFBF75BFFC4239B0081464B
:10A5A0009846201CE3580221984700254246715DD9
:10A5B000A258201C01359047BD42F7D1C4239B000F
:10A5C000E358201C494698470823FF33E25C822168
:10A5D000890003326018311C08F00BF80A2004F0DF
:10A5E000F3FA002004F080FC0020F7E6CD239B0066
:10A5F000E258A61D0132E2500823FF33E75CFF3624
:10A600000337391C301CFBF723FFC4239B00814612
:10A610009846201CE3580221984700254246715D68
:10A62000A258201C01359047AF42F7D1C4239B00AC
:10A63000E358201C494698470823FF33E25C8221F7
:10A64000890060180332311C07F0D3FF0A2004F0A0
:10A65000BBFAC7239B00E35C012B00D01BE7012062
:10A6600004F042FC0020B9E632480521324AFEF7E8
:10A67000E9FACD239B00E258A61D0132E2500823DF
:10A68000FF33E75CFF360337391C301CFBF7E0FE75
:10A69000C4239B0081469846201CE358022198471A
:10A6A00000254246715DA258201C01359047BD42ED
:10A6B000F7D1C4239B00E358201C49469847082340
:10A6C000FF33E25C8221890003326018311C07F0FD
:10A6D00090FFC82300229B00E250184A2179A35C16
:10A6E00000208B421FD2E01840795D1CEDB2A554CA
:10A6F0000002A94200D875E165196D799E1CF6B279
:10A700002843A6540004B1420DD9A6197679DD1C60
:10A71000EDB2A5543602A94204D96519697904330A
:10A72000A3540E43304302F091FD002056E6C0468C
:10A73000B04C0200F84C0200584D02000B03000020
:10A74000A9482379225C00219A420CD2A1184979A8
:10A75000551CEDB225540902AB4204D965196D7937
:10A76000023222542943C8229200A2588918CC22CE
:10A770009200A25C8946002A00D0FFE0033B211C26
:10A780009AB24846083102F0ADFDCC239B00E35C51
:10A79000002B00D07FE6CD239B00E258A61D01329E
:10A7A000E2500823FF33E75CFF360337391C301CC7
:10A7B000FBF74EFEC4239B0081469846201CE358BD
:10A7C0000221984700254246715DA258201C0135A0
:10A7D0009047AF42F7D180E683492079635C00223D
:10A7E00083420DD2E21852795D1CEDB2655412021B
:10A7F000A84204D9651968790233635402431201EF
:10A80000C8239B00E250CD239B00E258A61D0132D5
:10A81000E2500823FF33E75CFF360337391C301C56
:10A82000FBF716FEC4239B0081469846201CE35884
:10A830000221984700254246715DA258201C01352F
:10A840009047BD42F7D148E60521684A6848FEF7BF
:10A85000F9F90120404202F035FDCD239B00E2587A
:10A86000A61D0132E2500823FF33E75CFF360337B1
:10A87000391C301CFBF7ECFDC4239B008146984635
:10A88000201CE3580221984700254246715DA258DA
:10A89000201C01359047BD42F7D1C4239B00E358EB
:10A8A000201C494698470823FF33E25C8221890037
:10A8B00060180332311C07F09CFE02F0F5FC00200A
:10A8C0008CE518AB181C00214022984607F0B3FE17
:10A8D000454A2179A35C994248D9E1184879013366
:10A8E000A354002842D008264146FF3602F0D4FC8B
:10A8F000A25D434628AD1878FF2A07D0511CA21844
:10A900000432C9B2FF325071A1550A1C0133AB4267
:10A91000F1D1CD239B00E158A61DD71C0131FF3694
:10A92000E150301C391CFBF793FDC4239B00E15818
:10A9300081460391201C0221039A984690470025E6
:10A940004246715DA258201C01359047BD42F7D1A7
:10A9500091E523792648013B0093A37904210193D3
:10A96000244A331CFEF76EF9012037E5C7239B000C
:10A97000E05C013843425841C0B2B4E7CD239B00AC
:10A98000E258A61D0132E2500823FF33E75CFF3690
:10A990000337391C301CFBF75BFDC4239B00824648
:10A9A0009846201CE3580221984700254246715DD5
:10A9B000A258201C01359047BD42F7D1C4239B000B
:10A9C000E358201C514698470823FF33E25C82215C
:10A9D000890060180332311C07F00BFE2379CDE6A5
:10A9E000FF27ADE500049EE60B030000684D020062
:10A9F000F84C02002C4D0200F8B54D4644465F4627
:10AA00005646F0B43149C7239B00C35C041C8946F9
:10AA1000081C2F4A0521FEF715F9C5239B00E358B2
:10AA2000002B01D0201C984782239B001B199B46BA
:10AA30002849294BA61C8A46022798460125311C25
:10AA4000201CFFF7E7F9011E27D1E3781F42F6D15A
:10AA50002279002AF3D05AB2002A21DB6179A0784A
:10AA60000622FF32A05462784020024002200243B6
:10AA7000134383225200A354184BE55484235B00F4
:10AA8000E1540823FF33E554201CFFF78FFC311CF1
:10AA9000201CFFF7BFF9011ED7D00028CFDBF3E75A
:10AAA0004146625C5A401542D8D10D4A6179A25C98
:10AAB0008A42D4D1201C5946FFF700FA63794846F0
:10AAC00004215246FEF7BEF8B9E7C046F84C020032
:10AAD000784D0200184D0200090200000B0300002F
:10AAE0000B02000070B5141C051C101CCE220E1C9D
:10AAF0009200002107F09FFD0E4AC3239B00E25005
:10AB00000D4AC4239B00E2500C4AC5239B00E2502F
:10AB100040236370CC2300229B002670E254C9239B
:10AB20009B00E018002102F047FBC6239B00E55084
:10AB300070BDC046319F0100219F0100119F01009F
:10AB400038B5041C08200D1C04F02AF8002807D092
:10AB5000CB229200A35845600360A050002038BD6E
:10AB60000C20FCE710B5041C082004F019F800289C
:10AB700008D0054A4260CB229200A3580360A0503F
:10AB8000002010BD0C20FCE7619F010038B504F0E7
:10AB9000F5F9037E041C002B0DD1827D012A11D012
:10ABA000002A0CD0022A10D08375FA21890060682F
:10ABB00004F0C4F938BD0023037683758382A58928
:10ABC000002D0CD1E589002D20D1A38A228A0133E2
:10ABD0009BB2A3829A420AD9A589002DE5D0A36829
:10ABE0002068012198470123A375291CDFE7002372
:10ABF000A375A382E37D002B10D0658A002DF4D1CC
:10AC0000A589002DEBD1E589002DCED00021A368C8
:10AC1000206898470223A375291CC8E7A368206809
:10AC20000021984700236376C4E7C04670B5041C32
:10AC300082B00E1C151C00211C2207F0FCFC231CFA
:10AC4000064AA66020C30193009201210022231C22
:10AC5000034804F055F902B070BDC0468DAB010049
:10AC6000C04D0200F8B54F464646C0B41F1C08ABA5
:10AC700089461E8809AB041C90461D7804F014F91F
:10AC80004B46A3814346E381012327826682E57513
:10AC90002376637604F00CF96068012104F04EF924
:10ACA0000CBC90469946F8BD0023C1604360036028
:10ACB00082607047F0B5474680B4051C8846141E74
:10ACC000012C31D08268016846685318013B9B1BF8
:10ACD0009A4200D89B1A9C4221D8971BA74217D8AA
:10ACE000EB68414698193A1C07F083FCA74205D24D
:10ACF0004046C119E21BE86807F07BFCAB68A61967
:10AD00009E4200D3F61A6E60201C04BC9046F0BD33
:10AD1000E968221C8819414607F06BFCEEE71C1C11
:10AD2000971BA742F4D8DBE742688068531C834234
:10AD300089410B402968994205D040460178E8686E
:10AD400081546B60E0E70024DEE7C046F0B547467B
:10AD500080B4051C8846141E012C30D082684168DE
:10AD6000066853189B1B9A4200D89B1A9C421ED817
:10AD7000971BEA6840469119A74214D83A1C07F07D
:10AD800038FCA74205D24346D819E21BE96807F010
:10AD900030FCAB68A6199E4200D3F61A2E60201C28
:10ADA00004BC9046F0BD221C07F023FCF1E7971B82
:10ADB000EA681C1C91194046A742F4D8DEE70368F4
:10ADC00041688B420CD05A1C0260C2684146D35C79
:10ADD0000B70026883689A42E1D300230360DEE7C8
:10ADE0000024DCE7F8B54F464646C0B40C1C2F499A
:10ADF000051CF5F7B5F9281C89462C49F5F76CF9BF
:10AE0000FA252B4AAD008618281C70432949C838FA
:10AE1000F5F762F986198008361A281C704326490E
:10AE2000C838F5F759F9071C2348291C7843F5F76A
:10AE300053F9361A6E43214BB046181C2049404442
:10AE4000F5F74AF9E121061C09014846F5F744F9EE
:10AE5000E121207109014846F5F782F98946081C6D
:10AE60003C21F5F739F93C2160714846F5F778F94E
:10AE70001348FA2270435200131C4344A171181A5C
:10AE8000291CF5F729F9E070092E09D80336A670B8
:10AE9000BFB20023278023810CBC90469946F8BDA1
:10AEA000093E0137A670BFB2F3E7C04680510100EA
:10AEB0006DFA0A00DA502D02C29205000CFEFFFF67
:10AEC0008877000000000000F0B55F4656464D460A
:10AED0004446F0B48BB08046099104F0A1FB414B8D
:10AEE0003F4A041C0D1CF5F71FFA3F49061CF5F7F5
:10AEF00037F9301C8A463C49F5F7EEF8FA263B4A0A
:10AF0000B6008718301C78433949C838F5F7E4F89B
:10AF1000C71980083F1A301C78433649C838F5F7FE
:10AF2000DBF8814633484B465843311CF5F7D4F8DB
:10AF30003F1A7743304ABB46101C30495844F5F756
:10AF4000CBF8E121071C09015046F5F7C5F8E121CE
:10AF5000079009015046F5F703F98A46081C3C2181
:10AF6000F5F7BAF83C2108905046F5F7F9F8234870
:10AF7000FA2278435200131C5B448A46181A311C8B
:10AF8000F5F7AAF8092F22D803374B46FFB29EB235
:10AF9000079AFF231840089B0292524601900393A0
:10AFA0000492201C291C0F4B0D4A0097F5F7BCF9A1
:10AFB000404605920999124A331C01F0EFFF4046C2
:10AFC0000BB03CBC90469946A246AB46F0BD4E46FF
:10AFD000093F0136FFB2B6B2DAE7C046C046C04606
:10AFE000E803000000000000805101006DFA0A0033
:10AFF000DA502D02C29205000CFEFFFF8877000098
:10B00000084E0200C046C04600B587B06B46D973F3
:10B010000F3305AA191C012300925B42012204F0A0
:10B0200087FB07B000BDC046E1235B020360082335
:10B0300043714E23C3710371012383717047C0466E
:10B0400070B5012384B0051C0393002603AC694648
:10B050000094281C0B310122002304F073FB00280C
:10B0600002D0301C04B070BD039B012BF9D1013616
:10B07000EDE7C04638B5C6239B00C458B425AD00E3
:10B080006359002B04D149B26068A36898476051A6
:10B0900038BDC046F0B5C6239B00C45885B063696F
:10B0A000A1690022684602728B420ED00121017212
:10B0B000E118097C01336D460170032B03D96261ED
:10B0C000287805B0F0BD6361FAE7B426B600A2594E
:10B0D000002A02D001204042F3E7642360686946F9
:10B0E00002AAE768B8476D462B7AA051002BE7D13A
:10B0F000F0E7C04670B5041C0D1E0A2D0DD0B42318
:10B100009B00C058002800D070BDA3686068291C4F
:10B110009847B4239B00E050F6E7B426B600835965
:10B12000002BF1D140680D21A3689847A051E9E7B1
:10B13000F0B54D4644465F465646F0B489464369ED
:10B1400081698DB0041C8B4200D1CCE0C3181B7CFC
:10B150004A461370436901334361032B50D8B4232B
:10B160009B00E35801931D1C002D41D14F463B78B5
:10B170001B2B48D0E02B3BD1019F0AAE08AD3221FA
:10B18000301C2F7002F018F801235B4229789A4690
:10B19000B4239B0088469B464346002B19D1301CA4
:10B1A00002F020F8002814D16369A269934200D10B
:10B1B00083E001222A70E218127C06A901330A708A
:10B1C000032B00D9434663610023CB56FF221A406C
:10B1D000924655464B2D00D1D3E000DCCBE04D2DFF
:10B1E00000D1C4E1502D00D003E1182349460B7073
:10B1F00001980DB03CBC90469946A246AB46F0BDC6
:10B2000000234361ABE7019F0AAE08AD3221301C39
:10B210002F7001F0D1FF01235B4229789A46B423B5
:10B220009B0088469B464346002B18D1301C01F0FA
:10B23000D9FF002813D16369A269934227D0012264
:10B240002A70E218127C06A901330A70032B00D978
:10B25000434663610023CB56FF221A40924657466D
:10B260005B2F00D191E057460137C1D05146CDB296
:10B27000A16900224B1C03209842524152421340C4
:10B2800062699A42B4D061180D74A361B0E75F4659
:10B29000E759002F07D106A960682A1C0023E76838
:10B2A000B847594660502B78002B00D0A1E101200F
:10B2B00003F08AFC2A789046B5E75F46E759002FED
:10B2C00007D106A960682A1C0023E768B8475946D9
:10B2D00060502B78002B00D08DE1012003F074FC2E
:10B2E0002A78904658E7B4239B00C55898460195A4
:10B2F000002D00D07CE7C623DB00C358002B0BD108
:10B300000123E568406849460AAA5B42A8474746C8
:10B310000190E051019D27E7B84F0AAE3570C5197D
:10B320003378002B00D026E1281C01F05BFF0028B9
:10B3300007D0B4233E229B00E2503E2701973D1CDC
:10B3400012E7494664236068321CE768B8473378DF
:10B3500041466050281C002B06D001F035FF4246C4
:10B36000A758002FDCD0E9E701F03CFF0028E0D12E
:10B370004346E758F5E7482D3BD105234F463B7040
:10B3800036E713234A46137032E700233221301C7C
:10B390002B7001F011FF01235B4229789A46B423F8
:10B3A0009B0088469B464346002B19D1301C01F078
:10B3B00019FF002814D16369A269934200D1C1E04A
:10B3C00001222A70E218127C06A901330A70032BAD
:10B3D00000D9434663610023CB56FF221A409246B0
:10B3E0005346333B112B00D988E0854A9B00D35844
:10B3F0009F465146013100D1FAE6A16900224B1C5B
:10B400000320984252415242134062699A4200D14D
:10B41000EEE6611855460D74A361E9E613234D4627
:10B420002B70E5E604234F463B70E1E618234A46BD
:10B430001370DDE6052349460B70D9E6002332215F
:10B44000301C2B7001F0B8FE01235B4229789A462C
:10B45000B4239B0088469B464346002B19D1301CE1
:10B4600001F0C0FE002814D16369A269934200D1A3
:10B4700083E001222A70E218127C06A901330A70C7
:10B48000032B00D9434663610023CB56FF221A40A9
:10B4900092465546013500D184E057467E2F00D1B3
:10B4A0009FE0A36903205A1C002190424941484271
:10B4B00061691040814205D0E3185B221A74A061D3
:10B4C000031C421C0020032595424041404210408D
:10B4D000814205D0E31833221A74A061031C421C78
:10B4E000002003259542404140420240914200D154
:10B4F0007EE6E31855461D74A26179E6A269002133
:10B50000531C03209842494149420B4061699942CA
:10B5100004D0A2185B201074A3611A1C5546013593
:10B5200000D165E6531C002003269E424041574649
:10B530004042FDB20340994200D159E6A218157469
:10B54000A36155E65F46E759002F07D106A9606859
:10B550002A1C0023E768B847594660502B78002B17
:10B5600043D1012003F030FB2A7890461BE70423E7
:10B570004D462B703CE60027E0E65F46E759002F7A
:10B5800007D106A960682A1C0023E768B847594616
:10B5900060502B78002B2AD1012003F015FB2A786C
:10B5A000904659E7A36903205A1C00219042494163
:10B5B000606949421140884205D0E3185B221A7441
:10B5C000A1610B1C4A1C00210325954249414942B7
:10B5D0000A40904200D10BE6E31833211974A261AE
:10B5E00006E67F2349460B7002E606A9F3E606A9A4
:10B5F0004AE706A92EE606A9E6E5C0462C060000A5
:10B600002C4E02000EB410B5041C83B000280ED0DE
:10B6100006AB0848211C059A0193FAF771FAB42386
:10B620009B00E05803B010BC08BC03B018470020D2
:10B63000F8E7C046F5B00100F0B557464E4645461E
:10B64000E0B4274C1F1C251C012382B0814688468C
:10B65000161C10359A46301C216801F033FF002873
:10B660000ED153463B700023AC420DD00434002B66
:10B67000F1D1002002B01CBC90469946A246F0BD14
:10B6800001235B42AC42F1D1002BF2D0154C1023C8
:10B690001B19301C21689A4601F014FF00280BD1B9
:10B6A000387054450CD004340028E2D0301C216896
:10B6B00001F008FF0028F3D0012568425445F2D17B
:10B6C0000028D7D0084B48460093084B08490193FF
:10B6D000321C43460125FFF795FF6842CAE7C04682
:10B6E000885002007450020094670200AC670200A8
:10B6F000BC500200F0B557464E464546E0B4804681
:10B70000C8688A468446021C00780023041C002670
:10B710002021002C16D065B2202D46D1013214789C
:10B7200065B2202DFAD05B2D25D0251C8D436DB23E
:10B730000136002DEDD001321478251C8D43FAD14D
:10B74000002CE8D1F71A32D15B494046FFF75AFF87
:10B750005046A9239B0041684046C258AA20800059
:10B76000031C5046046843444046A0471CBC904616
:10B770009946A246F0BD0133141C012707E00122BF
:10B78000A25601345D3A551EAA415242174025780F
:10B79000221C002D06D0202DF1D1002FEFD1202426
:10B7A0000136B6E700240136B3E765B2BBE753467E
:10B7B000996800250C782023002C16D062B2202A2C
:10B7C00078D101310C7862B2202AFAD05B2A3BD0C2
:10B7D000221C9A4352B20135002AEDD001310C7877
:10B7E000221C9A43FAD1002CE8D1002261469146EE
:10B7F0002023002816D044B2202C59D101310878DA
:10B8000044B2202CFAD05B2C37D0041C9C4364B289
:10B810000132002CEDD001310878041C9C43FAD190
:10B820000028E8D1A92189004346595855194A46AC
:10B83000AD1AA94200DB87E7404620493A1C63461F
:10B84000FFF7E0FE002091E70C1C012207E0012138
:10B85000615601345D394E1EB14149420A40267895
:10B86000211C002E06D0202EF1D1002AEFD1202459
:10B870000135A1E7002401359EE70120814401261E
:10B88000081C07E00121415601305D394C1EA141E1
:10B8900049420E400478011C002C06D0202CF1D126
:10B8A000002EEFD120200132A3E700200132A0E7D3
:10B8B00044B2A8E762B289E7304A0200E4500200CD
:10B8C000F0B5474680B44369826982B0041C0D1C00
:10B8D000934211D0C3181B7C0B7043690133436141
:10B8E000032B06D8B4239B00E05802B004BC90465A
:10B8F000F0BD00234361F5E7B427BF00C05900281D
:10B90000F3D1C623DB00E358002B07D10123606885
:10B910006A465B42E568A847E051E6E7194A6B468C
:10B920001870A618B8466A461378002B27D1301C29
:10B9300001F058FC002806D0B4239B003E22E250C0
:10B940003E23181CD1E76A466423E7686068291C17
:10B95000B8476F463B784246A050301C002B07D0BA
:10B9600001F032FC4246A358002BDCD0181CBCE787
:10B9700001F038FC0028DFD14746E359F4E7002303
:10B98000181CB2E72C06000070B54369041C8069DE
:10B99000834210D001201070E3181B7C0B70636988
:10B9A00001336361032B03D8B4239B00E05870BDBF
:10B9B00000236361F8E7B425AD0060590028F6D193
:10B9C00060680023E668B0476051F0E738B5B425F9
:10B9D000AD00041C4059002803D16068A368984753
:10B9E000605138BD70B5041C0D1E0A2D0DD0B42356
:10B9F0009B00C058002800D070BDA3686068291C57
:10BA00009847B4239B00E050F6E7B426B60080596F
:10BA10000028F1D160680D21A3689847A051E9E79B
:10BA2000014B0022C25070470C060000F0B54F4693
:10BA30004646C0B43F4985B0041CFFF7E3FD3E4BCA
:10BA4000E2580132162A06D8E250012005B00CBC9B
:10BA500090469946F0BD0026E6503849201CFFF775
:10BA6000D1FD6369A1698B4221D0E218127C6D4639
:10BA700001332A70032B16D863613149201CFFF76C
:10BA8000C1FD2B782022191C914351290DD05BB2A6
:10BA90001B2B0AD00D2B01D00A2BD6D1264B1722F7
:10BAA000E2500120D2E76661E7E70020CEE7B42349
:10BAB0009B009846E3586D46002BDED1C622D2008B
:10BAC000A258002A09D101236068694602AA5B4294
:10BAD000E668B0474746E051CFE71A4A02AE12196E
:10BAE000337091463378002BC7D1484601F07AFB7A
:10BAF000002804D0B4233E229B00E250BDE76946F3
:10BB000064236068321CE768B84733784146605068
:10BB10004846002B06D001F057FB4246A358002BA5
:10BB2000E0D0AAE701F05EFB0028E3D14746E359E5
:10BB3000F5E7C046304A02000C060000085102003A
:10BB4000105102002C060000F0B55F464D464446F9
:10BB50005646F0B495B012931EAB1B780024119397
:10BB6000B74B0B90C450081C13920D9106F073FD57
:10BB70000B9DC523DB00EC502F6880229200BA5841
:10BB800010900C97002A09D100250F950F9815B039
:10BB90003CBC90469946A246AB46F0BD3F680122A8
:10BBA000EA500997002FEFD0012500270A950F973B
:10BBB000099D2024AD68281C089506F04CFD0D9FBA
:10BBC000109D3F78089B0D9E0E90021C07970695CE
:10BBD000381C202800D1B0E0002800D1B9E0701C4A
:10BBE0009C460778851B3B1C011CA3430130002B9E
:10BBF000F7D1634607971878202800D1B5E00028D0
:10BC000000D114E194465F1C1A1C8846381C037846
:10BC1000B91AA3430137002BF8D1131C8B46624697
:10BC20004146002D00D107E15F46002F00D105E11C
:10BC30005D456AD8E04681468A460027AC46181C16
:10BC4000311CC35DCD5DDEB2321C613A192A02D8C7
:10BC5000331C203BDBB2EEB2321C613A192A02D807
:10BC6000351C203DEDB201379D424ED16745E8D1EC
:10BC7000069B4246DB1B069306985F465146D21B45
:10BC80004B46002878D10F9D002D7AD0139D129F2E
:10BC90002B683F68089D0124EE1999680898B446FE
:10BCA0000025261C0378002B1FD00A78002A1CD000
:10BCB000002E1AD0604518D0DFB23C1C613C013028
:10BCC0000131192C02D83B1C203BDBB2D7B23C1C03
:10BCD000613C192C02D83A1C203AD2B29A4200D0C8
:10BCE00090E003780135002BDFD1129F3D60119F5A
:10BCF000002F52D10F9D0B9F01350F95C5230B9D32
:10BD0000DB003F68EB580C970A9380230C9F9B0045
:10BD1000FB580A9DAB4200D838E72F1C2B1CC522CC
:10BD20000B9DD2000133AB500C9DBA0052590992C1
:10BD3000002A00D12AE70A933AE70699002908D099
:10BD40000F1C711C7678013F069707960E1C07980A
:10BD50003FE71878311C0025202806D04FE7013333
:10BD60001878013A202800D049E7002AF7D10022AC
:10BD70000698401B069086D0002AE7D10F9D002D23
:10BD800084D1119D0E98002D46D1129D099F2860E7
:10BD9000139D2F60119F002FACD0099809998068DE
:10BDA000C96803900291039A0B982649029BFFF7FA
:10BDB00029FC0B9AD569002D19D0099FB426BF68BC
:10BDC000B600381C019706F046FC041C0998C068B0
:10BDD000009006F040FC0019471C0B9CA84206D2BC
:10BDE000A159002910D0381C471CA842F8D3099D3E
:10BDF00015492A690B98FFF705FC0B98FFF716FE0B
:10BE0000119077E700264DE760682021A2689047EF
:10BE1000E569A051381CE7E70B980C49FFF7F2FBE6
:10BE2000099FBF68381C049706F015FCADE7181C85
:10BE3000002D03D100239B465F46D21B031C97E7CE
:10BE40000C0600002051020028510200304A020076
:10BE5000F0B556465F464D464446F0B48A46CF4953
:10BE6000071C97B0401800211C1C161C01F0A4F9F7
:10BE70000021CB4A381C06F0DEFBB5229200BD182B
:10BE8000C849C94AFE23281CFEF744F9C74B20992C
:10BE9000FF5053463B60C5230022DB00BC60F960C5
:10BEA0007E60FA508022920051468A580024002A6F
:10BEB00002D001220C68FA508023C5269B00F600B0
:10BEC0009946002C11D0A06806F0C5FB8046E068BA
:10BED00006F0C1FBFA694044904200D9F86151462E
:10BEE0004944BB5909688B425FD3381CB049FFF7FE
:10BEF00089FBB4239B002022F850D21900239A46D4
:10BF0000141CAB4600232022BB54A8239B00FB58E3
:10BF1000201C0D9306F09FFB0D990126B0460025CD
:10BF20000E1C42461090002A05D0381CA149221C44
:10BF3000FFF768FB109D381C0EA9FFF7F9F80028E1
:10BF400039D0B4239B00FD58002D43D1201C06F0AE
:10BF500082FB14900028D5D014AB0095381C211C0E
:10BF600015AAFFF7F1FDA92080003D50231C1A7887
:10BF7000002A02D128E001331A78202AFBD0395850
:10BF8000082905DC4A1CAA3189003A50CB511A789D
:10BF9000002A04D118E001331A78002A14D0202A8C
:10BFA000F9D1514619700133E1E75A1C51469B0003
:10BFB000BA515C5885E70EA90B787F2B00D99FE119
:10BFC0007D499A008A589746381C1599FFF792FBCD
:10BFD000002897D0794C3959002906D0C222D200C6
:10BFE000B818FCF717FE00233B51B4239B00F85808
:10BFF00017B03CBC90469946A246AB46F0BD012323
:10C000000093381C10AB211C12AAFFF79DFD031CE6
:10C01000581E8341DBB2201C984606F01CFB80E7CB
:10C020006749381CFFF7EEFA013603235246B34244
:10C03000524153421E40F101A0317918201C06F0F4
:10C0400002FB201C06F007FB0123984669E7002D40
:10C050002AD0B4239B009846FB58002B05D1786862
:10C060000821BA6890474346F850201C06F0F3FABE
:10C070000021013D884654E7109A954214D27B195D
:10C0800020331B785BB298460A2B00D12AE1B423F7
:10C090009B00F858002806D178684146BA68904756
:10C0A000B4239B00F8500135201C06F0D4FA00237D
:10C0B000984636E74249381CFFF7A4FA201C06F0E0
:10C0C000CAFA012290462CE71099002956D1201C6B
:10C0D00006F0C1FA0022904623E752460092381C2F
:10C0E000211C12AA10ABFFF72FFD0028DCD0201C6A
:10C0F00006F0B1FA1099002289469046884200D392
:10C100000FE7129B201C996806F09DFA49467B18A0
:10C11000203352461A702A49381CFFF773FA201C44
:10C1200006F099FA01239846FBE6109B002BBBD042
:10C13000002D2DD09D4266D3013D7B192033524600
:10C140001A70B4239B009846FB58002BBFD1786827
:10C150000821BA6890474346F8500028B7D178685C
:10C160002021BA6890474346F850002810D17868DB
:10C170000821BA6890474346F85009E053460093B7
:10C18000381C211C12AA10ABFFF7DEFC012819D0C5
:10C19000201C06F060FA00218846C2E62C0600004A
:10C1A0003406000095B0010075B00100EC050000F8
:10C1B0008851020098510200744E020024060000CB
:10C1C000304A0200A8239B00FD580323002D00D015
:10C1D0006B1ED801A0303818211CF7F717FA002879
:10C1E00000D1AEE6E801A0303818211C06F02BFA89
:10C1F000A8239B00FA580132FA50032A00D8A0E67F
:10C200005246FA509DE66A1E90462032D219291CE9
:10C210005B1B91462031B4255A1C79184846AD0065
:10C22000109306F0E6F97B59002B04D178680821B9
:10C23000BA6890477851B425381C4946AD00FFF7DD
:10C24000E1F97B59002B04D178682021BA68904726
:10C250007851109DB4239B0001359946002D17D0CD
:10C260004B46FB58002B05D178680821BA689047E7
:10C270004B46F850013DF1E70EA90B780C99109A46
:10C2800088467D192035BA182B7021325346137019
:10C29000201C06F0E0F900214546884641E6381C9E
:10C2A0004C49FFF7AFF9002E00D191E0013EF101BA
:10C2B000A0317918201C06F0C6F9201C06F0CBF935
:10C2C000012188462DE6BE22D200BB1801225D4620
:10C2D0001A70281CFDF73CFF011EFADB281CFEF734
:10C2E00065F8F6E7B4239B00F9589946002900D079
:10C2F000D9E678680D21BA6890474B46F850C9E6F0
:10C3000059B288461E2954DD109A7E2A47D8954294
:10C3100033D26B1C0C93291C2033FB1820310132C3
:10C320007918181C521B0B9306F06CF9B4239B0070
:10C33000F9589946002905D178684146BA6890476E
:10C340004B46F8500B99381CFFF75CF91099B42351
:10C35000491B9B00884699464346002B8CD04A4691
:10C36000BA58002A05D108217868BB689847494621
:10C370007850012252429044EEE7B4218900894668
:10C380007958002908D14146BA68786890474B46E9
:10C390000EA9F850109A0B78691C884671E7B423EF
:10C3A0009B00FA589846002A00D07DE6786807215D
:10C3B000DFE6534620220749BB54381CFFF722F919
:10C3C000201C06F048F901210D9E00258846A8E5AD
:10C3D00003266CE7304A02000048704770E5FF1FF3
:10C3E000F0B557464E464546E0B4016882B0002994
:10C3F0000AD0214E8022920014210918B358884691
:10C40000814692467F2B05D902B01CBC90469946C6
:10C41000A246F0BD4A469468002B0ED0351C00277A
:10C420002B68201C996801F04DF8002809DB524662
:10C43000B35801370435BB42F2D89A004946B1508F
:10C440000EE05346F358781CBC008000DF1B311906
:10C45000BA00301806F0D6F852464946B358315162
:10C46000142152460133C1468844B3504246143A1F
:10C470001268002AC6D1C7E770E5FF1FF0B547462E
:10C4800080B4061C171E012F0BDD1D1D094B012456
:10C49000984604CD301C41460134FFF7B3F8BC4246
:10C4A000F7D1301C0449FFF7ADF8002004BC9046DA
:10C4B000F0BDC046B4550200304A0200F8B5061C73
:10C4C0005868171C1D1C00F0B9FD0021041CF3F76F
:10C4D00003FF002818D1022F08DDAB681B785BB280
:10C4E000682B13D06D2B1DD0642B15D01049201C48
:10C4F000F4F71CFBF3F75AFF02F066FB301C0D4902
:10C50000FFF780F80020F8BD0024E4E7201C0A496A
:10C51000F4F70CFB041CE9E7201C0849F4F706FBC0
:10C52000041CE3E7201C0649F4F700FB041CDDE7CC
:10C5300000007A44304A02000000614500C0A8476C
:10C540000000704270B50021061C98681D1C00F0A8
:10C550005BFF0021041CE86800F056FF051C2B1C43
:10C56000301C0349221CFFF74DF82560002070BDE8
:10C57000B855020010B50021041C986800F044FF73
:10C580000349021C0368201CFFF73CF8002010BD83
:10C59000C8550200F0B556464D4644465F46F0B4D5
:10C5A000002187B0061C9868151C1C1C00F02CFF8D
:10C5B000032398430190301CFFF732FA032D6ADC05
:10C5C000402200923B4B3C4A3C4F9A469346009B8C
:10C5D0009846042B01D904239846424692004346CC
:10C5E00091460422002B00D04A46019902A806F089
:10C5F00000F8301C3249019AFFF704F801250024A5
:10C600000EE0301C5146FEF7FDFF301C391C072C94
:10C610004BD02022FEF7F6FF102D0BD00135013450
:10C62000A3089845EDD902AB1A5D301C5946FEF7B8
:10C63000E9FFEAE7301C5146FEF7E4FF4A460024D2
:10C640004D46002A0FD002AA135D2E22191C203954
:10C650005F2900D81A1C301C391C0134FEF7D2FFA8
:10C66000AC42F0D1A946301CFFF7E0F9009B4246EE
:10C670009B1A0093019B1A1C009B4A440192002BB9
:10C6800001D00028A3D1002007B03CBC90469946B9
:10C69000A246AB46F0BDE068002100F0B5FE0330D5
:10C6A0008008009000D08DE7EDE72D22FEF7AAFF6D
:10C6B000B4E7C046DC550200DC2E0200983E0200C2
:10C6C000D855020008B5012002F00EFC002008BD7C
:10C6D00008B5002002F008FC002008BD30B591B07C
:10C6E000041C02F075FA69464022051C00F01AFD90
:10C6F0002A1C031C0949201CFEF784FF02F052FF8C
:10C700004021051C6846FEF7DFFB0549031C2A1C77
:10C71000201CFEF777FF002011B030BDE05502006D
:10C7200008560200F0B54D4644465F465646F0B402
:10C7300095B0814602F076FA8046002800D1FEE0EE
:10C74000002400250026301C02F06EFA00280CD0D0
:10C750000EA902F079FB002807D1139A0023049256
:10C760000593049A059BA4185D4101364645EAD11C
:10C7700048467749FEF746FF2B1C234300D0A1E033
:10C78000744A4846111C92460025FEF73BFF0EAC4A
:10C79000714E02E0013545451CD0281C02F044FAD8
:10C7A0000028F7D0211C02F04FFB0028F2D1237C97
:10C7B000311C0093E36848460193A26802926368C3
:10C7C0002A1CFEF71FFF013548465146FEF71AFFA7
:10C7D0004545E2D107A808A902F0ECF9089B079AA1
:10C7E00093426DD300230793002701F00DF85B49B6
:10C7F0008046F3F771FC041C01F00CF85749051C46
:10C80000F3F76AFC564A574B0297D31A0093079BDB
:10C81000554F0193554B089AFB1A504F061C039233
:10C820005349544A4846FEF7EDFE381C60434346E0
:10C83000FA21181A8900F3F74FFC01967E43FA217A
:10C8400000908900A81BF3F747FC231C02904A497B
:10C850004A4A4846FEF7D6FE09A8642100F0ACFC1F
:10C86000002400E0013409A800F0BCFC0028F9D045
:10C87000221C48464249FEF7C5FE48464149FEF79C
:10C88000C1FE0BA90020FCF763F83F4C0BAA211C4A
:10C890004846FEF7B7FE48463C49FEF7B3FE0BA9F3
:10C8A0000120FCF755F84846211C0BAAFEF7AAFE0A
:10C8B000002015B03CBC90469946A246AB46F0BD60
:10C8C000D71A92E732494846FEF79CFE214B48466C
:10C8D000191C9A46FEF796FE1F4A00270EAE934695
:10C8E00003E00137474500D174E7381C02F09CF99A
:10C8F0000028F6D0311C02F0A7FA0028F1D1337CD1
:10C9000059460093F36848460193B26802927368EF
:10C910003A1CFEF777FE7069642200230021F3F7CA
:10C9200023FD221C2B1CF3F7FFFC1A49021C48466E
:10C93000FEF768FE48465146FEF764FED1E74846DA
:10C940000349FEF75FFE48460249FEF75BFE41E7FA
:10C9500030560200304A02006856020040420F0082
:10C96000F0F6FF1FF4E0FF1FF4E0FF1F00E0FF1FE1
:10C97000905602006C690200C4560200F056020094
:10C98000F856020000570200045602001057020039
:10C99000605602008856020070B582B0041C002167
:10C9A00068460170012A07DD5A68201C1F496B4642
:10C9B000FEF742FE00280BD01D4BE358002B17D08A
:10C9C0001C4A201C1C49FEF71DFE002002B070BD51
:10C9D0006A461578002D0DD0154BE05800281AD066
:10C9E000201C1649FEF70EFE114BE358002BE7D131
:10C9F000134AE6E70E4EA359002B07D0C222D200FD
:10CA0000A018FCF707F9A5510D4ADAE7201C0D49DB
:10CA1000FEF7F8FDD0E7C422D200A4500A4AE25043
:10CA2000C222D200A018FCF7DFF8C5E73457020095
:10CA30002406000020570200745702003C570200F1
:10CA4000285702005C5702004DCA010008B5FEF7E6
:10CA5000C9FF002008BDC04670B5151C041C1E1C73
:10CA6000FCF790F80A49021C201CFEF7CBFD022DB2
:10CA70000CDDB06805F066FD40B2FCF77DF8FCF710
:10CA800081F80449021C201CFEF7BCFD002070BD8B
:10CA900090570200B0570200F0B55F4656464D462B
:10CAA0004446F0B487B0061C02F002FE83462049DB
:10CAB000301C5A46FEF7A6FD5B4600250020002BE1
:10CAC0002DD01C4B99461C4B98461C4B9A4618E09F
:10CAD00004AC2A1C4946FEF795FD381C211C02F0C7
:10CAE00041FE627923790092A279301C0192E279A9
:10CAF000414602920135049AFEF784FDE8B283456F
:10CB00000DD902F0D7FD071C301C002FE0D12A1CE4
:10CB100051460135FEF776FDE8B28345F1D8002095
:10CB200007B03CBC90469946A246AB46F0BDC04615
:10CB3000CC570200EC5702000058020014580200C3
:10CB4000F0B55F4656464D464446F0B48FB008AE49
:10CB500083460C1C101C311C1D1C9246189F02F0B1
:10CB600001FE002D19DD386805F0F2FC002800DC1C
:10CB7000FCE03060012D0CD07A681378453BDBB2C5
:10CB80002A2B00D9F8E09A4A9B00D3589F460022EE
:10CB900093465046311C02F0DFFD727933790092E2
:10CBA000B279201C0192F27992490292089AFEF71A
:10CBB00029FD5B46002B00D0A5E006AD07AA009238
:10CBC000012350460AA9102202F0BCFD0023994619
:10CBD00000280DD1079A9146002A09D000270AAAF9
:10CBE000D157201CFEF7F2FE079B0137BB42F6D857
:10CBF000102701230022B8462B70171C12E06A464A
:10CC0000117C01292FD0012249B250469144FEF7F0
:10CC1000FBF901235B4298444246002A10D02B784E
:10CC2000002B0DD0201C04A92A1CFEF7ADFE2B788A
:10CC3000002BEED05B46002BE1D16B46197CE2E77E
:10CC40004B46B846002B5AD04246002AB6D0201C8C
:10CC50006949FEF7D7FC00200FB03CBC90469946CE
:10CC6000A246AB46F0BD6F461B376449201CFEF759
:10CC7000C9FC727933790092B2795E490192F279F6
:10CC8000201C02923268FEF7BDFC5D49201CFEF7B5
:10CC9000B9FC5C49201CFEF7B5FC5B49201CFEF783
:10CCA000B1FC201C391CFEF70BFE0023FB564E2B5B
:10CCB00022D00BDC312B18D0322B0FD01B2BD4D130
:10CCC0000027201C5149FEF79DFCA2E76E2B13D0D4
:10CCD000782B01D0582BC8D10127F2E7012250460A
:10CCE000311CB27102F038FDBFE701235046311C00
:10CCF000B37102F031FDB8E700239B46E0E7012065
:10CD000001F062FFA0E7201C4149FEF77BFC54E7DD
:10CD10004F233371022D00D13BE7BA680023D3566D
:10CD2000382B2FD108237371032D00D131E7FA6816
:10CD30000023D356312B58D0322B29D0201C354913
:10CD40007A69FEF75FFC042D00D122E73A69137877
:10CD5000343BDBB23E2B42D82F4A9B00D3589F4630
:10CD60004E233371D6E745233371D3E7201C2B497B
:10CD7000BA68FEF747FCFDE6201C2949FA68FEF771
:10CD800041FCC7E7201C27493A69FEF73BFCCBE78B
:10CD90000223B371D7E75223F371052D00D1F8E6D2
:10CDA0007A691378303BDBB2492B06D81E4A9B00C8
:10CDB000D3589F4601239B46EBE6FA69201C1B498A
:10CDC000FEF720FCE5E64E23F371E6E74823F37116
:10CDD000E3E74323F371E0E73423F371DDE7201C3D
:10CDE0001349BA69FEF70EFCD7E70123B371AAE72E
:10CDF000CC5102000058020058590200304A02008B
:10CE0000D458020000590200405902006C59020037
:10CE1000C05802006C5802007852020024580200E8
:10CE20003C5802005458020074530200A0580200FB
:10CE300084580200F0B5474680B4071C84B0986857
:10CE400090461E1C05F07EFBC4B2051C02F030FCAF
:10CE5000844213D2201C02F02DFC0390021E1BD032
:10CE6000381C1849FEF7CEFB0C364346033B0096B0
:10CE7000391C039A0120FFF763FE08E002F018FC5A
:10CE8000FF22031C2A40381C0F49FEF7BBFB002081
:10CE900004B004BC9046F0BD201C03A902F02AFC9B
:10CEA000FF222A40002807D1381C0849FEF7AAFBB8
:10CEB000039A002AEBD0D3E7381C0549FEF7A2FB02
:10CEC000E5E7C046B0590200C45902007C5902008F
:10CED0009459020008B50248FFF782FA08BDC0461F
:10CEE0009C540200F0B5B425094C0A4F0A4E83B099
:10CEF000AD00FFF771FA3B1C011C0096201C0022BC
:10CF0000FEF7A6FF6359002BF3D003B0F0BDC04677
:10CF100074E7FF1F99D80100D1D8010030B589B05E
:10CF200005AC0D1CC068211CFDF75CFFE178228870
:10CF3000A37800912179281C019161790291A1794E
:10CF40000391024900F04AFA09B030BDC84D020011
:10CF500010B5847D82B0027D437D002C05D1081C74
:10CF6000054900F03BFA02B010BD081C00940349CB
:10CF700000F034FAF7E7C046085C0200005C0200EB
:10CF800042688368013A934207D25A1C8260026861
:10CF9000D154026883680021D15470470CB400B5A5
:10CFA00085B006AB04CB002201900291039202707F
:10CFB00001A9069A03480093F8F7A2FD05B008BC42
:10CFC00002B0184781CF01000CB410B584B006AC94
:10CFD00008CC0291019005F03EFB01A90390069A4E
:10CFE000231C04480094F8F78BFD04B010BC08BC67
:10CFF00002B0184781CF0100F0B58446002A1AD04C
:10D00000002404E0002B15D00134A24212D0604667
:10D0100003570E571F1C413F351C192F00D82033D2
:10D02000371C413F192F01D8351C2035581B2B4385
:10D030000028E7D0F0BD0020FCE7C046F0B5474629
:10D0400080B40024071C3E5D73B2202B35D00D2B1D
:10D0500033D0F2B2111C093901292ED92D2B2ED033
:10D060002B2B32D0FE239B059846303A0025092A07
:10D0700014D82A49281CF3F759FD76B2051C301C38
:10D080003038F4F713F8011C281CF3F7FFF90134CA
:10D090003E5D051C331C303B092BEAD976B22E2E9F
:10D0A00017D0FE27BF054146281CF3F73FFD391C6A
:10D0B000F3F758FB04BC9046F0BD0134C3E7184BAE
:10D0C000984601343E5DF2B2CFE7FE239B059846B9
:10D0D000F7E701343C192678FE27331C303BBF05A7
:10D0E000092BE0D80D49281CF3F720FD76B2051C6A
:10D0F000301C3038F3F7DAFF011C281CF3F7C6F9AF
:10D100000649051C381CF3F711FD6678071C331C13
:10D11000303B0134092BE5D9C5E7C046000020416A
:10D12000000080BF70B50D1CFA218900161CF2F7B3
:10D13000D3FF1C49041CF2F7CFFF0022031C2A7006
:10D1400027D1E121201C0901F2F7C6FF031E16D1E9
:10D15000201C3C21F2F7C0FF031E08D00201121A66
:10D160009200A41A281C311C0F4AFFF72DFF281C1F
:10D17000311C0E4A231CFFF727FF281C70BDE1223B
:10D1800012014243311CA41A281C094AFFF71CFF54
:10D19000DEE7044A311C4243281CA41A054AFFF763
:10D1A00013FFCEE780510100285C0200385C0200CA
:10D1B0001C5C0200105C020038B50D1C041C01F060
:10D1C00007FD21C438BDC04610B5041C01F000FDA8
:10D1D000206010BD10B5041C01F0FAFC2368C01AD1
:10D1E00010BDC04610B5041C01F0F2FC2368C01A43
:10D1F000636883428041404210BDC04610B5041CA4
:10D2000063680020002B07D001F0E2FC2368C01AFD
:10D21000636883428041404210BDC04610B5041C83
:10D2200001F0D6FC2268831A626800209A4200D37B
:10D23000D01A10BD08B5044B88601960C0890C3144
:10D24000F9F762F808BDC046A8EDFF1F70B5114D93
:10D25000041C2B685E68002E06D0186823041B0C83
:10D2600000210022B0472B68181C9B680C30D9891C
:10D27000F9F75AF80020002C0AD02B681C209B6874
:10D28000DA891B689B68DB685A43A242A4412040AC
:10D2900070BDC046A8EDFF1F08B501384342584194
:10D2A000C0B2FBF795FA08BD054B10B51B685C686A
:10D2B000002C04D01868032100220023A04710BDD1
:10D2C000A8EDFF1F064B10B51B685C68002C04D04E
:10D2D0001868022100220023A047002010BDC0468C
:10D2E000A8EDFF1FF0B55F4656464D464446F0B4E4
:10D2F00087B00591354982460B6891465C688B463C
:10D30000002C04D01868012152464B46A047002447
:10D310004B46002B4FD0002C4DD15B461E6850462B
:10D32000B5682B689B68DC68211CF2F7D5FE81B2DA
:10D33000071C88465046211CF2F712FF8AB20904E6
:10D34000090C049249444A4603928C4203D2049B3E
:10D35000E41AA4B20394EB89434534D93F043F0C4B
:10D36000301C0C30391CF8F7F7FF002814D0594650
:10D370000B68059A986841460092039B049AFAF755
:10D3800045FD039B05994A46C9189A44D31A9BB296
:10D39000041C05919946BBE759460B6841469868BD
:10D3A000FAF778FD5A46041C1068391C0C30F8F75F
:10D3B000E3FF002CDBD0201C07B03CBC9046994614
:10D3C000A246AB46F0BD0124F5E7C046A8EDFF1F1D
:10D3D00003685A1C026019707047C0460EB400B54D
:10D3E00084B00190002809D006AB059A054801A930
:10D3F0000393F8F785FB019A0023137004B008BC6F
:10D4000003B01847D1D3010030B5031E57D00278BE
:10D41000002A54D0002920D1002012E02034052C0D
:10D420003DD930390024092904D8000152B28018AE
:10D4300030380124002B14D01A78002A11D0002C87
:10D440000FD0D1B20C1C613C0133052CE6D8000191
:10D4500052B2801857380124ECE7411800208B4263
:10D4600000D130BDD4B2251C613D0133052D0CD84F
:10D47000000152B2801857380125002BF1D01A78DC
:10D48000002AEED0002DEAD1EBE7251C413D052D09
:10D490000BD8000152B2801837380125EDE70001A2
:10D4A00052B2801837380124C4E7303C0025092CDB
:10D4B000E3D8000152B2801830380125DDE70020A2
:10D4C000CFE7C046F0B5071C002404E0002B18D0BD
:10D4D0000134002A15D03B5D0A5DDDB22E1C413EB1
:10D4E000192E02D82B1C2033DBB2D5B22E1C413EA4
:10D4F000192E02D82A1C2032D2B25DB256B2A81B15
:10D50000E4D0F0BD30B5144C051CABB0201C052197
:10D51000124A2B1CFBF796FB684600236A46291C1F
:10D520000130137005F08FF80D4B0122186852423C
:10D53000694601F05FFB6A461378002806D0201C7C
:10D540000421084AFBF77EFB2BB030BD201C0621CE
:10D55000054AFBF777FBF7E7485C0200485D0200ED
:10D56000ACEDFF1F2C5D0200185D0200F0B54446D3
:10D570005F464D465646F0B43E4A3F4C89B083461E
:10D58000002590466668434601211868494203F029
:10D5900075FAF1790223994301394B425941B37924
:10D5A00049017F2B61D833681A680023D360B379AF
:10D5B0001F2003400B431360802113681942FCD0E5
:10D5C00013699A461F2313604246106802F028FF31
:10D5D0005346226898B2636891465246DE799F8826
:10D5E00013041B0C9A46032E31D9082E1BD0F3F7D7
:10D5F000B9FD5346029300960197F5F7F9FB2A1CF3
:10D60000049005914B4658461C490135FDF7FAFF39
:10D610000834042DB6D1002009B03CBC9046994690
:10D62000A246AB46F0BDF3F79DFD1549F3F77EFA30
:10D63000DE218905F3F77AFA1249F3F7A1FB1249C3
:10D64000F3F790F8011C1148F3F79AFBD1E7F3F7D1
:10D6500089FD0790381CF3F785FD011C0798F3F747
:10D6600065FA0B49F3F77EF8C3E733681A681023AD
:10D67000D3609CE7B0EDFF1F045E02009C5D0200DA
:10D68000333353406210383FDAC9E03A0000C841F2
:10D6900000007A4C08B5042002F074FC0D4B1860B1
:10D6A000DB2000F07DF800F0B5F80B4A04230B49AD
:10D6B00000F0B6F86023400118400C231843084BD3
:10D6C00000229860DA601A6246225A621F221A60AB
:10D6D00008BDC046B0EDFF1F645D0200001BB7002F
:10D6E00000B0034070B5254D0121041C4942286853
:10D6F00003F0C4F9E1790223994301394B425941BE
:10D70000A37949017F2B33D823681A680023D3609B
:10D71000A3791F2003400B43136080211368194233
:10D72000FCD01F2316692868136002F079FEE379A4
:10D73000032B17D9082B02D0B0B200B270BD36044B
:10D740000F4A360C7243FA2312149B0053430D4ABE
:10D7500064209B1858430C49F2F70CFD0B4BC01882
:10D7600080B2EAE7A3883004000C5843000CE4E7D9
:10D7700023681A681023D360CAE7C046B0EDFF1FC4
:10D78000E40C00006807F5FF4DF9FFFFC409000035
:10D7900008B50248FEF724FE08BDC046745D0200CD
:10D7A00010B54309052B18D012D9062B0DD0072B25
:10D7B0000AD182230A4A5B011F2420400124D15848
:10D7C0008440201C0843D05010BD054A054BF3E7A8
:10D7D000042BF9D1024A044BEEE7014A034BEBE775
:10D7E000007004403C1000003410000038100000AD
:10D7F000014B18607047C046B8EDFF1F014B186021
:10D800007047C046B4EDFF1F014B18687047C04613
:10D81000B8EDFF1F014B18687047C046B4EDFF1FFD
:10D82000F0B54546984601235B4257464E469A4618
:10D830004346E0B481460F1CC244002B1BD0012696
:10D84000151C0024764202E00435002E0DD0484617
:10D850002968F2F741FCB84204D8381AB04201D224
:10D86000A246061C01344445EED150461CBC9046ED
:10D870009946A246F0BD01235B429A46F5E7C046B1
:10D88000044980230B7600230B700C228B791A42FB
:10D89000FCD170470040064008B5034B1868FDF7FF
:10D8A000B3FB002008BDC046BCEDFF1F10B5074C00
:10D8B000C0B2211C01F01EFF20680D21FDF7A4FB62
:10D8C00020680A21FDF7A0FB10BDC046BCEDFF1F7C
:10D8D00010B5141C00222270094A84B0106803AAF3
:10D8E0000092012201F02EFF002802D1039B012BA0
:10D8F00002D0002004B010BD024A23701370F8E774
:10D90000BCEDFF1FC0EDFF1F08B588220E4B0A219A
:10D91000520199500D4A2821117000221A60A82145
:10D920000B4A49059950A920FFF73AFFAA20FFF7B3
:10D9300037FFAB20FFF734FFAC20FFF731FFAD20FE
:10D94000FFF72EFF08BDC0460070044000E007400E
:10D950000410000008B5044A044B80214902D1504C
:10D96000FFF78EFF08BDC046007004404410000061
:10D9700038B50A4D0A4C0B482959090F0131F2F705
:10D98000ABFBFFF735FF29590648090F0131F2F7C4
:10D99000A3FB4008FFF732FF38BDC04600700440CB
:10D9A00044100000006CDC020E4B01205A78510735
:10D9B0000CD41A780020910608D41A78022052B2AA
:10D9C000002A03DB1A780420510600D570471A7824
:10D9D00003209107FAD41B78012018400623181A57
:10D9E000F4E7C04600F0074072B6012803D1044AAC
:10D9F000044BDA60FEE7044B044A0021D150F9E7FA
:10DA00000400FA0500ED00E004110000007004407D
:10DA100008B501F049FA044A044B5521D150AA2116
:10DA2000D15001F045FA08BD007004400411000017
:10DA300000207047012040427047C04670B50589FC
:10DA40001C248D4201D8201C70BDC568D618AE427A
:10DA5000F9D869434069002412185118034A049800
:10DA6000116193821A1C04F0C4FDECE7C4EDFF1FA2
:10DA700070B505891C248D4201D8201C70BDC56875
:10DA8000D618AE42F9D80D4C69434069A382049B75
:10DA900012185218A36003232261237103F048FF78
:10DAA000074B2060597880220A435A7001220020D7
:10DAB0000121524204F02EF8E468DEE7C4EDFF1FB6
:10DAC0000000024010B50289031C1C208A4200D8C5
:10DAD00010BDDA685B6951430B4CC9180023A3825F
:10DAE00001232161237103F023FF084B2060597843
:10DAF00080220A435A70012200200121524204F080
:10DB000009F8E068E4E7C046C4EDFF1F00000240EA
:10DB10000D4B00221A710D4A0D4B0121D0580143C3
:10DB2000D1500C4B3F215A780A405A700A4BC122FF
:10DB300092009858094901408020C0010143995042
:10DB400020221A607047C046C4EDFF1F00700440D9
:10DB50003C1000000000024000E100E0FF00FFFF79
:10DB600070B5002182B0A04B01911A79022A00D130
:10DB700079E04ED9032A22D0042A00D068E09B4ADB
:10DB800070201178084200D08FE0988A002800D1D8
:10DB90008EE0032800D900E19A68694615781C696F
:10DBA000561C0D70012800D1BDE05578961C4D70B3
:10DBB000022800D115E1957800200332B8E08B48A7
:10DBC000702404709D8A04241C71D960002D67D0D4
:10DBD00018699C68024000D06CE0621C013D24780A
:10DBE0006946ADB20C70002D00D1CDE0141C227836
:10DBF000013DADB24A700134002D00D1C7E0621C76
:10DC0000013D2478ADB28C70141C002D00D1C0E011
:10DC10005BE0012A1CD1754A702010700220D96087
:10DC200018711B6903218B430921D171190CC9B2E9
:10DC30009171190AC9B2DBB2517113716C4B802119
:10DC4000D86849020143D9608023137002B070BDC7
:10DC5000664B3F215A780A405A70654B654AD9682D
:10DC60000A40DA60F2E7614A702011780140481EEC
:10DC70008141D96051783F20014051705C4A5D4933
:10DC8000D0680140D1601868002101AA03F0ECFFC0
:10DC9000019B002BDAD08022574B52051A60D5E742
:10DCA00042783F210A404270E8E70121D960E1E76C
:10DCB000D860DFE7067869460E70012A97DD46785E
:10DCC0004E70022A9BDD82788A702278013DCA70EC
:10DCD0000134AAB29A820978444A9C60117269465A
:10DCE0000131097880245172694602310978640251
:10DCF0009172694603310978D17203218843062164
:10DD0000D171010CC9B29171010AC9B25171C1B28C
:10DD1000117137490430CD682C43CC6080211170DB
:10DD20001861019BB5E7627800204A70321CA57823
:10DD30008D70E5789A60CD702C4A097898821172BE
:10DD40006946013109780620517269460231097825
:10DD50009172694603310978D17203218C43D071E5
:10DD6000200CC0B29071200AE1B2C0B250711171A2
:10DD70001F498020CC6840022043C8608021117078
:10DD80001A6904321A6161E744784C70141C827875
:10DD90008A70C278CA7000229CE7996804380C78AF
:10DDA00014724C7854728C789472CC780431D4729A
:10DDB0001D690324A5432C1C0625D571250CEDB245
:10DDC0009571250AEDB2E4B255711471084C8025A5
:10DDD000E6686D023543E56080241470996098828E
:10DDE000CEE7321C0020A2E7C4EDFF1F0000024076
:10DDF000003000F0FFFFFEFF04ED00E010B5041C52
:10DE000001F0BCF803688268201CDA6001F088F831
:10DE100010BDC046F8B556464D465F464446F0B480
:10DE2000434D444BC822521992469946424A434BAD
:10DE3000061C90469B4611E01B69083519400B1CD7
:10DE4000FB401B1A581E83413D49301CFDF7DAFB8D
:10DE5000301C3C49FDF7D6FB554543D02C686A6819
:10DE6000301C4946FDF7CEFB2368374A934240D029
:10DE7000364A934243D0364A934246D0354A93427B
:10DE800049D0354A93424CD041466268301CFDF778
:10DE9000B9FB2368A1685A690A4091420CD01A69FB
:10DEA0006768207B0A40FA400228C5D12069BC007F
:10DEB000205801242040BFE71A681B6860680A40A8
:10DEC0001940237BC140CB1AC240591E8B41301CE4
:10DED0002249FDF797FB0835301C1A49FDF792FBE4
:10DEE0005545BBD100203CBC90469946A246AB4666
:10DEF000F8BD301C11494122FDF784FBC4E7301CFA
:10DF00000E494222FDF77EFBBEE7301C0B4943223F
:10DF1000FDF778FBB8E7301C08494422FDF772FB97
:10DF2000B2E7301C59464522FDF76CFBACE7C04612
:10DF3000905E020060610200706102006C6102008C
:10DF400088610200304A020000F00F4040F00F40AC
:10DF500080F00F40C0F00F4000F10F4078610200E8
:10DF6000F0B55F46564644464D46F0B49F6883B0D0
:10DF70008246381C04F06FFB264B81461C1DC433BF
:10DF80009846254B00269B460DE073685046009549
:10DF900059463A1CFDF736FB00260123444510D0B4
:10DFA0000834002B17D12568381C291C4A46FFF776
:10DFB00023F800230028F1D1002EE6D1261F444586
:10DFC000EED1002B07D1002E07D1504613493A1C41
:10DFD000FDF718FB16E0002E14D031680A68886837
:10DFE0004C68D06013681568097B03402840E04006
:10DFF000E340441A611E8C417268504600940849FF
:10E00000FDF700FB002003B03CBC90469946A246B9
:10E01000AB46F0BD905E020098610200D461020040
:10E02000BC610200037B002905D0002B05D00368EA
:10E0300082689A607047002BF9D0036882685A6042
:10E04000F8E7C046F0B544494D4610205F465646B5
:10E050004446F0B448604B69404C03434B61802315
:10E06000DB028B604A69022713434B6180231B0349
:10E070008B604A69042513434B61A760636980265E
:10E080003B436361364B82469D605A69AB462A43E7
:10E090005A615E6058692022304358613148944685
:10E0A0008260151C4269B0462A4342614660456958
:10E0B0002A1C324342612C4A750255605669354329
:10E0C0004646B6025561566055692E4345466D0475
:10E0D0005661956056693543556101255D60A846D6
:10E0E0002E1C5D6935435D614E69351CBD434D6134
:10E0F0004E69351C5E46B5434D6161694546A9438D
:10E10000616159695646B943596159690827B9434C
:10E11000596159696546B14359615969A9435961C2
:10E120005F6940218F435F614369B3434361436942
:10E130005E468B43436151690C4B0B4053615369FD
:10E140005B005B0853616369B34363613CBC904609
:10E150009946A246AB46F0BD00F00F4040F00F409C
:10E1600080F00F40C0F00F4000F10F40FFFFFFBFF5
:10E17000036881685A698A435A61704703688268F4
:10E1800059690A435A61704700B5031C85B00029DC
:10E1900015D0017B002915D11968986848600B4992
:10E1A0000B48009103A90191111C002200F0A8FE68
:10E1B000002802D1039800F0CFFE05B000BD017B1E
:10E1C0000029E9D1196898688860E8E7FDDD010059
:10E1D000F4610200037B002B03D1036882685A605C
:10E1E0007047036882689A60FAE7C046037B002B99
:10E1F00003D1036882689A607047036882685A6036
:10E20000FAE7C046037B002905D0002B05D0036840
:10E2100082689A607047002BF9D0036882685A6060
:10E22000F8E7C04603681A6883681A404368DA4012
:10E23000037BD01A431E9841C0B27047037B4168EC
:10E24000022B04D102698B009B5801221340026803
:10E25000806812691040C840C31A581E8341D8B262
:10E260007047C04608B50248FEF7BAF808BDC04678
:10E27000D05F020008B50A1C0149FCF7D7FC08BDB5
:10E2800025E001007047C046014B18687047C04642
:10E29000DCEDFF1F00B5154883B001F0ABFC01F0C9
:10E2A000A3FC134B1860FFF763FBFFF731FC00F092
:10E2B000ABFEFFF7C7FE00F049F8FFF7EBF901F0FE
:10E2C00057FA01F009FA01F00DF9FFF7DBFF03231C
:10E2D0000093C0220023019306495200064802F031
:10E2E00001FD02F0C7FE002003B000BD786302000C
:10E2F000DCEDFF1F886302008122020010B50023BD
:10E3000082B001930E4B802219680E4C0A431A60AA
:10E31000A368002B01D0E06898476068002805D00A
:10E32000002101AA03F0A0FC00236360019A002AE7
:10E3300003D08022044B52051A6002B010BDC046C3
:10E3400000000440E0EDFF1F04ED00E010B5A02048
:10E35000FFF726FA184B07211A7E04208A431A7603
:10E360001A7A0E218A431A72597801220A435A7086
:10E37000197803220A431A7001F004FE0F4B0121A1
:10E3800018600F4BFF241A688A431A601A684021EC
:10E390008A431A601868802202431A6000225A6079
:10E3A000084BC72292009858A043014399508022FD
:10E3B00052051A6010BDC04600400640E0EDFF1F48
:10E3C0000000044000E100E0F0B5294E294D474629
:10E3D0008846012180B4041C49423068171C02F0B1
:10E3E0004DFB2B68012293432B602B684022934303
:10E3F0002B602A68802313438022E0005202811898
:10E400002B60090C01292AD04B1E012B2CD0002493
:10E410000134E4B25B08012BFAD1E3007822022137
:10E420001A40A140134B7C255C68AC435C605C687F
:10E4300022435A600818F1F74FFE0E4B0004000CFF
:10E44000986019684246B26040220A43F7601A6039
:10E45000196801220A431A6004BC9046F0BD6A683C
:10E46000042313436B60E5E702210022DAE7C0468C
:10E47000E0EDFF1F000004401D4B012170B5494233
:10E48000041C186802F0FAFA1A480123436080233A
:10E490005B02E118090C012922D04B1E012B24D963
:10E4A00000220132D2B25B08012BFAD8D3007826C1
:10E4B00002211E4091400F4B7C255868321CA84316
:10E4C0005860586802435A600819F1F705FE094B75
:10E4D0000004000C9860196841220A431A6070BD5C
:10E4E0004268042313434360EEE702210026E2E77B
:10E4F000E0EDFF1F0000044008B5064B41211A68FB
:10E500008A431A6000225A60034B186801F088FFA2
:10E5100008BDC04600000440E0EDFF1F82680023F4
:10E520009375437E1F21194001238B40044A191C17
:10E530008023D1504368034A99680A409A60704723
:10E5400000E100E0FFFF00FF10B58368083311CB46
:10E5500011C1002010BDC046F0B54F4680B4069DE5
:10E560001E1C8F18002381462B600120B94211D058
:10E5700000280FD04A469368321C18684C1C01F0E2
:10E58000C3FF002803D02B68002601332B60211C19
:10E59000B942EDD1002004BC9146F0BDF0B54E4625
:10E5A00045465746E0B48568061C00F035FEAB7D55
:10E5B000002B6BD17468684BA2681340A3606B7D1D
:10E5C000002B00D18AE0737E307E5AB28146002A49
:10E5D00000DAA0E06149920892005218C021890037
:10E5E000575803200340FF20BC46DB00071C9F4018
:10E5F0009A466346BB439C464B469F01384057466C
:10E60000B840634603435350737E1F221A400123D0
:10E6100093401A1C514B1A6000F0FEFDA2684E4B4D
:10E62000A8681340A3606368E368A2688023DB05E1
:10E630001343A36001012869F1F74EFD484B98424E
:10E6400000D9181C20606B7B072B27D0FF23EB75AC
:10E650002B7B452B27D04F2B29D0A3680222934335
:10E66000A360EB7D7F2B2DD0AB7B2268012B6AD082
:10E6700080239B0113432360A268B0239B031343B1
:10E68000A36001232B75AB7500F0D2FD00F0D0FD27
:10E6900000201CBC90469946A246F0BD7F23EB7536
:10E6A0002B7B452BD7D1A3680122934302E0A268BC
:10E6B00001231343A360A26802231343A360EB7DED
:10E6C0007F2BD1D1A36810229343A360AB7B012B96
:10E6D0003DD0A36802229343A360CDE7FFF794F8EF
:10E6E000012128610022706901F024FC0022686089
:10E6F0000121306901F01EFC2860281C0830FCF75D
:10E7000093FC01236B75737E307E5AB27468814628
:10E71000002A00DB5EE70F221A40083A11499208EE
:10E720009200521803210B40FF21DB00D769081C1F
:10E73000984087434846BC46870139409940634624
:10E740000B43D36160E7084B1340236094E7A26852
:10E7500002231343A3608FE7FFFF00FF00E100E007
:10E76000FF1F000000ED00E0FFDFFFFF10B5041CFD
:10E77000807EFFF715F86368227B596812070A4309
:10E780005A60627B996812070A439A609968024A44
:10E790000A409A6010BDC046FFFF00FFF8B55F4613
:10E7A000564644464D46F0B483460A9898460023A0
:10E7B00003605B469E688023DB028F18814601243C
:10E7C0009A46B9420DD0002C0BD070684246002307
:10E7D0004D1C01F0EFFC041E012C09D0291CB9428C
:10E7E000F1D100203CBC90469946A246AB46F8BD0C
:10E7F000337D002B05D149460B6801330B60291C82
:10E80000EDE700F009FDF37B4F2B0BD05846426833
:10E81000936880200004034393600023337500F065
:10E8200007FDE8E759464A68044893680340936047
:10E83000936851460B42FBD1EAE7C046FFFFFBFF5E
:10E8400038B585682B1C083314C914C3446800F01C
:10E85000E3FCA268304B28691340A3606368E36857
:10E86000A2688023DB051343AA68A3601101F1F7B6
:10E8700033FC2A4B984200D9181C20606B7B072B75
:10E8800021D0FF23EB752B7B452B21D04F2B23D0A1
:10E89000A36802229343A360EB7D7F2B27D0AB7B41
:10E8A0002268012B2FD080239B0113432360A26891
:10E8B000B0239B031343A36001232B75AB7500F0BA
:10E8C000B7FC002038BD7F23EB752B7B452BDDD1BA
:10E8D000A3680122934302E0A26801231343A360CB
:10E8E000A26802231343A360EB7D7F2BD7D1A368DB
:10E8F00010229343A360AB7B012B08D0A3680222B4
:10E900009343A360D3E7064B13402360CFE7A2688D
:10E9100002231343A360CAE7FFFF00FFFF1F0000AD
:10E92000FFDFFFFF70B5002382B00193354B8022DB
:10E930005C68D203144202D09968114243D180230B
:10E940001B041C4203D02F4DAA681A4227D18023F2
:10E950009B031C4203D02B4A9168194211D1294BC9
:10E96000802259681203114202D059680A435A6042
:10E97000019A002A03D08022234B52051A6002B06C
:10E9800070BD224BD168D87D014068460170997DE9
:10E99000002922D191681E4B0B409360DFE71B4E8C
:10E9A000B37D002B20D101233375164B194A99688A
:10E9B0000A409A60F27B4F2AC9D199688022D2031B
:10E9C0000A439A60C3E79968134A0A409A609968B3
:10E9D0008022D2020A439A60B1E71868694601AA08
:10E9E000002301F037FDBAE77068694601AA02F01A
:10E9F00061F80128D7D168460378EB60337D002B9E
:10EA0000A5D0D2E70040054004ED00E0F0EDFF1F87
:10EA1000FFFFDFFFFFFF7FFFFFFFBFFF70B500239A
:10EA200082B00193354B80225C68D203144202D03D
:10EA30009968114243D180231B041C4203D02F4DFF
:10EA4000AA681A4227D180239B031C4203D02B4A79
:10EA50009168194211D1294B802259681203114241
:10EA600002D059680A435A60019A002A03D08022D2
:10EA7000234B52051A6002B070BD224BD168D87D7D
:10EA8000014068460170997D002922D191681E4B92
:10EA90000B409360DFE71B4EB37D002B20D1012399
:10EAA0003375164B194A99680A409A60F27B4F2ACF
:10EAB000C9D199688022D2030A439A60C3E7996852
:10EAC000134A0A409A6099688022D2020A439A60E7
:10EAD000B1E71868694601AA002301F0BBFCBAE758
:10EAE0007068694601AA01F0E5FF0128D7D16846A0
:10EAF0000378EB60337D002BA5D0D2E700500540B2
:10EB000004ED00E008EEFF1FFFFFDFFFFFFF7FFFC8
:10EB1000FFFFBFFF70B51E4C8823E558842382B0E9
:10EB2000061CE0580023002200210093022303F07A
:10EB300025F8301CA84702F0FBFE031C201C221CF9
:10EB40007C30002404E082420AD0043200290FD134
:10EB500015680021AB42F6D1146001218242F4D144
:10EB6000002905D10B4804210B4AFAF76BF808E09D
:10EB7000181C02F08FFB0521031C084A0548FAF710
:10EB800061F8FAF7DBF8002002F0D2F902B070BDAC
:10EB900020EEFF1F50580200FC63020018640200C0
:10EBA00008B500F089FF08BD08B5002801D000F0C5
:10EBB000F1FF08BD38B5051C0C1CFFF765FB28608C
:10EBC00001F012F8206038BD08B502F007FD08BD5D
:10EBD00008B502F059FB08BD10B5141C002201F065
:10EBE000A9F9031C20600020002B00D010BD0C20D0
:10EBF000FCE7C04608B5002301F0DCFA0138421EEC
:10EC00009041404216230340181C08BD08B501F08E
:10EC10007BFC0138421E9041404216230340181CE1
:10EC200008BDC046202070471F2803D8024B800033
:10EC3000C05870470020FCE720EEFF1FF0B5564695
:10EC40005F464D464446F0B47A4E1F1C8C239046D6
:10EC5000F25C83B081468A46002A2AD04024002FE5
:10EC600000D0BCB280230121F058494201F006FFD8
:10EC700002F05EFE8423F05052468823F2500C9B33
:10EC80000D9A009301926C48221C4946434602F0BB
:10EC900029F80C24012800D198E08023F05801F0D5
:10ECA000BFFB201C03B03CBC90469946A246AB4635
:10ECB000F0BD01220420F25401F064F98023F050E9
:10ECC00000218022301C03F0B6FC02F0EFFA351C64
:10ECD0008346002405E00134202C18D00435002B95
:10ECE0001DD12A680023002AF5D1584602F0D2FA35
:10ECF0005A46031C0092019450480521504AF9F7E6
:10ED0000A1FF01345B462B600123202CE6D1002BB0
:10ED100005D14A4804214B4A2023F9F793FF03F019
:10ED200039FA00248346434D05E00134202C18D0E5
:10ED30000435002B1DD12A680023002AF5D158463E
:10ED400002F0A8FA5A46031C009201943B480521A0
:10ED50003B4AF9F777FF01345B462B600123202CF7
:10ED6000E6D1002B05D135480421364A2023F9F796
:10ED700069FF02F0DDFD002483462E4D06E00134DC
:10ED8000202C19D00435002B00D067E72A68002317
:10ED9000002AF4D1584602F07DFA5A46031C00922C
:10EDA000019426480521264AF9F74CFF01345B46B9
:10EDB0002B600123202CE5D1002B00D04EE71F480B
:10EDC0000421204A2023F9F73DFF47E70122524260
:10EDD0000020012102F09EFE0D9B184A1F68184B6F
:10EDE000351C00249146984605E00134202C16D0AD
:10EDF0000435002B11D12A680023002AF5D1381CD4
:10EE000002F048FA0097031C019448460521424647
:10EE1000F9F718FF2F600123E7E700243DE7002BF7
:10EE2000FBD106480421074A2023F9F70BFF0024F1
:10EE300033E7C04620EEFF1F15EB010050580200DB
:10EE4000346402005864020038B50C1C2060051CB4
:10EE500002F020FA6060281C02F0FCF8E060281C38
:10EE600002F052FDA060281C02F0C8F8042815D852
:10EE70000C4B80001B589F46532323740023002013
:10EE8000636138BD44232374F8E743232374F5E713
:10EE900052232374F2E742232374EFE755232374AC
:10EEA000ECE7C046E863020008B500F0B5F908BD1C
:10EEB00008B500F0BDF908BD10B5041C042001F030
:10EEC00061F8031C20600020002B00D010BD0C2036
:10EED000FCE7C04608B50121494201F0CFFD08BD5D
:10EEE00008B501F09DFA08BD08B5431E9841C0B2AF
:10EEF000FEF77AFD08BDC04608B5FFF7F5FF08BD6F
:10EF000010B582B0049C009403F0C0F8002804D02F
:10EF1000059B1860002002B010BD0C20FBE7C04626
:10EF200000B5012383B05B4200930521002200233A
:10EF300003F002F9002003B000BDC04600B5012374
:10EF400083B05B420A1C00930421002303F0F4F811
:10EF5000002003B000BDC04610B582B0041C02F012
:10EF600093F901235B42021C0093201C0121002322
:10EF700003F0E2F8002002B010BDC04608B503F06F
:10EF800013F908BD034B04211A698A431A6130BF83
:10EF90007047C04600ED00E0F8B5174B5F464D46A0
:10EFA00044465646F0B41C1D8533FF339B46134B35
:10EFB000E0279A46124B051C9946124BFF009846D3
:10EFC0002668231F1A6851462379281C3E40FCF707
:10EFD00019FB320A4946281CFCF714FB0C34281C88
:10EFE0004146FCF70FFB5C45EAD100203CBC904653
:10EFF0009946A246AB46F8BDA86402002866020006
:10F0000030660200304A0200164AC0239B0030B529
:10F01000136053608023DB00136513495365134865
:10F02000134D144C80235B0003618364C3646B60E5
:10F030008B60CB616361E361136453649367136610
:10F040000B60436083602B604B60CB600B614B6156
:10F050008B612361A361D367AB6000239364D364A6
:10F06000536730BD00D0044000B00440009004401D
:10F0700000A0044000C00440014B02225A647047C3
:10F0800000D00440164AC0239B0030B51360536083
:10F090008023DB001365134953651348134D144C4B
:10F0A00080235B0003618364C3646B608B60CB610E
:10F0B0006361E36113645364936713660B60436099
:10F0C00083602B604B60CB600B614B618B61236174
:10F0D000A361D367AB6000239364D364536730BDEF
:10F0E00000D0044000B004400090044000A0044060
:10F0F00000C0044008B50248FDF772F908BDC046DB
:10F1000080640200002382B00193064B1B68013328
:10F1100001D072B6FEE772B6019B002BFCD002B0A4
:10F120007047C04608E0FF1F00000000000000001C
:10F130000B4A13681868203080F30988022080F396
:10F140001488BFF36F8F3FBCAE4608BC04BC62B6E8
:10F150001847C046C046C046C046C046C046C04626
:10F16000B8EFFF1FC046C046C046C046C046C046B6
:10F1700010B58024031F64041C60043B196003491C
:10F18000043B1960143B40381A6010BD05F10100C2
:10F190007047C046144BFF22196812040A4330B569
:10F1A0001A601968FF2212060A431A600F4B104AB0
:10F1B00000241C600F4914600F4A104D1160072293
:10F1C0001A6083B02C60FFF7B3FF02F01FFA2B68C0
:10F1D0000194013301D072B6FEE772B6019B002B99
:10F1E000FCD0002003B030BD20ED00E010E000E0D6
:10F1F00018E000E07FBB000014E000E008E0FF1F23
:10F20000044B802252051A60BFF34F8FBFF36F8FFC
:10F210007047C04604ED00E072B6044B1A68013234
:10F220001A60BFF34F8FBFF36F8F704708E0FF1F67
:10F23000054A1368002B01D172B6FEE7013B13604B
:10F24000002B00D162B6704708E0FF1FEFF310807B
:10F2500072B6704780F310887047C0460000000007
:10F26000EFF309800E4B1A6820381060F0C0444656
:10F270004D4656465F46F0C008B572B602F0C6F974
:10F2800062B60CBC116808681030F0C8A046A946E8
:10F29000B246BB4680F309882038F0C81847C046FC
:10F2A000B8EFFF1FC046C046C046C046C046C04675
:10F2B00010B5FFF7CBFF041C02F002F8002803D0C2
:10F2C0008022034B52051A60201CFFF7C3FF10BDBC
:10F2D00004ED00E0F0B54F464646C0B4244B254946
:10F2E00000221A600878244AC0B218601478234FAC
:10F2F00024022043224C1860E079224E1871FF232B
:10F300000B700621137089468022042101230120FD
:10F3100090461D4D8C4603E0082B14D00133DBB220
:10F320005A1EE179D2B211410842F5D0012A18D013
:10F33000002A11D0052A0AD0072AEDD1124B10213C
:10F34000DA698A43DA610CBC90469946F0BDEA69F5
:10F3500061468A43EA61E1E7326841460A43326026
:10F36000DCE7FA7849460A43D2B2FA70D6E7C046DB
:10F37000E4EEFF1F05C0074006C00740003007400D
:10F3800000C007400000044000D0034010B50F2823
:10F390000ED80322131C074C0340800800195B00A1
:10F3A00004789A4094439940231C0B43DBB20370CA
:10F3B00010BDC04600C00740072808D8012383407D
:10F3C000181C002904D1054B1A7982431A71704721
:10F3D000024A13791843C0B21071F8E700C0074021
:10F3E00000487047E4EEFF1F80B582B000AF3A4B93
:10F3F0001B687B6021E07B685A1E3749131C5B0049
:10F400009B189B00CB189B68002B13D07B685A1E5F
:10F410003149131C5B009B189B00CB1899687B68D3
:10F420005A1E2D48131C5B009B189B00C3185B6879
:10F43000181C88477B68013B7B607B68002BDAD116
:10F4400001F01AFF254B03229A70244B03225A70B5
:10F45000234B234A126904210A431A611F4B5B782C
:10F46000DBB23B603B68FFF707FE30BF1C4B1C4A1A
:10F47000126904218A431A61FFF704FE01F0FAFFC2
:10F4800000237B6020E014497A68131C5B009B1802
:10F490009B00CB1808335B68002B12D00E497A68AA
:10F4A000131C5B009B189B00CB18083359680A4853
:10F4B0007A68131C5B009B189B00C3185B68181CC0
:10F4C00088477B6801337B60034B1A687B689A42EC
:10F4D000D9D8BD4602B080BDB0EEFF1F00E00740A6
:10F4E00000ED00E0F0B5264A4F464646FF23C0B483
:10F4F0001370244A062113708946802204210123B7
:10F50000214C0120214F224E9046224D8C4603E093
:10F51000082B14D00133DBB25A1EE179D2B211416B
:10F520000842F5D0012A25D0002A1ED0052A17D07E
:10F53000072AEDD1174B1021DA698A43DA61164B9D
:10F5400000221A601A71154BC122920099580902C3
:10F55000090A995080221A600CBC90469946F0BD69
:10F56000EA6961468A43EA61D4E7326841460A4360
:10F570003260CFE7FA7849460A43D2B2FA70C9E757
:10F5800005C0074006C0074000C0074000300740E4
:10F590000000044000D00340E4EEFF1F00E100E063
:10F5A0007047C04638B5FFF737FE01F06DFE0D4AD3
:10F5B0000D491368C41A0D4B1D688C4208D9116897
:10F5C0000948091811601A68FA21890052181A604E
:10F5D000FFF72EFEFA21201C8900F0F77DFD40196F
:10F5E00038BDC046ECEEFF1F40420F00F4EEFF1F97
:10F5F00010B5041CFFF710FE064B1C6001F044FE22
:10F60000054B1860054B1A6801321A60FFF710FEAF
:10F6100010BDC046F4EEFF1FECEEFF1FF0EEFF1F23
:10F62000F8B5FFF7F9FDFFF7F7FD01F02DFE1C4CD3
:10F630001C4A2368C61A1C4B1F68964208D92268C8
:10F640001849521822601A68FA21890052181A6063
:10F65000FFF7EEFDFFF7E0FD01F016FE2368002541
:10F66000C41AFFF7E5FDFA21201C8900F0F778FDA8
:10F670000C1CFA21301C8900F0F72EFD074B064ABE
:10F68000C0190021F0F770FE24184D41FFF7D0FD9E
:10F69000291C201CF8BDC046E80300000000000043
:10F6A000ECEEFF1F40420F00F4EEFF1FC046C046C5
:10F6B00003207047022809D8054A012312688340B5
:10F6C0001A4203D0034B8000C05870470020FCE76B
:10F6D000F8EEFF1F8066020038B5054D002428595A
:10F6E000043403681B6898470C2CF8D1002038BDFF
:10F6F0008066020070B5041C0D1C022803D900238B
:10F700000B60132070BD084B8200D6583368301C44
:10F710005B689847054B0122A240141C1A682E60B2
:10F7200014431C60EEE7C04680660200F8EEFF1F3F
:10F7300030B583B0069D04680095E468A04703B027
:10F7400030BDC04630B583B0069D0468009524697D
:10F75000A04703B030BDC04608B503685B69984751
:10F7600008BDC04608B503689B69984708BDC046F8
:10F770007047C04610B50E490E4C8C4208D00E4A58
:10F78000920803D09200201C02F033FF0B4B9C60C8
:10F790000B490C4A521A02D00B4802F02AFF0B48C0
:10F7A0000B4A121A02D0002102F045FF10BDC046DC
:10F7B00000000000000000000000000000ED00E07C
:10F7C0006C690200606A020000E0FF1FF4E0FF1FA6
:10F7D000F0F6FF1F7047C046FEF796F8FFF7FAFFF6
:10F7E000FEF7B8F8FFF7C6FFF0F73AFCFEE7C046B1
:10F7F00038B5051C1820FFF7D3F9041E0BD0281CC0
:10F80000FFF7CEF9011E08D0201C2A1CFBF74CFA8A
:10F81000002363612361201C38BD0020FFF7C4F979
:10F82000201CFFF7C1F90024F5E7C046F0B54746B4
:10F8300080B4041C82B08846171C1E1CFFF7ECFC29
:10F84000201C41463A1CFBF735FA051E0FD1002E4D
:10F8500020D02369002B20D0FFF7EAFC012001F023
:10F86000BDFE731CEAD0013E002EE7D10DE06669B3
:10F87000002E0FD000276761FFF7DAFC0097301CDD
:10F8800000210022022302F079F9281C02B004BCF6
:10F890009046F0BDFFF7CCFCF7E702F049F8206195
:10F8A000FFF7C6FC321C0020012102F033F9431E91
:10F8B0009841404206402561D6E7C046F0B547462C
:10F8C00080B4041C82B08846171C1E1CFFF7A4FCE1
:10F8D000201C41463A1CFBF739FA051E0FD1002EB9
:10F8E00020D06369002B20D0FFF7A2FC012001F09B
:10F8F00075FE731CEAD0013E002EE7D10DE02669AB
:10F90000002E0FD000272761FFF792FC0097301CD4
:10F9100000210022022302F031F9281C02B004BCAD
:10F920009046F0BDFFF784FCF7E702F001F8606154
:10F93000FFF77EFC321C0020012102F0EBF8431E91
:10F940009841404206406561D6E7C04670B582B036
:10F950000D1C124C061CF6F745FD83235B01E35892
:10F9600001A904220193F6F743FD0D4B01A9E358C9
:10F9700004220193F6F73CFD0A4B01A9E358042247
:10F980000193F6F735FDF6F731FD291C031C064AF5
:10F99000301CFDF703FB02B070BDC0460070044090
:10F9A0005C10000058100000902D0200FEE7C046D9
:10F9B0007047C0467047C0464368083305C905C351
:10F9C0000020704710B54368083311CB11C10020E7
:10F9D00010BDC046406808B54068FFF727FF029B8E
:10F9E0001860002008BDC04610B54368141C0029EB
:10F9F0000CD0012901D0162010BD58681168E368A9
:10FA00005268FFF75BFFA0600020F5E718681168F7
:10FA1000E3685268FFF70AFFA0600020ECE7C046E9
:10FA2000406808B50068FFF749FF029B1860002096
:10FA300008BDC04638B54468051C2368002B0ED0AD
:10FA40006368002B05D0201C0830FBF7EDFA00207E
:10FA500038BDE868FFF7CCFE60606C68F3E780684B
:10FA6000FFF7C6FE20606C68EAE7C04610B5104A92
:10FA70001368834201D21A1CFAE751685418844271
:10FA800003D1406841185160101C41684418A342DA
:10FA900009D1084C2468A34205D05C681B68611832
:10FAA0004160036000E00360824200D0106010BD3E
:10FAB00018EFFF1F14EFFF1FF8B54F464646C0B4BE
:10FAC0002E4F041C386800284FD001F0D5FB2C4B7A
:10FAD00000251E68311C214040D1002C3ED0231C43
:10FAE00008330D1C9C4239D207221A4206D0181C3A
:10FAF0009043021C0832934230D2131C0025002B85
:10FB00002CD020490A6888469146934226D81E493F
:10FB10000C6804E02068002804D0211C041C6268E2
:10FB20009342F7D838680025844217D02068251CF6
:10FB300008600835D11A102919D849468B1A13497B
:10FB4000404603600868834200D20B6000232360B4
:10FB50000F4B324362601A6801321A6001F08AFC6E
:10FB6000281C0CBC90469946F8BD72B6FEE7E0181A
:10FB700041606360FFF77AFF6268DEE714EFFF1F02
:10FB800028EFFF1F10EFFF1F18EFFF1F24EFFF1FCD
:10FB90000CEFFF1F10B500281FD0041C0F4A083CB3
:10FBA00063681268134201D172B6FEE7206800282C
:10FBB00001D072B6FEE79343636001F05DFB084B32
:10FBC000606819680A18201C1A60FFF74FFF054B80
:10FBD0001A6801321A6001F04DFC10BD28EFFF1FBA
:10FBE00010EFFF1F20EFFF1F014B18687047C04642
:10FBF00010EFFF1FF0B54D465F4656464446F0B441
:10FC0000374D83B02B68002B01D072B6FEE74268F7
:10FC1000002A45D00727061CBB46324F0836002471
:10FC200001960021061CA1460020B84633685E46B6
:10FC30001E4204D0DF1DB743DB1BD2183B1C00283B
:10FC40001DD1D218083A5F46BA4346467060336009
:10FC5000D61A50601060B4465E601A609246002961
:10FC600000D00B60019E6444371C08373A1C043AEC
:10FC7000126801300197002A18D05146D6E70029B2
:10FC80002AD0994225D2D2185E46083AB2434F464E
:10FC9000D61A57601760B4465E601A609246E0E775
:10FCA000114B1A60114B1A6072B6FEE753462B6077
:10FCB0000D4B1C600D4B1C60002CF5D00C4B8022B2
:10FCC00012061A6003B03CBC90469946A246AB4669
:10FCD000F0BD296072B6FEE7296072B6FEE7C04645
:10FCE00014EFFF1F18EFFF1F24EFFF1F10EFFF1F80
:10FCF00028EFFF1F031C0833012243605242C360F8
:10FD000003610023826003607047C04600230361E3
:10FD10007047C04643689A684B608A609A68516031
:10FD200099600368086101330360704730B50C685F
:10FD3000021C0832631C01D10DE01A1C53681D68B7
:10FD4000AC42FAD24B60996003688A60013351601B
:10FD50000861036030BD02695368F3E74268816857
:10FD60000369916081684A605A68824206D0002225
:10FD700002611A68013A1A60186870475960F6E71C
:10FD800070B5161C026C041C856B002A08D106682D
:10FD9000101C002E29D1A06801F02AFEA66024E0E4
:10FDA000002E0DD1406802F024FC6168226C301CEA
:10FDB0008B18A16863608B4217D32268626014E0DD
:10FDC000C06802F016FC236CE1685A428B18216867
:10FDD000E3608B4202D2A3689A18E2600020022EF0
:10FDE00003D12B1C5A1E9341ED1A0135A56370BD3A
:10FDF000026C10B5002A0CD0C468A3188468C360D4
:10FE0000A34201D30368C360C368081C191C02F035
:10FE1000F0FB10BD70B5051CFFF7FEF94523EC5C47
:10FE2000E4B263B2002B17DD6B6A002B14D02E1CDA
:10FE3000243606E0013CE4B2002C0DD06B6A002BA6
:10FE40000AD0301C01F0B4FC0028F3D0013CE4B22D
:10FE500001F054FD002CF1D14523FF22EA54FFF7B5
:10FE6000E7F9FFF7D9F94423EC5CE4B263B2002B65
:10FE700017DD2B69002B14D02E1C103606E0013C38
:10FE8000E4B2002C0DD02B69002B0AD0301C01F0FD
:10FE90008FFC0028F3D0013CE4B201F02FFD002CD0
:10FEA000F1D1FF224423EA54FFF7C2F970BDC046E6
:10FEB00038B5041C0D1C00280BD0C16B002906D0DE
:10FEC00001204042F0F708F9216C884203D272B653
:10FED000FEE772B6FEE7FFF79FF9226CE06B23683E
:10FEE0005043821A191863609B18A160E360442292
:10FEF000FF230021A163A3544522A354002D06D162
:10FF00002369002B0CD1FFF793F9012038BD201C89
:10FF10001030FFF7EFFE201C2430FFF7EBFEF2E776
:10FF2000201C103001F044FC0028ECD0FFF768F9E9
:10FF3000E9E7C04670B5061C0D1C00280BD0012057
:10FF40004042311CF0F7C8F8A84204D3281C704383
:10FF5000031C493301D972B6FEE74830FFF7ACFD08
:10FF6000041E0CD0021C4832031C002D00D0131CB0
:10FF70002360E6632564201C0121FFF799FF201C04
:10FF800070BDC046F0B557464E464546E0B44820E1
:10FF900084B0FFF791FD041E00D1A8E000250123E5
:10FFA00020600121C3630564FFF782FF226C256096
:10FFB000A560E5600195002A00D0F3E001F0BEFCE9
:10FFC000002800D1F0E000274426B8464525FFF779
:10FFD00023F9A36BE26B934277D3019B002B00D1F3
:10FFE00083E0002F02D102A801F04CFCFFF720F9BA
:10FFF00001F042F9FFF710F9A35D5BB2013301D1C3
:020000022000DC
:100000004246A255635D5BB2013301D1434663555D
:10001000FFF70EF902A801A901F040FC002800D06A
:10002000B7E0FFF7F9F8A36BE26B934266D0FFF7F6
:10003000FFF8FFF7F1F8675DFFB27BB2002B18DD28
:10004000636A002B15D024231B19994606E0013F53
:10005000FFB2002F0DD0636A002B0AD0484601F092
:10006000A7FB0028F3D0013FFFB201F047FC002FAF
:10007000F1D1FF236355FFF7DBF8FFF7CDF8A75D5C
:10008000FFB27BB2002B18DD2369002B15D01023A3
:100090001B19994606E0013FFFB2002F0DD02369DE
:1000A000002B0AD0484601F083FB0028F3D0013F23
:1000B000FFB201F023FC002FF1D1FF23A355FFF77E
:1000C000B7F801F0D7F9012781E7201C00210022B1
:1000D000FFF756FE636A002B03D0201C243001F08A
:1000E00067FB002801D0FFF78BF8FFF7A1F8201C71
:1000F00004B01CBC90469946A246F0BDFFF798F8A4
:1001000010221219101C0199914601F0D7FAFFF73D
:1001100083F8675DFFB27BB2002B18DD636A002BAA
:1001200015D024231B199A4606E0013FFFB2002F89
:100130000DD0636A002B0AD0504601F039FB00282D
:10014000F3D0013FFFB201F0D9FB002FF1D1FF2323
:100150006355FFF76DF8FFF75FF8A75DFFB27BB25D
:10016000002B0BDD2369002B08D0484601F020FB53
:10017000002814D1013FFFB2002FF3D1FF23A35574
:10018000FFF756F801F076F900289CD1FFF738F810
:1001900099E7201CFFF73EFE01F06CF9A7E701F09C
:1001A000ADFBE7E772B6FEE7019B002B00D10AE743
:1001B00072B6FEE7F0B544464D465F465646F0B48B
:1001C00085B0041C89460192984600D1F8E00029C8
:1001D00000D11EE14246022A00D114E101F0AEFB3B
:1001E000002800D1EEE0FFF717F8A36BE26B0027C1
:1001F0004426BA46452593427BD34346022B78D00A
:10020000019A002A00D1FAE0002F00D1F3E0FFF7B5
:100210000FF801F031F8FEF7FFFFA35D5BB2013389
:1002200000D1E5E0635D5BB2013300D1DDE0FEF7B4
:10023000FFFF02A801A901F031FB002800D0C7E0B0
:10024000FEF7EAFFA36BE26B934266D0FEF7F0FF86
:10025000FEF7E2FF675DFFB27BB2002B18DD636A39
:10026000002B15D024231B199B4606E0013FFFB24B
:10027000002F0DD0636A002B0AD0584601F098FA7F
:100280000028F3D0013FFFB201F038FB002FF1D17D
:10029000FF236355FEF7CCFFFEF7BEFFA75DFFB25D
:1002A0007BB2002B18DD2369002B15D010231B19FE
:1002B0009B4606E0013FFFB2002F0DD02369002BC3
:1002C0000AD0584601F074FA0028F3D0013FFFB27B
:1002D00001F014FB002FF1D1FF23A355FEF7A8FF77
:1002E00001F0C8F80127FEF797FFA36BE26B93427A
:1002F00083D2201C49464246FFF742FD636A002B29
:1003000003D0201C243001F053FA002801D0FEF75E
:1003100077FFFEF78DFF012060E0FEF789FF1023D5
:100320001B19181C01999B4601F0C8F9FEF774FFD0
:10033000675DFFB27BB2002B18DD636A002B15D01E
:10034000221C2432009206E0013FFFB2002F0DD0A4
:10035000636A002B0AD0009801F02AFA0028F3D033
:10036000013FFFB201F0CAFA002FF1D1FF2363551C
:10037000FEF75EFFFEF750FFA75DFFB27BB2002BDA
:1003800004DC11E0013FFFB2002F0DD02369002BE8
:100390000AD0584601F00CFA0028F3D0013FFFB212
:1003A00001F0ACFA002FF1D1FF23A355FEF740FF77
:1003B00001F060F8002895D1FEF722FF012792E7AF
:1003C00072B6FEE7019B002B00D10CE772B6FEE788
:1003D000201CFFF71FFD01F04DF8002005B03CBCCC
:1003E00090469946A246AB46F0BD524662551EE77E
:1003F0005346A35516E702A801F044FA07E7FEF7B3
:1004000017FF0020EAE7E26B012A00D1E6E672B6A8
:10041000FEE7036C002B00D1DCE672B6FEE7C046B7
:1004200070B5041E07D0866801F082FA0025864266
:1004300003D0281C70BD72B6FEE7E3680125013BBE
:10044000E360002BF5D1201C00210022FFF7B2FE53
:10045000EFE7C046F0B5454657464E46E0B4041CAB
:100460000D1C171C9846002815D0002936D043468D
:10047000022B2ED0FEF7EAFEA36BE26B061C934222
:100480000FD30025301CFEF7E5FE281C1CBC90464F
:100490009946A246F0BD72B6FEE7FEF7D7FEA36B03
:1004A000061C4522A35C9146DBB29A464246201CBC
:1004B000291CA36BFFF764FC524653B25A1C14D09C
:1004C0007F2B10D053460133DBB24A46A35401259B
:1004D000D8E7E36B012BE0D072B6FEE7026C002A8E
:1004E000C5D072B6FEE772B6FEE7636A0125002B3F
:1004F000C8D0201C243001F05BF90028C2D0002FA6
:10050000C0D03D60BEE7C046F0B5454657464E46B2
:10051000E0B484B0041C8846019200D142E1002975
:1005200000D150E101F00AFA002800D13CE100239B
:100530009A469946FEF770FEA76B44264525002F84
:1005400000D022E1019B002B00D133E15346002B68
:1005500002D102A801F096F9FEF76AFE00F08CFEC7
:10056000FEF75AFEA35D5BB2013301D14B46A355A2
:10057000635D5BB2013301D14B466355FEF758FE14
:1005800002A801A901F08AF9002800D0A4E0FEF732
:1005900043FEA36B002B52D1FEF74AFE24231B1906
:1005A000181C01999A4601F089F8FEF735FE675D3F
:1005B000FFB27BB2002B04DC11E0013FFFB2002F41
:1005C0000DD0636A002B0AD0504601F0F1F80028E4
:1005D000F3D0013FFFB201F091F9002FF1D1FF23D9
:1005E0006355FEF725FEFEF717FEA75DFFB27BB24F
:1005F000002B18DD2369002B15D010231B199A46F8
:1006000006E0013FFFB2002F0DD02369002B0AD076
:10061000504601F0CDF80028F3D0013FFFB201F0C1
:100620006DF9002FF1D1FF23A355FEF701FE00F075
:1006300021FF002800D0A0E0FEF7E2FD9DE0FEF7DC
:10064000F7FDFEF7E9FD675DFFB27BB2002B18DD19
:10065000636A002B15D024231B199A4606E0013F3C
:10066000FFB2002F0DD0636A002B0AD0504601F074
:100670009FF80028F3D0013FFFB201F03FF9002FAF
:10068000F1D1FF236355FEF7D3FDFEF7C5FDA75D4E
:10069000FFB27BB2002B18DD2369002B15D010238D
:1006A0001B199A4606E0013FFFB2002F0DD02369C7
:1006B000002B0AD0504601F07BF80028F3D0013F10
:1006C000FFB201F01BF9002FF1D1FF23A355FEF774
:1006D000AFFD00F0CFFE50E0FEF79EFD675DFFB27C
:1006E0007BB2002B18DD636A002B15D024231B1965
:1006F0009A4606E0013FFFB2002F0DD0636A002B3F
:100700000AD0504601F054F80028F3D0013FFFB260
:1007100001F0F4F8002FF1D1FF236355FEF788FDB7
:10072000FEF77AFDA75DFFB27BB2002B18DD2369CF
:10073000002B15D010231B199A4606E0013FFFB28B
:10074000002F0DD02369002B0AD0504601F030F85D
:100750000028F3D0013FFFB201F0D0F8002FF1D113
:10076000FF23A355FEF764FD00F084FEFEF754FD61
:10077000A36B002B1ED0FEF75BFD01239A46FEF70C
:100780004BFDA76B002F00D1DCE6201C4146013F4A
:10079000FFF72EFBA7632369002B1AD1FEF748FD54
:1007A00001200AE072B6FEE7019B002B00D1BEE6F5
:1007B00072B6FEE7FEF73CFD002004B01CBC90467C
:1007C0009946A246F0BD036C002B00D1AAE672B692
:1007D000FEE7201C103000F0EBFF0028DED0FEF713
:1007E0000FFDDBE7F0B557464E464546E0B484B012
:1007F000041C019104D0036C002B03D072B6FEE7F9
:1008000072B6FEE701F09AF8002803D1019B002B95
:1008100000D01DE100239846FEF7FEFCA36B0027E5
:100820004426B9464525002B00D083E0019B002BD0
:1008300000D1EBE0002F02D102A801F023F8FEF76F
:10084000F7FC00F019FDFEF7E7FCA35D5BB2013396
:1008500001D14B46A355635D5BB2013301D14B46D9
:100860006355FEF7E5FC02A801A901F017F800287E
:1008700079D1FEF7D1FCA36B002B6BD1FEF7D8FC2E
:100880002368002B00D1EFE024231B19181C0199C9
:100890009A4600F013FFFEF7BFFC675DFFB27BB224
:1008A000002B04DC11E0013FFFB2002F0DD0636A82
:1008B000002B0AD0504600F07BFF0028F3D0013F08
:1008C000FFB201F01BF8002FF1D1FF236355FEF7B3
:1008D000AFFCFEF7A1FCA75DFFB27BB2002B18DDD9
:1008E0002369002B15D010231B199A4606E0013FFF
:1008F000FFB2002F0DD02369002B0AD0504600F024
:1009000057FF0028F3D0013FFFB200F0F7FF002FA0
:10091000F1D1FF23A355FEF78BFC00F0ABFD0028BF
:1009200001D1FEF76DFC0127FEF776FCA36B002BCF
:1009300000D17BE7013BA3632368002B02D101F0C8
:10094000DDF8A0602369002B00D083E0FEF770FC87
:10095000012070E0FEF76CFC201CFFF75BFA01271A
:1009600000F088FDE0E7FEF757FC675DFFB27BB261
:10097000002B18DD636A002B15D024231B199A461F
:1009800006E0013FFFB2002F0DD0636A002B0AD0B2
:10099000504600F00DFF0028F3D0013FFFB200F0F9
:1009A000ADFF002FF1D1FF236355FEF741FCFEF7A9
:1009B00033FCA75DFFB27BB2002B18DD2369002B4F
:1009C00015D010231B199A4606E0013FFFB2002FF5
:1009D0000DD02369002B0AD0504600F0E9FE002814
:1009E000F3D0013FFFB200F089FF002FF1D1FF23C8
:1009F000A355FEF71DFC00F03DFDFEF70DFCA36BBB
:100A0000002B1ED0FEF714FC01278DE74346002B78
:100A10000ED072B6FEE7FEF7FFFB636A0021002BE3
:100A200003D0236B04211B68C91AA06801F01EF8CB
:100A3000FEF7FEFB002004B01CBC90469946A2467F
:100A4000F0BDFEF7F5FB4346002BE4D10020F2E7B2
:100A500072B6FEE7201C103000F0AAFE002800D17C
:100A600074E7FEF7CDFB71E7FEF7D6FBA06800F058
:100A700075FF8046FEF7DCFB06E7C04670B5041C38
:100A80000D1C002813D0866800F052FF864209D062
:100A9000201C291CFFF7A6FE002802D0E3680133C2
:100AA000E36070BDE36801200133E360F9E772B6EB
:100AB000FEE7C046F0B557464E464546E0B4041C36
:100AC0000E1C171C002827D000293BD0FEF7BEFBC8
:100AD000A56B8246002D33D044239846E35C201C4E
:100AE000DBB29946311CFFF783F94A46013D53B208
:100AF000A5635A1C12D07F2B15D04B460133DBB2B5
:100B00004246A35401245046FEF7A4FB201C1CBC03
:100B100090469946A246F0BD72B6FEE72369002BC7
:100B200003D10124EFE772B6FEE7201C103000F07D
:100B30003FFE0028F5D0002FF3D001233B60F0E703
:100B40000024E0E7026C002AC0D072B6FEE7C0467F
:100B500070B5051C141C0E1CFEF75EFB4423EA5CFA
:100B600052B201325DD04523E85C40B2013055D02D
:100B7000FEF75EFBAB6B002B05D1281C2430311C2B
:100B8000221C00F0CFFDFEF747FB4523EC5CE4B2EE
:100B900063B2002B17DD6B6A002B14D02E1C243699
:100BA00006E0013CE4B2002C0DD06B6A002B0AD0A9
:100BB000301C00F0FDFD0028F3D0013CE4B200F051
:100BC0009DFE002CF1D14523FF22EA54FEF730FBB5
:100BD000FEF722FB4423EC5CE4B263B2002B17DD8A
:100BE0002B69002B14D02E1C103606E0013CE4B219
:100BF000002C0DD02B69002B0AD0301C00F0D8FD42
:100C00000028F3D0013CE4B200F078FE002CF1D1D2
:100C1000FF224423EA54FEF70BFB70BD0022EA5486
:100C2000A6E70022EA549EE7F0B5144A474680B48E
:100C3000134E144F144D904614E0FEF7EDFAFB6886
:100C4000DC68201DFFF78AF83368013B33602B68AE
:100C5000013B2B60FEF7ECFA206BFEF79BFF201C9C
:100C6000FEF798FF2B68002BE7D142461368012B53
:100C700001D9FEF7C5FAFEF785F9F3E764EFFF1F28
:100C8000FCEFFF1F38EFFF1FF8EFFF1F70B5104B91
:100C9000104C1E68051C2068AD190430FFF75EF883
:100CA00023685D60AE420BD80B4B18682168043195
:100CB000FFF73CF8094B1A68954200D21D6070BDE1
:100CC000074B186821680431FFF730F8F7E7C04692
:100CD000C4EFFF1FB8EFFF1F30EFFF1FBCEFFF1F78
:100CE000C8EFFF1FF8B592005F4656464D46444692
:100CF000F0B48246101C0D1C99460A9E9346FEF7DE
:100D0000DBFE071E00D1B2E05C20FEF7D5FE041E1C
:100D100000D1A9E05A460763A521381C01F08BFCDD
:100D20005B46206B043BC318072293439B46002D70
:100D300000D1BBE02A783423E2540023EB56002B89
:100D400025D06A783523E2540123EB56002B1ED0C0
:100D5000AA783623E2540223EB56002B17D0EA7808
:100D60003723E2540323EB56002B10D02A79382383
:100D7000E2540423EB56002B09D06A793923E2545C
:100D80000523EB56002B02D0AA793A23E254002225
:100D90003B23E254032E01D972B6FEE70025211D44
:100DA000081CE662E66325648846FEF7AFFF201C58
:100DB0001830FEF7ABFF04239E1B201C00211022DD
:100DC0002461A6616462443001F035FC231C543375
:100DD0004A461D705D709D70DD701D71584651460C
:100DE000FEF7C6F90B9A2060002A00D01460FEF7C7
:100DF00013FA434B434E1A6801321A603268002AD4
:100E00004CD0414F3B68002B3AD13268E36AD26A3A
:100E10009A4241D83D4A346011683D4D013111601C
:100E20003C4A1168994235D39A00D3189B00E918BF
:100E30004A689C4693684046E3609368A2605860A5
:100E4000906060462A58616101322A50FEF7F0F93D
:100E50003B680125002B0CD03368DA6AE36A9A42BA
:100E600007D2FEF7CDF904E0381CFEF793FE01250A
:100E70006D42281C3CBC90469946A246AB46F8BD44
:100E8000E36A234D214A116801311160214A11683A
:100E90009942C9D21360C7E71D4DF3E734601B6860
:100EA000012B06D0E36A1A4D174FEBE73423E554C4
:100EB00070E7174D281CFEF71DFF281C1430FEF7A5
:100EC00019FF281C2830FEF715FF281C3C30FEF7C0
:100ED00011FF114B181C9946FEF70CFF0F4F381CE1
:100EE000FEF708FF0E48FEF705FF0E48FEF702FF6B
:100EF0000D4B484618600D4B1F60E36A024FC1E777
:100F0000FCEFFF1FB8EFFF1F34EFFF1FE0EFFF1FE5
:100F100064EFFF1F00F0FF1FE4EFFF1F4CEFFF1F08
:100F2000CCEFFF1F38EFFF1F30EFFF1FC8EFFF1F91
:100F300070B5041CFEF770F9274D002C37D0261D24
:100F4000301CFEF70BFFA26A002A03D0201C1830C9
:100F5000FEF704FF214B1A6801321A602B689C428D
:100F600027D01F4B1A68013A1A601E4B1A68126884
:100F7000002A16D101221C4B52421A60FEF758F982
:100F80002B689C4205D0206BFEF704FE201CFEF768
:100F900001FE164B1B68002B02D02B689C4211D01F
:100FA00070BD1B68DB681A680F4B1A60E6E72C6897
:100FB000C5E70F48311CFEF7ADFE0E4B1A68013233
:100FC0001A60DBE70C4B1B68002B01D072B6FEE702
:100FD000FEF716F9E4E7C046B8EFFF1FE0EFFF1F8A
:100FE000FCEFFF1F30EFFF1FBCEFFF1F34EFFF1FB1
:100FF00038EFFF1FF8EFFF1FB4EFFF1F70B5041E9F
:101000001DD0104B1B68984217D0FEF705F90E4B08
:1010100064691E680D4B1D68FEF70AF9B44208D0DA
:10102000AC4206D00A4B9C4205D00120002C02D0D5
:1010300070BD0220FCE70420FAE70020F8E772B652
:10104000FEE7C046B8EFFF1F30EFFF1FC8EFFF1FDE
:1010500038EFFF1F10B5041CFEF7DEF8201E04D089
:10106000C46AFEF7E5F8201C10BD014B1868F7E7CD
:10107000B8EFFF1FF8B580204F464646C0B4400089
:10108000FEF71AFD051E00D193E05C20FEF714FD6B
:10109000041E00D199E08022A52105635200281C7E
:1010A00001F0C9FA266B0723FC369E4349223423FC
:1010B000E25444223523E2544C223623E2544522A2
:1010C00037230025E2543823E5543B23E554201D03
:1010D000E562E56325648046FEF718FE201C1830A3
:1010E000FEF714FE0423201CA361002110222461BA
:1010F0006462443001F09FFA231C543300221D70B7
:101100005D709D70DD701D714A49301CFEF730F82E
:10111000494B20601C60FEF77FF8484B484F1A6827
:1011200001321A603A68002A54D0464E3368002BC8
:1011300041D0E36A444D454A116801311160444A87
:101140001168994200D213609A00D3189B00E918E5
:101150004A689C4693684046E3609368A260586082
:10116000906060462A58616101322A50FEF760F8AB
:101170003368002B06D03B68DA6AE36A9A4201D2F0
:10118000FEF73EF800F040FF012810D172B6314B57
:10119000012252421A60304B002230601A60FDF783
:1011A000F9FF2E4B1B680CBC90469946F8BD0130E8
:1011B000F7D172B6FEE73A68E36AD26A9A4202D879
:1011C0003C60214DB7E7204DB5E7281CFEF7E2FC57
:1011D00072B6EFE73C601B68012B03D0E36A1A4D3F
:1011E000184EA8E7184D281CFEF784FD281C143063
:1011F000FEF780FD281C2830FEF77CFD281C3C30C3
:10120000FEF778FD1649081C8946FEF773FD154E5A
:10121000301CFEF76FFD1448FEF76CFD1348FEF717
:1012200069FD134B4A461A60124B1E60E36A054E75
:1012300081E7C046290C0200C0EFFF1FFCEFFF1F33
:10124000B8EFFF1F34EFFF1F64EFFF1FE0EFFF1F3A
:1012500000F0FF1FBCEFFF1FC4EFFF1F0CE0FF1FDC
:10126000E4EFFF1F4CEFFF1FCCEFFF1F38EFFF1F16
:1012700030EFFF1FC8EFFF1F024B1A6801321A60E0
:101280007047C046B4EFFF1F014B18687047C04657
:10129000C4EFFF1F002801D034307047024B18689C
:1012A0000028F9D172B6FEE7B8EFFF1F034B1868AC
:1012B000002800D0704772B6FEE7C046C0EFFF1F9F
:1012C000F0B55F4656464D464446F0B45E4B83B09B
:1012D0001B68002B72D15D4B1D6801351D60002D10
:1012E00063D05B4A136800249D4200D275E05948E0
:1012F000594B5A4E5A4982469C46B04601959146F2
:10130000504603681B68002B4AD00368019DDB68C8
:10131000DB685868854200D28CE0D8689E685A69BC
:10132000B060D86855681F1D4660BD4244D0106843
:10133000002601385E6110609A6A002A0ED0DE69CC
:10134000186A1D1CB060186A183546605668AE42AF
:101350005CD0002098621068013810604546D86A59
:101360002A68904200D928608200121892009346A1
:101370008A185668B5689E60DD60B5686F60B760B2
:101380005E465A618B59624601338B511368DB6AA2
:101390009842B5D35046036801241B68002BB4D192
:1013A00001234A465B4213601AE02A4B1A6812680E
:1013B000002A2DD072B6FEE75060B8E7294B002412
:1013C0001A6801321A60F2F791FF201C03B03CBC8E
:1013D00090469946A246AB46F0BD1F4B20499C461D
:1013E00065462B68DB6A9A00D3189B00CB58012B0B
:1013F00000D901241B4B1B68002B01D1F2F776FFAB
:10140000194B1B68002BE0D00124DEE75060A0E7F9
:10141000164A1968106818601160154A1168013180
:1014200011601A681268002A07D1094A01235B4239
:10143000136057E74A461060D2E71B68044ADB682E
:101440001B6813604EE7C046B4EFFF1FC4EFFF1FD9
:10145000BCEFFF1F30EFFF1FB8EFFF1F00F0FF1FB3
:1014600064EFFF1F60EFFF1F04F0FF1FC8EFFF1FB7
:101470002CEFFF1FF8B544465F4656464D46F0B484
:101480004C4C2368002B01D172B6FEE7FDF7C4FE79
:101490002368013B23602368002B72D1464B1B68F5
:1014A000002B6ED04549464D464E0023464C4748DA
:1014B00089469846AC46B3464F463A68002A44D01F
:1014C0004F46FB68DB68D9691D6A9A6A8D60196AA4
:1014D000DE691D1C576818354E60AF425DD041462D
:1014E00099621168013911609D68DE685A69AE60C1
:1014F000D96857684D601D1DAF424CD041465961B7
:1015000011686646013911603168DA6A8A4200D989
:101510003260910089188E0087197968BA468F6801
:101520009960DF608F687D608D6051465961815997
:101530005D46013181512968C96A8A42BCD30126BE
:1015400026604F463A68002ABAD1002B08D0204BBB
:101550001A681268002A22D101221E4B52421A60D8
:101560001D4E3568002D09D00127FFF7A9FE002880
:1015700000D02760013D002DF7D135602368002B96
:1015800013D10024FDF754FE201C3CBC9046994624
:10159000A246AB46F8BD5160B0E751609FE71B68BB
:1015A000DB681A680B4B1A60DAE7FDF729FE0124A5
:1015B000E8E7C046B4EFFF1FFCEFFF1FCCEFFF1FB3
:1015C00000F0FF1FB8EFFF1F04F0FF1F64EFFF1FC5
:1015D00030EFFF1FBCEFFF1F60EFFF1F08B50028B3
:1015E0000ED0094B1A68002A01D072B6FEE71A68BD
:1015F00001321A60FFF74AFBFFF73CFF002801D1D8
:10160000FDF7FEFD08BDC046B4EFFF1F264B10B529
:101610001B68002B41D1254A2548136002682549E3
:1016200093009C18A4000C59002C27D1002A21D02B
:10163000531E9C00E418A4006458002C1CD1002BFD
:1016400018D0931E9C00E418A4006458002C13D1F9
:10165000002B0FD0D31E9C00E418A4006458002C6B
:101660000AD1002B06D0131F9A00D21892005258AC
:10167000002A01D172B6FEE71A1C9B009B189B0042
:10168000C9184B680C1C5B6808344B60A34208D037
:10169000D968094B1960026010BD044B01221A6021
:1016A000FAE75B684B60F3E7B4EFFF1F04F0FF1F3E
:1016B00000F0FF1F64EFFF1FB8EFFF1F70B50D1C98
:1016C000002822D0124C21681831FEF72FFB114B55
:1016D0001E682068AD190430FEF740FB23685D608A
:1016E000AE420BD80C4B186821680431FEF71EFB84
:1016F0000A4B1A68954200D21D6070BD084B1868ED
:1017000021680431FEF712FBF7E772B6FEE7C04628
:10171000B8EFFF1FC4EFFF1F30EFFF1FBCEFFF1F2D
:10172000C8EFFF1F70B50D1C002834D01B4C436858
:1017300021689E68CB6121680E6226689968183618
:101740004E602168183199602368986203680133FC
:101750000360002A01D001256D42114B1E682068EC
:10176000AD190430FEF7FAFA23685D60AE420BD87B
:101770000C4B186821680431FEF7D8FA0A4B1A6836
:10178000954200D21D6070BD084B18682168043175
:10179000FEF7CCFAF7E772B6FEE7C046B8EFFF1FD8
:1017A000C4EFFF1F30EFFF1FBCEFFF1FC8EFFF1F8D
:1017B000C368F0B5DB68002B54D0D869196A9A6AFF
:1017C0008160196A54684860181C1830844247D0F8
:1017D00000219962116801391160244A1268002AB7
:1017E0002ED19868DF685A698760D9681D1D4860E6
:1017F0005068A84238D00021596111680139116040
:101800001B49DA6A0868824228D89000194C80186F
:101810008000261871688F689960DF608F687D602E
:101820008D605E61235801332350134B00201B68E9
:10183000DB6A9A4203D9114B01221A600120F0BDE4
:101840000F4A51688C68D9611C628C68606088603E
:1018500011689A6201311160DA6AE6E70A60D4E73A
:101860005160B5E772B6FEE75160C4E7B4EFFF1F01
:1018700000F0FF1F64EFFF1FB8EFFF1F04F0FF1F12
:10188000CCEFFF1F034B1B680360034B1B684360D7
:101890007047C0462CEFFF1FC4EFFF1FF8B5041CB4
:1018A0000D1C002823D000291FD0FDF7B5FC114BDB
:1018B000114A1E6817686068BC462768311A674578
:1018C00001D0864202D22868814206D300232B60D1
:1018D0000124FDF7ADFC201CF8BD12681B68411AFD
:1018E0002960226063600024F3E772B6FEE772B6F7
:1018F000FEE7C046C4EFFF1F2CEFFF1F014B012284
:101900001A60704704F0FF1F00280BD0026B002004
:101910001378A52B05D10130135CA52BFBD08003D8
:10192000000C7047014B1868F0E7C046B8EFFF1F86
:10193000014B18687047C046B8EFFF1F054B0120E8
:101940001B68002B04D0044B1868434258414000E8
:101950007047C04634EFFF1FB4EFFF1FF8B5041EF9
:1019600021D0204DC36A2A68D26A934214D280697A
:10197000002804DB2A680421D26A8A1AA2619A002C
:10198000D318194E9B006269F3189A420DD02B6848
:101990000120DB6AE36205E02B68C06BDB6A9842DA
:1019A00080414042F8BD0020FCE7271D381CFEF7AF
:1019B000D5F92B680D4ADB6A1168E3628B4200D9C6
:1019C00013609A00D3189B00F1184A689068A260CF
:1019D000E060906847609760F25861610132F250B0
:1019E0000120DFE7B8EFFF1F64EFFF1F00F0FF1FCC
:1019F00070B5041E12D01A4B1B68984201D072B603
:101A0000FEE7036C002B01D172B6FEE7C16AC26B20
:101A1000013B0364914201D0002B01D0002070BD36
:101A2000051D281CFEF79AF9E36B0422D21AA26165
:101A30000C4AE36211688B4200D913609A000A498C
:101A4000D3189B00C81842689668A260E660966842
:101A500075609560CA5860610132CA500120DEE7A6
:101A6000B8EFFF1F00F0FF1F64EFFF1F70B5041EEB
:101A70000DD0026C002A01D172B6FEE7C36B994209
:101A800000D2191CE36A8B4201D0012A00D070BD3C
:101A9000174A1268944228D0A069E162002802DB4C
:101AA0000422511AA1619A00D318124D9B00626959
:101AB000EB189A42EBD1261D301CFEF74FF90E4A67
:101AC000E36A11688B4200D913609A00D3189A0018
